:02000004100DDD
:1000000000C00208DF4E0D100D0000004D4F0D1016
:1000100000000000000000000000000000000000E0
:10002000000000000000000000000000494F0D101B
:100030000000000000000000494F0D10494F0D1056
:10004000494F0D10494F0D10494F0D10494F0D10DC
:10005000494F0D10494F0D10494F0D10494F0D10CC
:10006000494F0D10494F0D10494F0D10494F0D10BC
:10007000494F0D10494F0D10494F0D10494F0D10AC
:10008000494F0D10494F0D10494F0D10494F0D109C
:10009000494F0D10494F0D10494F0D10494F0D108C
:1000A000494F0D10494F0D10494F0D10494F0D107C
:1000B000494F0D10494F0D10494F0D10494F0D106C
:1000C00010B5064C2378002B07D1054B002B02D02E
:1000D000044800E000BF0123237010BDECA7020814
:1000E00000000000B4E10D10044B10B5002B03D04C
:1000F0000349044800E000BF10BDC04600000000F6
:10010000F0A70208B4E10D100021124B124A10B5FD
:10011000D8601C68002C06DB914202D101204042CD
:1001200010BD0131F5E79142F8D00121996000211D
:100130001C69002C03DA9142F0D00131F8E79142BA
:10014000ECD0A0220368120600209342E8D01800E9
:10015000E6E7C04600002340983A00001FB50023A0
:100160000193D82300049B05C018029001AB02A89C
:100170000C000393FFF7C8FF002801D1019B236007
:1001800004B010BD13B5084BC47A986801A9C0B279
:10019000FFF7E4FF002803D1019B9C42804116BD7C
:1001A00001204042FBE7C04620AE02081FB5064BC7
:1001B0000004C018029001AB02A801910393FFF75D
:1001C000A3FF05B000BDC0460001003610B5034BCB
:1001D000C17A9868C0B2FFF7E9FF10BD20AE0208EF
:1001E000F0B50F000400002685B0BE4201D100200A
:1001F0003EE0A0221F4BD2009A582378032A04D055
:10020000092B02D801361034EFE71B4A0A33DB0012
:1002100099580029F6D0D3185B6801AD2B7163782B
:1002200001916B71A3782900AB71E378A068EB7141
:1002300023792B7263796B72E3886B8102F0D8FBB0
:10024000002815D1237B2900AB71637BA068EB717B
:10025000E3896B8102F072FB002809D1A06802F0EB
:100260004DFC002804D1A06802F030FC0028C9D061
:1002700005B0F0BD0000214020AE020870B50600B8
:100280000024104AA3019B180F491A68A3015B18A8
:100290001B68002A04DA0134102CF2D1002070BD52
:1002A000002BF8DB094B3100E518AD01280002F006
:1002B00045FB0028F3D1280002F008FC0028EAD012
:1002C000EDE7C04604202440242024408090000113
:1002D00073B50E0004000025B54201D1002076BDA3
:1002E0006A462378694613706378E0685370A37890
:1002F0009370E378D370A388938002F093FE002874
:10030000EDD16A46A37969461370E379E0685370CA
:10031000237A93706389938002F028FE0028DED14F
:10032000E06802F0F5FE0028D9D1E06802F0D6FEC0
:1003300010340028D3D10135CEE773B50E00040088
:100340000025B54201D1002076BD6A462378694672
:1003500013706378E0685370A3789370E378D37078
:10036000A388938002F05EFD0028EDD16A46A37950
:1003700069461370E379E0685370237A9370638958
:10038000938002F0F3FC0028DED1E06802F0CAFDA1
:100390000028D9D1E06802F0A1FD10340028D3D1A3
:1003A0000135CEE7F0B50F000400002685B0BE424F
:1003B00002D1002005B0F0BD236801AD019323797F
:1003C00029002B71637960696B71A379AB71E37953
:1003D000EB71237A2B72637A6B7263896B8102F003
:1003E00005FC0028E6D1237B2900AB71637B6069A3
:1003F000EB71A37B2B72238A6B8102F097FB0028A1
:10040000D8D1606902F08EFC0028D3D1606902F077
:1004100065FC18340028CDD10136C8E730B5174B3C
:1004200085B001930D2301AD2B71437804006B71EE
:1004300083782900AB71C378EB7103792B72437910
:100440006B72C38880686B8102F0D2FA002813D1E6
:10045000237B2900AB71637BA068EB71E3896B811F
:1004600002F06CFA002807D1A06802F047FB0028D0
:1004700002D1A06802F02AFB05B030BD00C002081E
:10048000B02310B55B055B78124C232B1BD00B21DE
:100490002000FFF7A5FE00281AD10F48FFF7EEFE57
:1004A000002815D10A210D48FFF712FF00280FD1AF
:1004B00004210B48FFF741FF002809D10121094819
:1004C000FFF770FF04E02000FFF7A8FF0028DED050
:1004D00010BDC0466CC70D1068C60D1074C60D1057
:1004E00014C70D1054C70D1010B501210148FFF7B6
:1004F00077FE10BD1CC80D100022124B124910B51A
:10050000D8601C68002C05DB8A4201D1012010BD97
:100510000132F6E78A42F9D001229A6000220B49A3
:100520001C69002C03DA8A42F0D00132F8E78A42D3
:10053000ECD0A0220368120600209342E7D01800F6
:10054000E5E7C04600002340983A00000094357764
:1005500010B5D42488B005930A9BA40506930B9B81
:100560000094029002AC68460194039104920793B0
:10057000FFF7C2FF08B010BD00B5064B89B000936D
:10058000029002AB6846019303910492FFF7B4FF17
:1005900009B000BD000B003510B5074C88B00094C1
:1005A000029002AC68460194039104920593FFF710
:1005B000A3FF08B010BDC046000E003500B5064BC5
:1005C00089B00093029002AB6846019303910492B4
:1005D000FFF792FF09B000BD000C003510B588B0E0
:1005E00005930A9B074C06930B9B0094029002AC68
:1005F00068460194039104920793FFF77DFF08B0CA
:1006000010BDC046000D003500B5054B89B0009304
:10061000029002AB68460193FFF76EFF09B000BD80
:10062000000A003500B5054B89B00093029002AB7B
:1006300068460193FFF760FF09B000BD0005003573
:1006400000B5064B89B00093029002AB6846019357
:1006500003910492FFF750FF09B000BD000400357C
:100660001FB5054B02900093684602AB01930391BE
:10067000FFF742FF05B000BD001000357FB5064B07
:100680000390019301A803AB029304910592FFF735
:1006900033FF07B000BDC0460011003510B5074C50
:1006A00086B00094029002AC6846019403910492D3
:1006B0000593FFF721FF06B010BDC04600120035BC
:1006C00010B5074C86B00094029002AC68460194C5
:1006D000039104920593FFF70FFF06B010BDC046CB
:1006E000000900357FB5054B0390019301A803ABCA
:1006F0000293FFF701FF07B000BDC04600060035BA
:100700007FB5064B0390019301A803AB02930491BC
:100710000592FFF7F1FE07B000BDC04600070035A7
:100720007FB5054B0390019301A803AB029304919D
:10073000FFF7E2FE07B000BD000800357FB5064BAD
:100740000390019301A803AB029304910592FFF774
:10075000D3FE07B000BDC0460002003510B5074CFF
:1007600086B00094029002AC684601940391049212
:100770000593FFF7C1FE06B010BDC046000100356D
:1007800010B58CB006930E9B0A4C07930F9B0194F7
:100790000893109B03900993119B03AC0A93129B3F
:1007A00001A80294049105920B93FFF7A5FE0CB0EB
:1007B00010BDC04600030035F0B58DB01D0012AB72
:1007C00040CB02921B780F000393002305AA04A9D3
:1007D0000493059300F03DF9041E3BD1204B3A00F1
:1007E00000930599029B049807F050F8002834DD27
:1007F000022007AA06A9FF300694079401F0AEF97B
:10080000002803D12900069800F0F4FF812007AAF0
:1008100006A9400001F0A2F9652400281ED131008C
:10082000069800F077FD041E14D108A9380000F0E6
:1008300028F9041E0ED131000B9800F063FB041E52
:1008400008D1039A29000B9800F03AF9040008989F
:1008500006F0B2FF20000DB0F0BD14246442F9E7A9
:10086000005F2D00F0B51F00002387B002910392B6
:1008700004A905AA0493059300F0EBF8041E2ED1F9
:10088000059800F07FF8040007F00EFC051E31D03B
:100890001A4B0200009305992300049806F0F6FF16
:1008A000002822DD280006F0E1FF061E20D001000E
:1008B000134800F09FF8002814D00069002811D0D8
:1008C000039B220000930197029B2900FFF774FF0E
:1008D0000400300006F070FF280007F0EFFB200056
:1008E00007B0F0BD01246442F3E714246442F3E747
:1008F0000524FBE764246442F1E7C046005F2D0055
:100900002CC80D1010B5010004000B4808F076FA51
:10091000002398420DD02100084808F06FFA012307
:10092000002806D02100064808F068FA43424341F7
:100930005B00180010BDC04633C90D103CC90D1036
:1009400048C90D1010B5010004000B4808F056FA14
:10095000002398420DD02100084808F04FFA0123E7
:10096000002806D02100064808F048FA43424341D7
:100970005B00180010BDC0464DC90D1056C90D10C2
:100980005EC90D1003235843800898430430704714
:10099000F8B5C3680D000860062B21D18468124F9A
:1009A000002C01D12000F8BD266A002E06D03100AF
:1009B0000E4808F023FA002802D16C602468EFE7A3
:1009C00031000B4808F01AFA002801D1AC60F5E7B5
:1009D0003100380008F012FA0028EFD1EC60EDE7A2
:1009E00002204042DFE7C04675C90D1066C90D10F0
:1009F0006CC90D10F0B507000D00002491B001AED8
:100A0000002D02D1280011B0F0BD296A002904D0C0
:100A1000380008F0F3F90028F4D0AB68002B06D0BA
:100A20000E2C12D8A200955101341D00E8E72B6866
:100A3000002BFAD1002C0AD0013CA3009B591B6863
:100A4000002BF2D1002CF7D1EFE70025DAE72500E3
:100A5000D8E7F8B50E002E21170008F0C1F9041EE2
:100A60000CD0451C2E21280008F0BAF9002805D02A
:100A7000001B0138386000203560F8BD1620404268
:100A8000FBE770B5050000200C0006F07BFE280097
:100A900006F0ECFE002803D02100FFF779FF70BDBF
:100AA00005204042FBE7002304220133002901D145
:100AB000904203D952001D2BF7D102331800704722
:100AC000F0B589B005900C000100C24807920027DC
:100AD000FFF790FFB84200D145E18568069702957F
:100AE0000497029B002B00D08AE0EB68062B00D015
:100AF00039E12E00B84F31003800FFF77BFF079A2D
:100B0000037E9A4200D0DEE03100B448FFF772FF66
:100B10008369237029003800FFF76CFF2278037E79
:100B20009A4200D1A8E12D68002DF3D12900AC48EC
:100B3000FFF760FF002806D02300FF335B7B012B0B
:100B400001D18369A3602900A648FFF753FF00285D
:100B500008D02300FF339B7A012B03D1C3685A1EB0
:100B6000934163702900A048FFF744FF002808D094
:100B70002300FF331B7B012B03D1C3685A1E934113
:100B8000E37029009948FFF735FF002806D02300BD
:100B9000FF331B7B012B01D183692371290094480A
:100BA000FFF728FF002809D02300FF331B7E012B0D
:100BB00004D1C3685A1E9341E21CD37729008D48A3
:100BC000FFF718FF002800D1A6E0C368052B00D06E
:100BD000A2E082682300200012331530FF33FF307B
:100BE000002A00D198E01978012903D119009669EB
:100BF000F5390E700133984200D18DE01268EFE7AD
:100C000002997D48FFF7F6FE002804D0836801931F
:100C1000019B002B03D1029B1B68029361E70199A2
:100C20007648FFF7E7FE00284AD0036974491800A8
:100C3000039308F0E3F8002842D07249039808F0C3
:100C4000DDF800283CD000266F4AB300995803987D
:100C500008F0D4F8071E05D00136172EF4D1052769
:100C6000183E7F4201996948FFF7C4FE002801D071
:100C70008369069301996648FFF7BCFE002804D0FB
:100C8000C1698069FFF70FFF0490731C18D0049BA3
:100C9000002B15DD92227300E31852009A5C012AA2
:100CA00004D1320006990A32D20011512622FF32B5
:100CB0009B5C012B04D10A36F600049BA6197360D5
:100CC000019B1B68A3E73668002E00D012E721E7DE
:100CD0004C49380008F092F8002800D0FFE03100BD
:100CE0004A48FFF787FE002806D02300FF331B7C0D
:100CF000012B01D18369636131004548FFF77AFE1A
:100D0000002800D1EBE02300FF331B7C012B00D037
:100D1000E5E08369A361E2E029003E48FFF76AFE4F
:100D2000002817D0C368052B14D182682300200047
:100D300015331830FF33FF30002A0BD01978012902
:100D400003D119009669F5390E700133984201D02C
:100D50001268F1E729003048FFF74CFE002835D033
:100D600000278369A37005992C48FFF743FE0028EC
:100D700058D000258668002E54D031002448FFF753
:100D800039FE00280BD063191A001A32FF3212788C
:100D9000012A04D102326A439B1882699A623100A7
:100DA0001F48FFF727FE00280BD063191A001932DD
:100DB000FF321278012A04D102326A439B188269F9
:100DC0005A6202350A2D2DD03668D4E7A07007008C
:100DD000C9E7C04633C90D109CC80D1051C80D108D
:100DE00058C80D107AC90D1062C80D106AC80D10D0
:100DF00079C80D1080C80D1035C80D1082C90D10AE
:100E00003FC80D1044C80D10C0A00208D2C90D1073
:100E10004CC80D108AC80D1097C80D109FC80D1032
:100E2000A9C80D1005992F48FFF7E4FD051E20D035
:100E300001002D48FFF7DEFD00280AD02423FF33F0
:100E4000E35C012B05D1C3685A1E934122004D3249
:100E5000137029002548FFF7CDFD002809D0912304
:100E60005B00E35C012B04D1C3684C345A1E9341F0
:100E70002370380009B0F0BD29001D48FFF7BAFD06
:100E8000002800D152E68668002E00D14EE63100DF
:100E90001848FFF7AFFD002821D007691649380030
:100EA00007F0ACFF002800D012E731001348FFF72D
:100EB000A1FD002806D02300FF339B7B012B01D12D
:100EC0008369E36031000E48FFF794FD002806D0E7
:100ED0002300FF33DB7B012B01D18369236136685B
:100EE000D2E7C046AFC80D10BBC80D10C7C80D1063
:100EF00035C80D1082C90D103FC80D10D2C90D1094
:100F00004CC80D10F8B507000C000100BA48FFF7F7
:100F100071FDBA4E051E2AD001003000FFF76AFDB0
:100F2000002808D0230068331B78012B03D1006907
:100F3000FFF708FD20702900B148FFF75BFD00288E
:100F400008D0230069331B78012B03D10069FFF718
:100F5000D9FC60702900AB48FFF74CFD002806D093
:100F600023006A331B78012B01D18369A3703900F8
:100F7000A548FFF73FFD051E2AD001003000FFF70E
:100F800039FD002808D023006B331B78012B03D1D7
:100F90000069FFF7D7FCE07029009948FFF72AFDA8
:100FA000002808D023006C331B78012B03D1006983
:100FB000FFF7A8FC207129009248FFF71BFD0028CD
:100FC00006D023006D331B78012B01D18369637137
:100FD00039008E48FFF70EFD051E00D184E00100A8
:100FE0003000FFF707FD002808D023006E331B7880
:100FF000012B03D10069FFF7A5FCA07129008048EF
:10100000FFF7F8FC002808D023006F331B78012B72
:1010100003D10069FFF776FCE07129007948FFF7FA
:10102000E9FC002806D0230070331B78012B01D186
:101030008369237229007648FFF7DCFC002808D07A
:10104000230071331B78012B03D1C3685A1E9341CF
:10105000637229006F48FFF7CDFC002808D02300F9
:1010600072331B78012B03D1C3685A1E9341A372BC
:1010700029006948FFF7BEFC002808D0230073331D
:101080001B78012B03D1C3685A1E9341E3722900D8
:101090006248FFF7AFFC002808D0230074331B78A8
:1010A000012B03D1C3685A1E9341237329005C4866
:1010B000FFF7A0FC002808D0230075331B78012B14
:1010C00003D1C3685A1E9341637329005548FFF743
:1010D00091FC002808D0230076331B78012B03D124
:1010E000C3685A1E9341A37339004F48FFF782FC2F
:1010F000050001003000FFF77DFC002808D0230028
:1011000077331B78012B03D10069FFF71BFC207498
:1011100029003C48FFF76EFC002808D023008C33E0
:101120001B78012B03D12300826964331A702900D4
:101130003E48FFF75FFC00282AD000268768002F72
:1011400026D039003A48FFF755FC00280AD0A319E9
:101150001A0078321278012A04D1023272439B18A5
:1011600082695A6139003348FFF744FC00280AD0ED
:10117000A3191A0079321278012A04D1023272437B
:101180009B1882699A6102360A2E01D03F68D6E721
:1011900029002948FFF72EFC00282BD00025032723
:1011A0008668002E26D031002148FFF723FC002856
:1011B0000AD063191A0082321278012A04D13A0047
:1011C0006A439B188269DA6331001A48FFF712FC00
:1011D00000280AD063191A0083321278012A04D138
:1011E0003A006A439B1882691A6402350A2D01D0BD
:1011F0003668D6E70020F8BDD9C80D10DDC80D103F
:10120000E8C80D10F0C80D10F4C80D10F7C80D1087
:10121000FEC80D1006C90D1025C90D10E3C90D102B
:10122000EDC90D10F4C90D100BC90D100FC90D102B
:10123000A9C80D104CC80D101DC90D1070B50400C3
:101240000D0086B00021142201A806F06BFF2900D2
:101250002000FFF7CFFB0400002C18D021001C4811
:10126000FFF7C8FB0028F7D00569002D0AD0194EFA
:101270002900300007F0C2FD00280BD1310001A881
:1012800007F0C6FD210001A8FFF7B4FB0400200011
:1012900006B070BD104E2900300007F0AFFD0028E9
:1012A000ECD029000D4807F0A9FD0028E6D00C4E2F
:1012B0002900300007F0A2FD0028DFD029000948EE
:1012C00007F09CFD0028DDD121000748C1E7C0469A
:1012D00082C90D10AAC90D1093C90D109AC90D101D
:1012E000A2C90D1087C90D108DC90D1010B5FFF7DB
:1012F00081FB0124002809D08168002906D0044818
:10130000FFF778FB002801D0C468E4B2200010BDCC
:101310002BC90D10F0B5050085B000200C0006F0BB
:1013200031FA280006F0A2FA0190002800D14BE221
:101330000100A148FFF75EFB051E00D0B4E00123C9
:101340005B42009301999D48FFF754FB051E00D0B6
:10135000EEE001235B42009301999948FFF74AFBB5
:10136000051E00D03EE101235B42009301999548A0
:10137000FFF740FB071E00D122E2934E0100300030
:10138000FFF75CFF390005003000FFF7AFFF0600F4
:10139000002D00D1F6E12869FFF7D4FA2300773356
:1013A00020741E70894E39003000FFF747FF390066
:1013B00005003000FFF79AFF002D00D1E6E1230081
:1013C000AA6964331A702833187039008048FFF70F
:1013D00011FB051E00D1E6E101007E48FFF72EFF5C
:1013E000290006007B48FFF781FF0390002E00D103
:1013F000D0E1B369029329007748FFF71FFF290066
:1014000006007548FFF772FF002E00D1C7E1B669EC
:10141000230022002100143378323C31029D5E60AB
:101420001D606D462D7B0833507015700232994255
:10143000F4D139006948FFF7DDFA061E00D1BFE19B
:10144000644F01003800FFF7F9FE31000500380055
:10145000FFF74CFF0390002D00D1A8E1AB69029388
:101460005D4F31003800FFF7E9FE3100050038001C
:10147000FFF73CFF002D00D19EE1AD692300220063
:101480003C338232643402995D6019606946097B9D
:101490000833507011700232A342F4D1019806F063
:1014A0008BF9009805B0F0BD474F01003800FFF7F9
:1014B000C5FE290006003800FFF718FF0700002EC0
:1014C0002FD03069FFF73EFA2300683320701F7079
:1014D0000023434F290038000093FFF7AFFE290097
:1014E00006003800FFF702FF0700002E1CD030690D
:1014F000FFF708FA2300693360701F70334F29002B
:101500003800FFF79BFE290006003800FFF7EEFECB
:10151000002E00D113E7B369A37023006A3318705B
:1015200010E701235B42D4E701235B420093E5E728
:10153000254F01003800FFF781FE29000600380022
:10154000FFF7D4FE0700002E2DD03069FFF7FAF91F
:1015500023006B33E0701F70214F29003800FFF724
:101560006DFE290006003800FFF7C0FE0700002EC0
:101570001DD03069FFF7C6F923006C3320711F704E
:10158000124F29003800FFF759FE290006003800E5
:10159000FFF7ACFE002E00D1DBE6B36963712300D8
:1015A0006D331870D8E601235B420093D4E7012322
:1015B0005B420093E4E7C046D9C80D10F4C80D1093
:1015C000F7C80D100BC90D10DDC80D10F0C80D10B7
:1015D0000FC90D10A9C80D104CC80D101DC90D1054
:1015E000E8C80D107A4F01003800FFF727FE2900E8
:1015F00006003800FFF77AFE0700002E00D1A1E0B8
:101600003069FFF79FF923006E33A0711F70714F8F
:1016100029003800FFF712FE290006003800FFF706
:1016200065FE0700002E00D190E03069FFF76AF9EF
:1016300023006F33E0711F70674F29003800FFF7F8
:10164000FDFD290006003800FFF750FE002E00D1F6
:1016500080E0B36923722300703318705F4F290054
:101660003800FFF7EBFD290006003800FFF73EFECB
:10167000002E73D0F3685A1E9341637223007133B6
:101680001870574F29003800FFF7D8FD29000600D1
:101690003800FFF72BFE002E64D0F3685A1E9341EA
:1016A000A3722300723318704E4F29003800FFF7E1
:1016B000C5FD290006003800FFF718FE002E55D0A2
:1016C000F3685A1E9341E372230073331870464F38
:1016D00029003800FFF7B2FD290006003800FFF7A7
:1016E00005FE002E46D0F3685A1E93412373230053
:1016F000743318703D4F29003800FFF79FFD290013
:1017000006003800FFF7F2FD002E37D0F3685A1EAE
:1017100093416373230075331870354F29003800E7
:10172000FFF78CFD290006003800FFF7DFFD002ED3
:1017300000D118E6F3685A1E9341A3732300763351
:10174000187013E601235B42009360E701235B42BC
:10175000009371E701235B4200937FE701235B4223
:1017600000938EE701235B4200939DE701235B42D8
:101770000093ACE701235B420093BBE701235B428C
:101780000093CAE701235B4200930BE601235B420F
:1017900000931AE601235B42029600932BE6012395
:1017A0005B42009334E601235B42009341E6012350
:1017B0005B420295009353E601235B4200935DE692
:1017C00001235B42009369E605235B42009368E6D0
:1017D000DDC80D10E8C80D10F0C80D10FEC80D10C2
:1017E00006C90D1025C90D10E3C90D10EDC90D1066
:1017F000F4C90D10F0B5050085B000200C0005F00F
:10180000C1FF280006F032F80190002800D181E1E4
:101810000100C248FFF7EEF8051E00D13AE1C04FC3
:1018200001003800FFF70AFD290006003800FFF725
:101830005DFD002E00D109E1B36923702300FF3361
:1018400058720023B74F290038000093FFF7F6FCC9
:10185000290006003800FFF749FD002E00D1F8E00E
:10186000F3685A1E934163702300FF339872AE4FA2
:1018700029003800FFF7E2FC290006003800FFF7D6
:1018800035FD002E00D1E8E0F3685A1E9341E37065
:101890002300FF331873A54F29003800FFF7CEFC53
:1018A000290006003800FFF721FD002E00D1D8E006
:1018B000B369A3602300FF3358739D4F290038009C
:1018C000FFF7BCFC290006003800FFF70FFD002ED3
:1018D00000D1CAE02200B369FF32DBB223779074F3
:1018E0006377D074A3771075924F29003800FFF703
:1018F000A5FC290006003800FFF7F8FC002E00D1F7
:10190000B7E02200B369FF32DBB2611CE3775075A8
:10191000CB77A11C9075CB77D075874E290030000E
:10192000FFF78CFC290007003000FFF7DFFC002FD9
:1019300000D1A2E0FB685A1E9341E21CD37723003A
:10194000FF33187601997D48FFF754F80600002F01
:1019500000D19FE023000122794FFF3301009A73E9
:10196000DA731A745A743800FFF768FC3100050006
:101970003800FFF7BBFC0390002D00D181E0AB697C
:101980000293704F31003800FFF758FC310005001A
:101990003800FFF7ABFC002D00D177E0AD692200E5
:1019A00021002300253209315033FF32FF31029EDE
:1019B0005D601E606E46367B0833167050700232D2
:1019C0008B42F4D101996048FFF714F8061E00D14C
:1019D0006DE05E4F01003800FFF730FC310005007C
:1019E0003800FFF783FC0390002D57D0AB690293BA
:1019F000544F31003800FFF721FC3100050038005A
:101A0000FFF774FC002D4ED0AD69220023002100A9
:101A100019322433FF324C31029E5D601E606E46E7
:101A2000367B08335070167002329942F4D1019916
:101A30004748FEF7DFFF051E3DD101235B420093BF
:101A4000019805F0B9FE009805B0F0BD01235B4296
:101A5000F8E601235B42009309E701235B42009310
:101A600019E701235B42009327E701235B420093C0
:101A70003AE701235B4200934FE701235B42009367
:101A800060E701235B42029500937AE701235B4202
:101A9000009384E701235B42009393E701235B42B9
:101AA00002950093A4E701235B420093ADE7012375
:101AB0005B420093BBE7274F01003800FFF7BEFBF6
:101AC000290006003800FFF711FC002E1ED0F36835
:101AD0005A1E934122004C32137091235B00E05454
:101AE0001D4F29003800FFF7A9FB29000600380028
:101AF000FFF7FCFB002EA0D0F3685A1E9341220092
:101B00004D3213702423FF33E05499E701235B42E5
:101B10000093E5E705235B42009394E733C90D107A
:101B20009CC80D107AC90D1062C80D1058C80D1050
:101B300080C80D108AC80D1079C80D1035C80D1059
:101B4000D2C90D104CC80D109FC80D10A9C80D109A
:101B5000AFC80D10C7C80D10BBC80D107FB5DC2372
:101B60009B0500936C46002302AD01950290154839
:101B70006B60C460144C0668002E07DBA34203D1DF
:101B80000120404204B070BD0133F4E7A342F7D016
:101B90000123836000230669002E03DAA342EFD0FD
:101BA0000133F8E7A342EBD0A02300981B0698422C
:101BB00001D00098E6E7029B002013606B680B6081
:101BC000E0E7C04600002340983A0000F0B5170057
:101BD0008A22434C9200A544079008910EA8002148
:101BE000BFB2099306F09EFA0CAA0BA93800FEF7C3
:101BF000A5FD00260500B0422CD1C02280210B9B00
:101C0000D2051A40C9058A4237D10C9BDC1DE40875
:101C100020000D9406F048FA0925061E1AD001008E
:101C20000DAB22003800FEF799FD051E12D16B4660
:101C3000198C102304930293079B079A3033019366
:101C4000284B40320392009332000D9B0EA8FEF702
:101C500097FD0500300006F031FA002D05D1202255
:101C600009990EA8FEF7ECFC05000EA8FEF7DAFCB9
:101C7000280099239B009D44F0BD1B4A934207D145
:101C80000C9B5C0809230134E4085C433B34BFE748
:101C9000164A934203D10C9BDC082934B8E7144A56
:101CA000934205D103240C9BDB085C435A34AFE715
:101CB000104A934205D103240C9BDB085C434A3451
:101CC000A6E70D4A1B0C1B0493429ED00B4A04004E
:101CD00093429DD10C9BDC1DE4081234640097E70D
:101CE0009CFDFFFF0901202200000170000001603F
:101CF000000002700000026000000370000003603A
:101D000070B508000D0014000E1E05D0731B9C4218
:101D100003DCE043C017204070BD307803F024FDA1
:101D20000136F3E770B500240D001600A1420AD178
:101D3000200070BD03F024FDC0B2285501340A28EC
:101D4000F6D00D28F4D0B442F4DBF1E70000000037
:101D50000230800803D001300238FCD1C046C046B2
:101D60007047EFF3108072B6704780F310887047A9
:101D7000014B18607047C046E0AD0208044B1B6879
:101D80001A0008321B68D26F9B181868000E704743
:101D9000E0AD0208054B1B681A0008321B68D26FC1
:101DA0009B181868000AC0B27047C046E0AD020830
:101DB0001D4B98420FD010D840282FD005D80028AE
:101DC00030D0102828D019481EE0802828D0802341
:101DD0005B009842F7D1144816E0154B984214D096
:101DE00008D8A0231B0698421CD0124B9842EAD177
:101DF000A0200BE0104B98420AD0104B984209D01B
:101E00000F4B9842DFD10F487047A420C003FBE777
:101E10000D48F9E70D48F7E70D48F5E70D48F3E7FA
:101E20000D48F1E70020EFE706005200FF005200E6
:101E3000010000F0090000A0040000F0050000F01F
:101E4000030000F0010052000200520003005200A3
:101E500001005000020050000500520070B50A4D0C
:101E600004002B6831331B78834204D8E6210748ED
:101E7000490002F035FC2B681A00B0321088444348
:101E8000186A201870BDC046E0AD0208ECCB0D10FA
:101E900010B50020FFF7E2FF0A4B1C682300B433A3
:101EA0001B68C0180368002B0ADB074B1868FFF794
:101EB0007FFF012263689A609A68002AFCD110BDF6
:101EC0000248FCE7E0AD020808A802080200500042
:101ED0000D4B10B51860002804D0FE235B42038030
:101EE00000234380094B1B681A0050321278002AE5
:101EF00008D051331B78002B04D002220449002063
:101F000000F086FB10BDC04618A80208E0AD02082C
:101F1000C1A3020870B5C4050500E40D28D103F083
:101F200025F8144B144A1A605D609C60DC60134B0A
:101F30001B6854331978002915D0FFF71FFF0400E0
:101F4000FFF728FFFA210134013060430C4B0D4CA0
:101F500089004443186805F08DFD0100200005F05C
:101F600089FD094BC118802040000AF05DFB70BD5F
:101F70000648FCE708A802080001001CE0AD0208C2
:101F800020A1020860F590009808000006005200A9
:101F900070B5C40506000D00E40D2AD1002928D033
:101FA00002F0E4FF144B154A1A605C609E60DD602D
:101FB000134B1B6852331978002915D0FFF7DEFE4A
:101FC0000400FFF7E7FEFA210134013060430D4BB6
:101FD0000D4C89004443186805F04CFD01002000B9
:101FE00005F048FD094BC118802040000AF01CFB99
:101FF00070BD0748FCE7C04608A8020800010005BC
:10200000E0AD020820A10208C0EA21014826000034
:102010000600520070B506000C001500072903D910
:102020001449154802F05CFB1F232A009A4303D091
:102030001249114802F054FB114B1B689A695B6905
:10204000B01AC0090001C0181F231D40032C07D877
:10205000E400A340A54002689A431543056070BDA3
:10206000043CE400A340A54042689A431543456000
:10207000F5E7C046910200009ECC0D1092020000D0
:10208000E0AD0208F0B585B000900D001400002806
:1020900000D138E1002A00D135E1072903D94E21CA
:1020A0009A4802F01DFB2368012B03D94F21974862
:1020B00002F016FB0F2362689A4303D05021934825
:1020C00002F00EFB1F22237A934303D051218F4845
:1020D00002F006FBE368032B03D952218B4802F080
:1020E000FFFA2369012B03D95321884802F0F8FA3B
:1020F0006369012B03D95421844802F0F1FAA369E2
:10210000012B03D95521814802F0EAFAE369032B38
:1021100003D956217D4802F0E3FA236A012B03D943
:1021200057217A4802F0DCFA636A012B03D958215F
:10213000764802F0D5FAA36A012B03D959217348D6
:1021400002F0CEFAE36A032B03D95A216F4802F05A
:10215000C7FA236B072B03D95B216C4802F0C0FA46
:102160002668072D04D9CC216948890002F0B8FA05
:102170000122AA400192012E07D96649644802F063
:10218000AFFA009B019A9A6004E0002EF9D1009BFF
:10219000019A5A606668072D03D95F495C4802F0CE
:1021A0009FFA0F2332009A4303D05C49584802F04B
:1021B00097FA0F215A4FAB0002933B6808007D331A
:1021C0001A78009B0E40D2181368A9009C46AB00F9
:1021D000984063468E4083431E431660227A29004E
:1021E0000098FFF717FFE668082D03D94D494848C6
:1021F00002F076FA032E03D94B49454802F070FAF3
:10220000032108006B0003933B686F00B8400E4049
:10221000BE407C331A78009B9A18136883431E4390
:1022200016602669082D03D94049394802F058FA4A
:10223000012E03D93E49364802F052FA019A009B1A
:10224000D74301221640AE409B693B401E43009B92
:102250009E616669072D03D936492D4802F040FA80
:10226000012E03D934492A4802F03AFA01202C4BB6
:1022700006401968AE400B0084467E331B78009AF6
:10228000D3181A68174037431F600B0062467F332C
:102290001878009B6E001818A36910361340AB40E5
:1022A000E56902321540B540B2402B43019D0768F5
:1022B0002A4397433B4303600220042580310A7878
:1022C000009B9A18636A11685B000340A06A800053
:1022D000284003436046256A284018250343E06AE6
:1022E000C00028400343206BFF24400120400343EB
:1022F000FE20029D80000540AB400020A1430B431F
:10230000136005B0F0BD0D48FBE7C04647CC0D108B
:102310009ECC0D1031030000CD030000CE03000061
:10232000E0AD0208F1060000F206000072060000AF
:10233000730600000C0400000D04000001005A00A8
:102340000B4B70B51B680500B4331B680C00C31839
:102350001B68002B09DA0B0C03D00649064802F073
:10236000BFF90020A4B26C6070BD0448FCE7C04611
:10237000E0AD0208DE020000ECCB0D1001008A0087
:10238000036870B505000C00002B0BDAC2600B0C63
:1023900004D0B1210448890002F0A2F90020A4B2BF
:1023A000AC6070BD0148FCE7ECCB0D1001008A0069
:1023B00070B505000C1E03D1A221084802F090F967
:1023C000074B1B68B4331B68EB181B68002B03DA40
:1023D0000020EB68236070BD0248FCE7F6CC0D10CE
:1023E000E0AD020801008A00024B1A68002A00D101
:1023F000186070471CA80208F0B5314D1F002B680B
:1024000085B0040002910392002B03D1BE212D4818
:1024100002F066F92C23FF225C432B683D001C1957
:102420003B0A3F0CA760284F134063603B68154090
:10243000256031331B789D4204D3E62123484900AF
:1024400002F04EF93B681A00B032128855431A6AFE
:102450003233AD1825611B7865689D4204D3F421A1
:102460001A48490002F03CF93B681E6A2B00803391
:102470005B01F3186361A36801931B0C09D0134F30
:102480001349380002F02CF982213800890002F04B
:1024900027F9019B6D011B041A0C13430D4A751992
:1024A000AD182B60039BE361029B23620023A361B1
:1024B0000A9B002B01D01B88A38105B0F0BDC0464C
:1024C0001CA8020850CD0D10E0AD0208ECCB0D1099
:1024D0000702000008100000F0B5040085B00028D5
:1024E00003D15B21214802F0FBF86368032B03D979
:1024F0005D211E4802F0F4F8E36A002B03D161214C
:102500001A4802F0EDF8236B002B03D16221174823
:1025100002F0E6F8A36802AD2B80154B22681B6819
:10252000E16ADB8EE0689B18AB706368A26A039374
:1025300000952369266A676AFFF75EFF00213B006A
:102540000A0000913000FFF757FF216B280002F0CE
:102550004FF80022AB5E002B06DB1F2213401E3A11
:102560009A401300034A136005B0F0BD50CD0D1022
:10257000E0AD020800E100E0F7B504000F00151E11
:10258000019304D183211D48490002F0A9F81C4E93
:102590003368002B04D108211848FF3102F0A0F85D
:1025A0002C235C4332685F4314192669D719002E27
:1025B00020D0BB69002B1FD13368002B1CDA01220D
:1025C0006368140011009C407B6899402B680904E3
:1025D0009BB20B432B60019BF5607B62BA61230CBD
:1025E00004D0B1210748890002F07AF80020A4B293
:1025F000B460FEBD0448FCE70448FAE750CD0D1076
:102600001CA80208ECCB0D1004028A0007028A0005
:10261000F8B5114F04003B680E001500002B04D1E3
:1026200068210E48FF3102F05BF82C2060433C68C3
:102630002418236A002B04D16C210848FF3102F0D2
:102640004FF8E369AB4204D90020236AAD00EE5095
:10265000F8BD0348FCE7C0461CA8020850CD0D1089
:102660000A028A00002373B504000193984204D142
:10267000ED212C48490002F033F82369002B04D1E6
:10268000DC212848FF3102F02BF86369002B04D1CC
:10269000EE212448490002F023F8236A002B04D1DC
:1026A000DE212048FF3102F01BF86269D5682B0C4F
:1026B00022D01B04136013681B4B20691B68B433C2
:1026C0001B68C3181B68002B16DA01A9FFF770FE00
:1026D0000026B0420CD10198E26903681E0CDBB2FF
:1026E0009A4205D9226A9B009B58002B00D098473C
:1026F00031002069FFF724FEADB2002D09D06369D7
:102700001D6000251B68636AAB4205D0984765626F
:10271000A56163691B6873BDA36A002BF8D0984755
:10272000F6E7C04650CD0D10E0AD020870B5084C7C
:1027300005002368002B04D1DD210648490001F083
:10274000CFFF2C20454320684019FFF78BFF70BD59
:102750001CA8020850CD0D1070B50A4D04002B685E
:1027600031331B78834204D8E6210748490001F041
:10277000B7FF2B681A00B03210884443186A20183B
:1027800070BDC046E0AD0208ECCB0D10F8B5174B9C
:102790000D001B6831331B78834225D9002923D0D3
:1027A0001F240B681C401FD1FFF7D6FF07002B68C2
:1027B0000F4EDA0821003060686805F0B3FC210094
:1027C0003800FFF7BDFD21002A003068FFF7D8FD73
:1027D000041E07D101003068FFF7B2FD030020009E
:1027E000002B00D00348F8BD0348FCE7E0AD020829
:1027F00020A8020801018A0003018A00F7B5184FDA
:1028000004003B680191DE683368834226D90025C5
:10281000A94202D1FFF7A5FA050038680368002B2A
:102820001ADA1F2201232240934064097268A4002F
:102830001419226813420DD09A432260002400210B
:10284000FFF77EFD019B002B02D12800FFF78DFAD8
:102850002000FEBD034CF2E7034CF3E7034CF7E71F
:1028600020A80208020188000301880004018A00F0
:102870000A4B1B68DB681A6882420DD959681F230E
:10288000420918401E3B8340920050581840431E96
:102890009841034BC01870470248FCE720A8020883
:1028A0000001880004018A0070B5154E04003368E9
:1028B0000D009B6CC340DB0703D4A721114801F036
:1028C0000FFF0F2D03D9A8210E4801F009FFF022B8
:1028D0002B041203290013400F2211400B433168CF
:1028E000A402096964188021C9016350605810402E
:1028F000401B431E9841044B4042184070BDC046E7
:10290000E0AD0208ABCD0D100300C20070B5094D5B
:1029100004002B689B6CC340DB0703D4C721064827
:1029200001F0DEFE2B6810341B69A402E0580F236F
:10293000184070BDE0AD0208ABCD0D1070B50400BD
:102940000D00002804D17A212448FF3101F0C8FE8F
:102950006B89DB0B04D0BD212048490001F0C0FE8B
:102960000222AB799343012B04D07C211B48FF3119
:1029700001F0B6FE0222EB799343012B04D0BE2175
:102980001648490001F0ACFE6A897F231100994383
:1029900022D10721AB7952020B4013436A7A3131BD
:1029A00092071343EA79D2000A4013430122297A9D
:1029B0004A40920113431A0009490A409A420BD136
:1029C0006262606A0840801A43425841054B4042A7
:1029D0001840054BC01870BD0448FCE7ABCD0D1086
:1029E000DBFEFFE0FDFF3DFF0300C2000100C2006F
:1029F00070B504000D00002804D1C2212E48FF311B
:102A000001F06EFE6B89DB0B04D0E1212A484900FE
:102A100001F066FEAB79072B04D9C4212648FF31AB
:102A200001F05EFEEB79072B04D9E2212248490030
:102A300001F056FE2B79073B182B04D9C6211E48FE
:102A4000FF3101F04DFE6B897F22190091430A1E70
:102A50002ED12968FF3291430A006979A8790A4387
:102A600007215B02084018436B7A31319B071843FA
:102A7000EB79DB000B4018430123297A4B40F82106
:102A80009B0118432B7949051B060B4003436360E8
:102A90002260216891420DD16068084A1040C01A36
:102AA00043425841064B40421840064BC01870BD87
:102AB0000548FCE70348FAE7ABCD0D10FFFEFFFF2A
:102AC000FDFF3DFF0300C2000100C20010B5041E5F
:102AD00004D1FF210748490001F002FE8023626A09
:102AE0001B0613436362606A034BC00F0138184032
:102AF00010BDC046ABCD0D100300C20010B5041EC2
:102B000003D10749074801F0EBFD802362681B06EB
:102B1000134363606068044BC00F0138184010BD58
:102B20004E020000ABCD0D100300C20070B50400D2
:102B30000D00002803D12449244801F0D1FD0222D0
:102B4000AB799343012B04D0A5212048C90001F0A3
:102B5000C7FD0222EB799343012B03D01C491B488C
:102B600001F0BEFD1B4B1B682F331A78012A26D1BA
:102B700069897F230800984323D10720AB79490254
:102B800003400B43697A313089070B43E979C90067
:102B900001400B43297A4A40920113431A000E491F
:102BA0000A409A420DD16262606A0840801A43422C
:102BB00058410A4B40421840094BC01870BD0948A3
:102BC000FCE70948FAE7C04627050000ABCD0D1029
:102BD00029050000E0AD0208DBFEFFE0FDFF3DFF40
:102BE0000300C2000200C2000100C20070B505006F
:102BF0000C00002803D12F492F4801F071FDA37963
:102C0000032B03D92D492C4801F06AFDE379032BEE
:102C100003D92B49284801F063FD2379073B182B82
:102C200004D9AF212448C90001F05AFD254B1B6887
:102C30002F331A78012A36D161897F2308009843FF
:102C400033D10720A379490203400B43617A313025
:102C500089070B43E179C90001400B43217A4A40BF
:102C6000F821920113432279490512060A401343C1
:102C70001A0015490A409A4217D1FF232068984349
:102C8000030060796A6003432B60286898420ED184
:102C900068680840801A434258410C4B4042184033
:102CA0000B4BC01870BD0B48FCE70B48FAE708480F
:102CB000F8E7C04675050000ABCD0D1076050000A5
:102CC00077050000E0AD0208DBFEFFFFFDFF3DFFE2
:102CD0000300C2000200C2000100C20010B5041EC1
:102CE00003D10B490B4801F0FBFC0B4B1B682F3346
:102CF0001B78012B0AD18023626A1B06134363628F
:102D0000606A064BC00F0138184010BD0448FCE74C
:102D1000BD050000ABCD0D10E0AD02080300C20000
:102D20000200C20010B5041E03D10B490B4801F08C
:102D3000D7FC0B4B1B682F331B78012B0AD1802348
:102D400062681B06134363606068064BC00F01385E
:102D5000184010BD0448FCE716060000ABCD0D106E
:102D6000E0AD02080300C2000200C20070B504001A
:102D70000D00002803D12149214801F0B1FC2B7836
:102D8000032B03D91F491E4801F0AAFC6B78032BC3
:102D900003D91D491A4801F0A3FC1C4B1B682F33B3
:102DA0001A78012A26D1A9887F230800984323D1C5
:102DB00007202B78490203400B43E978313089071B
:102DC0000B436978C90001400B43A9784A4092013E
:102DD00013431A000E490A409A420DD16262606A9A
:102DE0000840801A434258410A4B404218400A4B5F
:102DF000C01870BD0948FCE70948FAE7560800000A
:102E0000ABCD0D105708000058080000E0AD0208D7
:102E1000DBFEFFE0FDFF3DFF0300C2000200C20039
:102E20000100C20070B504000D00002803D1214943
:102E3000214801F055FC2B78032B03D91F491E486C
:102E400001F04EFC6B78032B03D91D491A4801F0A1
:102E500047FC1C4B1B682F331A78012A26D1A988FE
:102E60007F230800984323D107202B784902034091
:102E70000B43E978313089070B436978C900014079
:102E80000B43A9784A40920113431A000E490A40A5
:102E90009A420DD1626060680840801A43425841EE
:102EA0000A4B404218400A4BC01870BD0948FCE765
:102EB0000948FAE7A7080000ABCD0D10A8080000EC
:102EC000A9080000E0AD0208DBFEFFE0FDFF3DFFCA
:102ED0000300C2000200C2000100C20010B5041EBF
:102EE00003D10B490B4801F0FBFB0B4B1B682F3345
:102EF0001B78012B0AD18023626A1B06134363628D
:102F0000606A064BC00F0138184010BD0448FCE74A
:102F1000EB080000ABCD0D10E0AD02080300C200CD
:102F20000200C20010B5041E03D10B490B4801F08A
:102F3000D7FB0B4B1B682F331B78012B0AD1802347
:102F400062681B06134363606068064BC00F01385C
:102F5000184010BD0448FCE744090000ABCD0D103B
:102F6000E0AD02080300C2000200C20070B5040018
:102F70000D00002803D12149214801F0B1FB2B7835
:102F8000032B03D91F491E4801F0AAFB6B78032BC2
:102F900003D91D491A4801F0A3FB1C4B1B682F33B2
:102FA0001A78012A26D1A9887F230800984323D1C3
:102FB00007202B78490203400B43E9783130890719
:102FC0000B436978C90001400B43A9784A4092013C
:102FD00013431A000E490A409A420DD16262606A98
:102FE0000840801A434258410A4B404218400A4B5D
:102FF000C01870BD0948FCE70948FAE7A8090000B5
:10300000ABCD0D10A9090000AA090000E0AD02082F
:10301000DBFEFFE0FDFF3DFF0300C2000200C20037
:103020000100C20070B504000D00002803D1214941
:10303000214801F055FB2B78032B03D91F491E486B
:1030400001F04EFB6B78032B03D91D491A4801F0A0
:1030500047FB1C4B1B682F331A78012A26D1A988FD
:103060007F230800984323D107202B78490203408F
:103070000B43E978313089070B436978C900014077
:103080000B43A9784A40920113431A000E490A40A3
:103090009A420DD1626060680840801A43425841EC
:1030A0000A4B404218400A4BC01870BD0948FCE763
:1030B0000948FAE7F9090000ABCD0D10FA09000044
:1030C000FB090000E0AD0208DBFEFFE0FDFF3DFF75
:1030D0000300C2000200C2000100C200094B1B68CD
:1030E0002F331B78012B0AD18023426A1B0613431E
:1030F0004362406A044BC00F0138184070470348D0
:10310000FCE7C046E0AD02080300C2000200C200B6
:10311000094B1B682F331B78012B0AD1802342688F
:103120001B06134343604068044BC00F013818402E
:1031300070470348FCE7C046E0AD02080300C20048
:103140000200C200036810B5020080241B0500D4F1
:10315000403C82239B00D3580020DB05DB0DA342BB
:1031600003D090239B00D150013010BD0368802014
:103170001B0500D440387047F0B5050085B00C0041
:103180001600002800D177E1002900D174E10B7806
:10319000022B03D94821B94801F0A2FA637B023B14
:1031A000062B03D94921B54801F09AFAA37B002BDD
:1031B00006D0023B012B03D94A21B04801F090FA16
:1031C000A31CDB7F012B03D94B21AC4801F088FA0B
:1031D000230028331B78012B03D94C21A74801F089
:1031E0007FFA2378012B00D93AE108236268083A74
:1031F00093429B415B42002B03D04E219F4801F03C
:103200006FFAA368053B042B03D94F219B4801F0BB
:1032100067FA6369FF2B03D95021984801F060FADF
:10322000A369FF2B03D95121944801F059FAA37CDB
:10323000002B0CD02378002B05D1A368092B02D1D9
:10324000A37B002B03D053218C4801F049FA8C4B0F
:10325000626B1A4203D05521884801F041FA894B2C
:10326000E26B1A4203D05621844801F039FA2378E0
:10327000022B03D10022A37F934201D063685A1E20
:10328000237F0021581E834118040823A768BB42EE
:10329000494107331A4080239B0413430343C90267
:1032A0000B432B602800276BFFF760FF874203D397
:1032B0006B21724801F014FA2800A76BFFF756FF44
:1032C000874203D36C216D4801F00AFA2800676A2F
:1032D000FFF74CFF874203D36D21684801F000FAE5
:1032E000C022217892040B0613402B64607FE76AAA
:1032F000431E984183010093A37C07205A1E9341EB
:10330000227C9B020193531E9A411302627C02931A
:10331000531E9A415302F02203937B1E12031B0497
:103320001340627B013A02401343A27B2930120111
:1033300002401A43009B1A43019B1A43029B1A4303
:10334000039B1A43AA64207B431E9841E37B00023F
:10335000002B00D08DE002394B4259414B02A2684C
:10336000511E0F2211400143C020194380002950F3
:10337000FF21A36909041B040B406169C9B20B4317
:10338000C42189006B502B581A400332974201D355
:10339000102F03D98321394801F0A2F90021E37FDE
:1033A00022788B4203D0531E59424B411902072009
:1033B0003027637B013A013B0340A07B000138408A
:1033C00003430B436B64237B0F20591E8B4119026F
:1033D000A368013B03400B4351424A41120413438B
:1033E0008022FF219200AB50236B05320B40FF324D
:1033F000AB50631CDB7F5F1EBB415F06A31CDB7F02
:10340000013B584243411806230028331B78013BF7
:103410005A4253411A04636A0B403B43034313432C
:103420002B65A36B626B194081239B00E950164BFF
:1034300030001340154AAB50E36B154A1340154A50
:10344000AB5000239E4209D01800134A7360B3604A
:103450003360F36033623363F362726305B0F0BDCF
:103460000023A27F9A4200D1C5E663685A1E062354
:10347000BEE680239B0072E70848EFE702CE0D10FE
:1034800092F4FFFF8CF8FFFF6D0B0000C80F0000E7
:1034900073070000880F0000EFCDAB000160AA00A9
:1034A000036810B50400002B07D0012001F00EF9CD
:1034B0002368013B2360002B01D0002010BD014890
:1034C000FCE7C0460200B200030A08704B70030C10
:1034D000000E8B70C870704770B504000D00002896
:1034E00041D000293FD0002B3DD05A62F922032160
:1034F000D20083588B4383502B68DBB2012B03D956
:1035000057311A4801F0ECF8AB68DBB2032B03D952
:103510005B21164801F0E4F86B68072B03D95C21A6
:10352000124801F0DDF8EB68DBB2012B03D95D2115
:103530000E4801F0D5F8C022E021AB6892011B03D0
:1035400013406A68C90212040A4013430122296821
:1035500000200A4080211343EA68490412060A4009
:103560001343236070BD0248FCE7C0465DCE0D10DA
:103570000400B20010B50400012907D9A0210748B2
:1035800001F0AEF801232268134304E00029F9D1C9
:10359000012203689343236010BDC0465DCE0D1029
:1035A00070B54E1EF3B204001500012B07D9042993
:1035B00025D0082927D0E521154801F091F8032DE1
:1035C00003D9E621124801F08BF8072E14D83000F9
:1035D00004F046FA041312171212121B80231B0167
:1035E000E418002C08D0C0222D0492022368154054
:1035F000084A13401D43256070BD8823EFE7032A66
:10360000DFD89023EBE7032ADBD89823E7E7C0460F
:103610005DCE0D10FFFFFCFFF0B5160089B00593DD
:103620000EAB04CB01901B780291049310AB1D7874
:10363000331FDBB20392129CFA2B04D83E213B4885
:10364000FF3101F04DF8049B043BDBB2FA2B04D8A8
:103650009F213648490001F043F86B1E012B08D921
:10366000FB222B1F134204D040213048FF3101F0D0
:1036700037F8119B2D02DF07039B3604002B46D041
:10368000059B002B04D1A0212848490001F028F80F
:10369000049BFF2B04D142212448FF3101F020F884
:1036A000F0231B011D40636A0793C0239B021E4049
:1036B000029B2B4333433E0C00270024C0221F43B0
:1036C000019B20001F650727049B92021B041340E7
:1036D0001D43039B9C4202D2154B984201D109B075
:1036E000F0BD019B5B6C3B40032B0CD8059B039901
:1036F0001B5D01342B4332008C4200D20022134365
:10370000019AE4B2136507A8FFF7CAFEE1E7F023C8
:103710001B011D40636A3F0C0793C0239B021E40A0
:10372000029B2B4333433E00C7E7C0465DCE0D10DE
:103730000200B200F7B50193043BDBB205000F00B5
:103740001600099CFA2B04D8D5211648490000F030
:10375000C7FF002E21D007226B6C1340032B1ED80D
:103760008023C021721EDB0292B21A43019B8902A0
:103770001B040B4013432B65381E0DD0089B27609C
:10378000F922A660E36102230020A361D200A958B8
:10379000013B0B436660AB50FEBD0348FCE70348AA
:1037A000FAE7C0465DCE0D100400B2000100B20081
:1037B000F7B50193043BDBB205000F001600099C2E
:1037C000FA2B04D89C211648890000F089FF002EAE
:1037D00022D007226B6C1340032B1FD88023C021FB
:1037E000721E92031B03920B1A43019B89021B0456
:1037F0000B4013432B65381E0DD0089BE760F92260
:103800006661236204230020A361D200A958023B11
:103810000B432661AB50FEBD0248FCE70248FAE7C5
:103820005DCE0D100400B2000100B200F0B51F0023
:10383000043BDBB28FB006000D001400FA2B03D856
:103840005B495C4800F04CFF002C00D1ABE0072244
:10385000736C1340032B00D9A7E0631E9B039A0BE4
:1038600080231B031343C0223F04920217401F43CF
:103870003765281E0ED0149B00205B6A07950393C2
:10388000042309940C900A930A9B042B02D14A4BFF
:10389000984201D10FB0F0BD099B079C0093330003
:1038A000C43301931D680F231D40009B9D4200D926
:1038B0001D00002D17D1009B07940993002B0CD1FC
:1038C000F92202210320D200B3588B43B3500A904F
:1038D0000C9B002B01D00C9B9847009B03A80993DD
:1038E000FFF7DEFDD0E7082D0AD13700D83738685A
:1038F0002100FFF7E9FD3868211DFFF7E5FD05E030
:10390000012D09D13300D0331B682370009B64194B
:103910005B1B0093019BC5E7022D06D13300D43316
:103920001B6823701B0A6370F0E7032D0AD1330074
:10393000D4331B6823701B0A63703300D0331B68B9
:10394000A370E3E73700D83738682100042DD4D0BE
:10395000052D06D1FFF7B8FD3300D0331B68237166
:10396000D4E7062D08D1FFF7AFFD3300D4331B6831
:1039700023711B0A6371C9E7072D0CD1FFF7A4FD62
:103980003300D4331B6823711B0A63713300D033B7
:103990001B68A371BAE7FFF797FD3868211DFFF791
:1039A00093FD0825B2E7054874E7054872E7C0466D
:1039B000CD0200005DCE0D100200B2000400B20086
:1039C0000100B20000290CD00722436C1340032BE6
:1039D00009D8C023013989B21B03194301650020AE
:1039E00070470248FCE70248FAE7C0460400B2000C
:1039F0000100B20000230B604B608B600B61CB6059
:103A00004B618B61802302681B0613430360704780
:103A100030B58B6987B0DB680C001500002B0FD028
:103A200019681A79012303932378C9B20293FF23FB
:103A30000193002304950093FFF7EEFD07B030BD1E
:103A40000048FBE78000B20070B5160000220400B9
:103A5000080086B00A9D039204951900037800922D
:103A60000293FF23200001931300FFF7D5FD0028E8
:103A700006D103000095012231002000FFF7D6FE99
:103A800006B070BD30B50F24012385B08D696C443C
:103A90002370AB6A002B0BD01B680092DBB22200B4
:103AA000FFF7D2FF002803D12378AA6B13402370BD
:103AB0002078431E9841C0B205B030BDF0B587B044
:103AC00017000C9A05000C001E00FFF7A1FF00284C
:103AD00012D1A3690122DB6B022B00D013000392E9
:103AE00022780C99029200220491009301923B00EB
:103AF00031002800FFF790FD07B0F0BD0023F0B5BE
:103B00008F6989B00D00F96A07AC06000292238024
:103B100099425FD03A6B9A425CD0BB6A002B59D075
:103B20001B68096812680593029BC9B2039104924D
:103B3000009322000B002900FFF786FF00282FD1F9
:103B40006B46FF6B1B7C0493402F1ED0802F29D027
:103B5000022F41D16B46029A1B7D29000092300052
:103B60002200FFF771FF00281AD10D22029B04A941
:103B700000935218039B29003000FFF765FF0028CF
:103B80000ED163781F43677002E023781F432770CC
:103B90002200029B0093049B29003000FFF78EFF58
:103BA00009B0F0BD0D22029B04A900935218039B9B
:103BB00029003000FFF748FF0028F1D18023627808
:103BC0005B4213430D226370029B04A900935218B9
:103BD000049BE1E70148E3E70148E1E78000B20028
:103BE0000300B200F0B51F008B6989B01C6A0500A4
:103BF000002C47D0002A47D0586A0E9EB04243D3CB
:103C00004869C6B24869002800D10E782168207939
:103C1000C9B207911099029604910021039161792C
:103C200001911B6807990093130002002800FFF719
:103C3000F3FC002824D1A1684B1C12D12169002972
:103C400004D02800FFF7BEFE002819D1109A237D6A
:103C500001920F9A3900009228000E9AFFF76AFD30
:103C60000EE0109B227B0493FF23039001930090AE
:103C70000300C9B202962800FFF7CEFC0028DDD071
:103C800009B0F0BD0148FBE70148F9E78000B20048
:103C90000400B200F0B5CDB006000C1E06920893E9
:103CA00003D1C449C44800F01BFD00230BAF656B72
:103CB0003B80BB70089A06993000FFF771FC002D1D
:103CC00003D1BE4A10004DB0F0BD2B682A79D9B29D
:103CD000529B3000049300230393069B02936B795D
:103CE0000193032300933B00FFF796FC021EE9D1EA
:103CF00029693000FFF766FE021EE3D152992B7D41
:103D00000CAD01910090FF3229003000FFF750FD0B
:103D1000021ED7D1529B5E6AA94B5299886903282B
:103D200012D09A42CED0002E0CD00120013E00F0DD
:103D3000CDFC3200531E9A41A24B52421A40A04B76
:103D4000D218E9E73200E8E7002ABBD12B78532BE1
:103D5000B7D16B78462BB4D1AB78442BB1D1EB788B
:103D6000502BAED12B79052BABD96B79012BA8D178
:103D7000297BA3686D18AD7806956D080540012D67
:103D800000D8B1E0022D00D1ADE00F251F278E082D
:103D90000936B6004CA880190138FF380068BC46C7
:103DA000054001356D00079505093D40079F013528
:103DB0006F4309970327400A3840834D4000405B1A
:103DC000099D45430DA8256485596646280E304057
:103DD000079E013070436E0F37407C4E7F00BE5B04
:103DE00040277043606460462E0A06401038284021
:103DF000AD0400D4383F01304000013646437E43D5
:103E00000CA8A6640E1D87197D7807902802FD78FE
:103E10002D0605430798865D3543BE783604354345
:103E200064D40135ED080798656047183D002835D2
:103E30002E78012528003609B0403E7F6062B540EB
:103E40000698A5610CAD800655D502260898B043AA
:103E5000012850D0082084467F7A8C441F600027B8
:103E600060461F71079F5E713F5C7F095BD1033E17
:103E70009E6060461F262D5C35401D6102251D7524
:103E80000623E56804262B6000232B71256907981B
:103E90002E602B71E5695C362E602B714118487FCE
:103EA0006569022728602B716B710125266A012044
:103EB0006D42337137607371B560336133750526B8
:103EC000A063A06A3A310660266B037133710878EB
:103ED0004006400F052800D9F4E6E16A03F0C0FD72
:103EE00065787E847878042020604EE78026033D44
:103EF0003606354397E70698400618D502260898F7
:103F0000B043012813D00A2084466E18F67A8C44F8
:103F10001E60002660461E715E712F5C7F09B742ED
:103F200001D1013EA4E7FF271E739F60A1E7102780
:103F30000698074017D06E18F67B01201E600F0010
:103F4000002658711E710E37EE5D760907D1013ECD
:103F50009E60ED5D1F2635401D6101258FE7FF2620
:103F600018739E60F5E701260698304014D00C20A7
:103F700084468C4460466E18767B1F711E605F71AC
:103F80002E5C760904D1013E9E6060462D5CE1E71F
:103F9000FF261F739E60F8E703251D60043D18711E
:103FA00058719D60186118756AE7E56335600D60AA
:103FB00088E6C046F9030000C4CE0D100500B2002B
:103FC0000200B200FEFF4DFFB4CE0D10BCCE0D10AE
:103FD0000123E763336034330B6073E64023E3630C
:103FE0003F3B33600433F7E78023E363423B3360B6
:103FF0000133F1E7F0B589B002900792002800D1B3
:104000001EE1002900D11BE14B680593002B00D174
:1040100016E1002A00D113E10B680693002B00D1B2
:104020000EE10023C02603930493B602039B059A76
:104030009B00D458002C4DD023785A1E012A09D950
:104040000422043B9343DBB2002B03D06E217D4856
:1040500000F046FB237A032B03D96F21794800F047
:104060003FFBA369002B03D17021764800F038FB99
:10407000A3691B68013B032B03D97121714800F030
:104080002FFB2278501E072800D9D7E003F0E8FC68
:104090000432D635D6D6D6388021029B09015D1868
:1040A000237A2968684F18043040394001430420BE
:1040B00029606168014226D0079902980091A169A0
:1040C000FFF7E8FD00281ED00823039A9340049AC6
:1040D0001A430492039B01330393039A069B934272
:1040E000A4D10020049B002B02D0B220000418436E
:1040F00009B0F0BD029B8821D0E7029B9021CDE75B
:10410000029B9821CAE763689B07E3D52169E068B1
:1041100003F036FD002903D08C214A4800F0E0FA74
:1041200023694A4A934202D95A1E134203D08D2171
:10413000444800F0D5FAFF218C466746E168A06943
:10414000B9438268036AA96021694942B943E960B9
:1041500001680320013901406069471EB84100022F
:1041600001432962002A2DD010680021471C08D085
:104170006746074080201179000609043140074353
:1041800039432964517990680904314069640021F8
:10419000471C07D08027117BC0B209043F0631407D
:1041A000384301430020A9641169814205D01F30C2
:1041B00001390140802000060843E864127D1204A2
:1041C00032402A65002B2CD019680022481C07D0E9
:1041D00080201A79C9B212040006324001430A4312
:1041E0002A665A799968120432406A660022481C8D
:1041F00007D080201A7BC9B2120400063240014366
:104200000A430021AA661A698A4205D01F31013A81
:104210000A40802109061143E9661B7D1B043340D7
:104220002B6702216268FF3111408022237A120637
:104230001B0433400A4313432B604BE7044851E708
:10424000034855E7C4CE0D10FFFFFCFFFFFF000041
:104250000400B200104B1B683C331B78834219D911
:10426000042910D94B1EFF3B132B13D81F231940D1
:104270000A4B8000C018C02304229B00C150403369
:10428000C250002070470723D0301940034B8000F4
:10429000C150F6E70248F5E7E0AD0208000026400D
:1042A00001004A0010B50F4B04001B683C331B781B
:1042B000834204D8A3210C48490000F011FA0B4BAB
:1042C000A400E418D0239B00E058072318400428DA
:1042D00007D1C0239B00E0581F23034080204000EB
:1042E000184310BDE0AD020823CF0D10000026409A
:1042F000F7B5041E03D14649464800F0F1F9B02352
:10430000454DDB00EB58002B00DA7FE0434B226881
:104310009A4203D942493F4800F0E2F9E279236822
:10432000511E8A419B0312069B0B1343B022D200FD
:10433000AB50A3883B4FBB4204D994213548890038
:1043400000F0CEF92389384EB34203D937493148BA
:1043500000F0C6F92389A28835491B04D204D20C87
:104360000B401343334AAB50A37A01910F2B04D96E
:1043700096212848890000F0B3F9E37A0F2B03D97E
:104380002D49244800F0ACF9A389BB4203D92B493D
:10439000204800F0A5F9FF22E37A29491B011340C8
:1043A000A28912020A400F211343A27A0A40C021B7
:1043B0001343A27B890512070A401343B122D2009E
:1043C000AB50A379042B03D91E49124800F088F999
:1043D000238AB34204D999210E48890000F080F95C
:1043E000E020A379184AC0001B02A95803401748CF
:1043F00001400B43AB50238A01981B04A95803408A
:104400001348014000200B43AB50FEBD1148FCE7B0
:104410003F02000023CF0D1000002640FFFF0300E5
:1044200049020000FF1F0000FF01000051020000D0
:104430000000FF0184050000590200005A0200003C
:1044400000FF1F00630200008C050000FFF8FFFF63
:10445000FFFF00FE03004A00F7B58022B2260700E6
:104460000500324B324C1206E158F6000A43E25086
:1044700000930422A359134201D1002D35D1B1205C
:104480008023C00022582B499B050A401343235028
:104490000191002F01D0002D06D0B0228023D20040
:1044A000A1581B060B43A3500126B223DB00E3589F
:1044B000334224D1002D1DD1002F24D0B121C900B9
:1044C0006258019B1C481A4080239B051343B0226D
:1044D0006350D200A3585B005B08A350009B009A76
:1044E000E3585B005B08A350FEBD012000F0EEF82E
:1044F000013DBEE7300000F0E9F8013DD5E7002FAF
:1045000001D0002DDAD0B122C0230020D200A15862
:104510009B050B43A3508742E6D0681E8541684245
:10452000064D054B2840C018DEE7C0468C0500004C
:1045300000002640FFFFFFCF02004A00FEFFB5FF4C
:1045400070B51A4E050033680C001A002832127834
:10455000012A15D182080721100088430FD10320BA
:104560002840C00084401B68920020339B18220022
:10457000FF24844019684A4014404C401C6070BDC0
:104580005B8FDBB28B4203D17F21094800F0A8F892
:104590000720802205408020336892011B680006B6
:1045A000A4180543A400E550E9E7C046E0AD0208C1
:1045B0007CCF0D100A4B70B59B680A4E10300D0071
:1045C0008400B34209D1002904D1A0210648490042
:1045D00000F086F83059355170BD044B1859FBE78F
:1045E00000ED00E000A002087CCF0D1000000D10CF
:1045F000F8B506000D00002841D04368032B03D90D
:104600003B21204800F06CF80023F05E002828DBF6
:10461000B178FFF795FF0024FF220327944600237B
:10462000F05E716883B21F40FF006646BA408901A0
:104630003140D243B940002815DB134E83089B005C
:104640009B19C026B6009F593A40114399510F4B10
:104650009A680F4B9A4202D12900FFF7ABFF200066
:10466000F8BD0C4CD8E70F263340083B074E9B089B
:104670009B009B19DE6932401143D961E7E7054C85
:10468000EDE7C0467CCF0D1000E100E000ED00E05A
:1046900000A002080100560070B5802504002D021C
:1046A000AC4205D8064B18686043FDF751FB70BD5E
:1046B000044B1868FDF74CFB034BE418F0E7C046C9
:1046C00030A1020828A102080080FFFF10B5034BAB
:1046D0001B785843FDF73CFB10BDC04634A10208CF
:1046E00070B50D00044C01001822200004F0B0FB4E
:1046F000A56101BEFEE7C046B0A702088022054BB7
:1047000012069A64986C044BC043C0171840034BC0
:10471000C018704700002740FDFFB9FF03004600A6
:104720008022054B120198585B68DBB2002B02D047
:104730008023DB021843704700002640FEE700009C
:1047400002680A4B10B5DA6142681A6282685A62DE
:10475000C2689A620269DA6242691A6382695A63BC
:10476000C2699A63FFF7EAFF10BDC046B0A702080E
:10477000F0B51922002800D14B322A4B8A429241CF
:104780001B6852421C00A83424881D686719032541
:104790003E68AE4316433E601E68A4192768224E49
:1047A000374027601C00AA3424881E68A7193E6879
:1047B000AE4332433A601A681B4EA2181468264072
:1047C000166000280ED00020102904D9213088421C
:1047D0008041404201300F225B68196891430843D1
:1047E0001860F0BD1A00553212788A42F3D21A00CE
:1047F0005632127801208A42EDD21A0057321278CE
:1048000000188A42E7D21A005832127828008A42E9
:10481000E1D21A0059321078884280414042043077
:10482000D9E7C046E0AD0208FFFCFFFFB0235B05FF
:104830005A782120002A01D05878C0B27047B0239E
:104840005B059A89002A02D0988980B2704780203F
:104850004000FBE770B5FFF7F2FF8023184A5B00CA
:10486000984215D111680F240B0002229833186862
:104870000B6818180368A3431343036008009C30B7
:104880000B6801685B181968A1430A431A6070BD80
:104890001268B0201100C025983114680968094BCE
:1048A0004005C35861180C68AD002B4323430B60CF
:1048B00011009C3113680A689B18034A8258E5E787
:1048C000E0AD0208481800004418000070B5FFF77A
:1048D000B6FF8023184A5B00984215D111680F2457
:1048E0000B000322983318680B6818180368A34359
:1048F0001343036008009C300B6801685B1819685B
:10490000A1430A431A6070BD1268B0241100C1208F
:10491000C026983115680968640540012358691854
:104920000D68B60033432B430B6011009C311368B4
:104930000A689B182258E5E7E0AD020810B5FFF7BA
:104940007EFF8023114A5B0098420DD11368104905
:104950001A00983212681B689B181A681140C0220E
:10496000D2010A431A6010BDB0211268094B4905F3
:10497000CB581100C0209831096812688000521885
:10498000116803430B431360EDE7C046E0AD020836
:10499000FF8FFFFF1818000070B5FFF750FF80234E
:1049A000144A5B0098420DD1136813491A009832DB
:1049B00012681B689B181A6811408022D2010A43B2
:1049C0001A6070BD1268B0241100C02698311568B5
:1049D0000A4809686405235869180D68B60033430E
:1049E0002B430B6011009C3113680A689B182258F6
:1049F000E6E7C046E0AD0208FF8FFFFF4C1800005D
:104A000010B50020FDF782FF0400FFF70FFF012221
:104A10001300222801D8634263411340180010BDDF
:104A200010B5074C236831331B78002B04D1E621E5
:104A300004484900FFF754FE2368186A10BDC046B9
:104A4000E0AD0208ECCB0D1030B5040085B00D00D0
:104A5000042803D927492848FFF742FE6B1E012B83
:104A600007D9FB222B1F134203D024492248FFF70A
:104A700037FE234BA400E458042D01D0012D1AD198
:104A800000200FE0A3682B420BD1E36829001A68CD
:104A90005B6802920193039302A823689847194B1D
:104AA0001C606469002C04D0174B9842EAD1012D98
:104AB000E8D105B030BD022D06D1124B1B68181E7F
:104AC000F7D01C6903E01C006369002BFBD10020B8
:104AD000002CEED0A3682B4209D1E36829001A68A4
:104AE0005B6802920193039302A8236898472469A4
:104AF000EEE7C046E5090000D5CF0D10E60900003D
:104B000048A8020844A80208FF004200F8B50400C3
:104B1000012803D92A492B48FFF7E2FDFFF786FE5B
:104B200085B2FFF78CFE070000208026FDF7EEFE21
:104B30007600002811D1B74211D1222D0FD880253F
:104B4000214B6D041B6824065968204B2C40CA5821
:104B50001F4D2A401443CC50F8BDB74229D0FFF76F
:104B60005FFF0500B7420FD1621E9441802362426D
:104B70005B001A40174BD21801212800FDF700FCFA
:104B8000002808D01448E7E7621E944102236242DD
:104B90001A40124BEFE70C4B1B68B4331B68EB1841
:104BA0001A68002AFCDBEB6800201B0EA02BE9D161
:104BB000D2E7222DE6D9FFF733FF0500D4E7C04640
:104BC0007F0A0000D5CF0D10E0AD020818F00000FC
:104BD000FFFFFFFE01000030040042000100000C56
:104BE000F7B50700012803D929492A48FFF778FDBE
:104BF000FFF725FE80235B0098421CD0FDF7B1F83B
:104C0000B0230190244D254A5B05002F1AD024497A
:104C100003205958A950234A23499C5C1F226B58F2
:104C2000E4B293431A000B2313436B50FFF74EFD7E
:104C3000FFF7B2FE12E0FFF7E3FE0028DED11B4EC5
:104C40003000FEBDAF50E8220120D2009C5CFFF78F
:104C50005DFFE4B2061E0DD1FFF7FCFD1F21124AD5
:104C60000C40AB588B431C43AC50002F06D1FFF7D0
:104C700065FE3E000198FDF778F8E1E70720FFF7B1
:104C800025FDFFF723FE0020FFF740FF0600F1E7B8
:104C900053080000D5CF0D1000002640307F0000E3
:104CA00010180000410700001CFF00000300420034
:104CB00010B5041E03D111491148FFF711FDF2226E
:104CC000104BD2011B68DB689A582260F022D20197
:104CD0009A5862600C4A9A58A2600C4A9A58E2604C
:104CE0000B4A9A5822610B4A9A5862610A4A9A58AA
:104CF000A2610A4A9B58E36110BDC046D40A000075
:104D0000D5CF0D10E0AD020804780000087800004F
:104D10000C7800001078000014780000187800006B
:104D200010B5041E03D110491048FFF7D9FCF0223A
:104D30000F4B61681B68D201DB689950A1680D4A6E
:104D40009950E1680C4A995021690C4A995061695F
:104D50000B4A9950A1690B4A9950E1690A4A995046
:104D60002168E832995010BDFC0A0000D5CF0D1023
:104D7000E0AD020804780000087800000C7800001C
:104D8000107800001478000018780000F7B50700CC
:104D9000012803D940494148FFF7A2FC404D6B6808
:104DA000002B4AD1FCF7DDFF6B680190002B56D138
:104DB0003C4E33681A0043321278002A07D09B68B1
:104DC000E0331B68DB0602D53748FFF771FFFFF7BA
:104DD00036FD80235B00984246D1380007F034FC52
:104DE000002433681A0043321278002A17D00028B2
:104DF00015D09B68E0331B68DB0610D5FFF716FD66
:104E0000294B212808D032681300B03319880723B2
:104E10004B43126A9B18DB681800FFF781FF01986B
:104E2000FCF7A3FF002C0ED16B68002B03D00821E8
:104E30000120FFF709FE2000FEBD01210800FFF759
:104E400003FE041EAED06B68002B03D002210120AC
:104E5000FFF7FAFD154B9C42EDD0154CEBE7042112
:104E60000120FFF7F1FDA3E7FFF7DAFD3368B43364
:104E70001B68C0180368002B0BDB04230D4A116963
:104E80000B431361012F02D030BF0020A8E720BFE1
:104E9000FBE70020054CA4E7AE020000D5CF0D10C3
:104EA00048A80208E0AD020824A802080500420054
:104EB000FF00420000ED00E0C022802006495200C1
:104EC0008B58C0059B009B0803438B508023885858
:104ED0001B0603438B507047000026407047FFF7C6
:104EE000FDFF72B6124C134DAC4209DA21686268BC
:104EF000A368043B02DBC858D050FAE70C34F3E750
:104F00000D4B0E4CA34208DA19685A680020043A87
:104F100001DB8850FBE70833F4E7094809490860DA
:104F2000BFF34F8F00F0E4F800F0F8FAFEE700005E
:104F3000C0E10D10D8E10D10D8E10D10E8E10D1021
:104F400000A0020808ED00E0FEE7FEE700B504203F
:104F50007146084202D0EFF3098001E0EFF30880C8
:104F60000430FFF7EDFBFEE770470000E02370B56B
:104F7000504C9B00E2580F23D021072013409A0089
:104F8000121989005158014066D0042958D04A4866
:104F9000002B66D1B223B1220321DB00D200E558F9
:104FA000A358A6581B0F360F0B400E4204D0A25830
:104FB000120F0A40012A01D1EA0701D4032B11D1B3
:104FC000B0233E4ADB00E558A158E658C904C90C95
:104FD00002F050FDAD03AD0B6843F101C90F013183
:104FE00002F048FDE0239B00E3589B069B0FD8404E
:104FF000334B1860334B1C691969240A090E0131BF
:1050000002F038FD304BE1B21860013102F032FDA0
:105010002E4B040018602E4B2E4918602E4BC018E2
:1050200002F028FDFA212D4B890018702C4BE01856
:1050300002F020FD2B4B18602B4BC003186070BD95
:10504000C021890052581F210A40112A01D0132A79
:1050500004D1802000029BE7244899E7FA20C00190
:1050600096E7012BBED1C823C0220321DB00D2006A
:10507000E558A358A6581B0F360F0B400E4204D01C
:10508000A258120F0A40012A01D1EA0701D4032BCA
:10509000A8D1C022D200A358A158A5587F221F260C
:1050A0001340090A3140584302F0E4FC290C314016
:1050B00096E7C0460000264000366E0184050000D9
:1050C00020A102080000214024A102081CA102081E
:1050D0002CA1020840420F003F420F0034A10208F9
:1050E000E703000030A1020828A1020800127A009C
:1050F00010B51B48FCF73CFEB022E0213020194CD3
:10510000D200A35889005B005B08A3506358834317
:10511000635080235B04A350134B144AE250A02237
:1051200004339201E250FF22114BE250FFF7C4FE1C
:10513000C02201215200A3588B43A350FFF714FF54
:10514000FFF714FFB0235B055A78002A02D05B7882
:10515000212B03D10022074BDA605A6010BDC046F4
:1051600034CB0D1000002640840500000100020031
:105170008C050000E0002340024BD86F0323184049
:105180007047C0460400214010B5FCF7EAFD07490E
:10519000074ACB6F1A40074B1343CB6710230649CE
:1051A0000A681A42FCD0FCF7E0FD10BD0400214063
:1051B000FCFF00000100FA058800214070B583055E
:1051C0000600002B04D0E8211048FF31FFF788FAD1
:1051D0000F4CFCF7C6FDE36F0500DB439B0701D1D5
:1051E000FFF7D2FFB0230B4A9B00D650E36F0A4A69
:1051F0000A491A400A4B1343E36710230A681A420C
:10520000FCD02800FCF7B1FD70BDC0462DD00D10BC
:105210000400214000002140FCFF000088002140E4
:105220000300FA0510B562B600F0B6FAFFF744FEC7
:10523000C02201210A48520083580A4C8B438350F4
:10524000094A0A48FCF71EFF094A0A492000FDF7EF
:1052500093FF802322681B061343236010BDC046C2
:10526000000026400000664098D00D1080023240B9
:10527000E4AD02084CD40D1010B50020FDF756FA2D
:1052800010BD0000802310B50C4C032023602300C8
:10529000210008336360FDF779FA0948FDF7A4F8A7
:1052A000084B1B6851331B78002B02D00648FDF7D2
:1052B00013F920001830FCF70BFE10BD00C00208E7
:1052C0003CC00208E0AD020858D10D1010B50448EA
:1052D000044A0021121A02F025FFFBF705F910BD60
:1052E0000000020800A002080022E82313B5019282
:1052F000019C9B0523430193019B090419430191E0
:10530000019B000218430123019001990B43019373
:105310000199124BD96012491868002806DB8A42AD
:1053200002D10120404216BD0132F5E78A42F8D091
:1053300001229A6000221869002803DA8A42F0D01C
:105340000132F8E78A42ECD0DB6800200193A02309
:10535000019A1B069A42E6D00198E4E70000234038
:10536000983A000010B5084B0024DB78013B012B74
:1053700007D801210800FFF7B7FF04006420FFF7FA
:105380008BF9200010BDC04674AF0208A02270B592
:10539000154DD200AA580400032A09D0FFF7E2FFF6
:1053A000021E05D0114B12491B68D86802F014FE8A
:1053B000104B1B68002B0CDA0F4A104B1048DA64B4
:1053C0000A4B1B68D96802F061FE72B607F044F917
:1053D00062B6AC239B00EC500A4B9C60236883F3BD
:1053E000088863689847FEE70000214084A102080E
:1053F00014D10D1000012640214334120000234037
:1054000044D10D1000ED00E070B50400FFF7AAFFD5
:10541000021E05D01A4B1B491B68D86802F0DCFD40
:10542000194B1B68002B23DA184A194B1948DA6408
:10543000134B1B68D96802F029FE72B6B023164AD6
:10544000164D9B001648EA50C36F164A16491A407B
:10545000164B1343C36710230A681A42FCD001207D
:10546000FFF71AF9B0239B00EC5007F0F5F862B68D
:105470002000FFF7A3FE0020FFF788FCFBE7C046F3
:1054800084A1020814D10D100001264021433412DA
:105490000000234044D10D100040001600002140C0
:1054A00004002140FCFF0000880021400300FA05B1
:1054B00010B5002820D1114C11482368D96802F09A
:1054C000E5FDFFF74FFF021E04D023680D49D868A1
:1054D00002F082FD0C4B1B68002B08DA0B4A0C4BC8
:1054E0000C48DA642368D96802F0D0FD72B60A4825
:1054F000FFF764FE07F0A0F810BDC04684A10208C3
:10550000CCD00D1014D10D100001264021433412CF
:105510000000234044D10D1000400016F0B589B0C2
:10552000FFF7B0FEFFF77EFE754C764A764B774D5F
:105530001A6023682800D96802F0A8FD2368744E19
:10554000D968300002F0A2FD7D232068019300237A
:10555000009301226F49C06802F03EFD23683000CD
:10556000D96802F093FD23682800D96802F08EFD07
:1055700023686948D96802F089FD802002AA03A93E
:105580004000FCF7EBFA051E00D0B4E0634E0300C8
:10559000634A31000398FBF765F9051E00D0AAE0C5
:1055A000B278022A05D923685E49D86802F014FD52
:1055B000B570F022F3685C4F12069B18BB6033692C
:1055C000FB6073699B18FB61B3693B62FAF758FF94
:1055D000051E38D1B378002B3CD0544A013B9B00C8
:1055E000534E9B58336000F043FC071E06D02368DF
:1055F000050002004F49D86802F0EEFC4E4A3168BF
:105600004E4800F0A7FC002F08D123684C48D96809
:1056100002F03CFD01214948FDF7ACFF68426841BA
:10562000FFF746FF23684748D96805AD02F02EFD15
:10563000280001F07FFD2368D968002813D0424874
:1056400002F024FDFEE72A0023684049D86802F0F2
:10565000C3FCE3E73E4BFA699A42DFD975702368D1
:1056600072693C49F2E73C4802F010FD04A9287930
:1056700000F010FD43425841FFF71AFF822201203B
:10568000364992008E588B58F605DB0B0340F60D19
:105690009B19002BF6D1049BAD68ED18059B1B8967
:1056A000ED18FFF713FE43425841FFF701FF1B4B74
:1056B0001878042819D802F0D3F90707030310005B
:1056C00002210020FDF7F0F82800FFF75FFE2368B5
:1056D0002348D96802F0DAFCFEE706210E20FDF728
:1056E000E3F82800FFF790FEF1E723681648D96831
:1056F00002F0CCFCFEE723682A001A49A6E7C04660
:1057000084A1020830D40D101CAE020898D10D10EF
:10571000A2D10D10E3D10D1018D20D1020AE020849
:1057200074AF020834D20D1040A1020838A102085B
:105730005CA80208A8D20D1004B002080000424084
:10574000DED20D1068D30D108CD30D106FD20D105A
:10575000FFFFFF07FBD20D10B2D30D100000664013
:10576000D9D30D10F7D30D1010B504002100034854
:10577000FDF7E8FC0028F9D010BDC04600006640E7
:10578000C221044A89005358DB05FCD0D0239B007A
:10579000D05870470000664010B500F009F800F0DE
:1057A00035F800F043F800F005F900F02DF810BDD1
:1057B00080218022124BC9001B68D205986810B561
:1057C00042501A00743212880E4C121810680440AD
:1057D000D4208001204310601C001A007234703203
:1057E0002478127898687333A2401C780323A3406E
:1057F00013438022120613434350435810BDC04642
:10580000E0AD0208FF00FFFF70470000054B1B687A
:105810001A003F321278052A03D900219A68024BF8
:10582000D1507047E0AD0208140C000010B51D4CBB
:105830001D4A00212000FCF725FC20001B4C1C4ABF
:105840000121FCF71FFC1B4A02212000FCF71AFC77
:10585000194A03212000FCF715FC184A04212000F6
:10586000FCF710FC164A05212000FCF70BFC154A3A
:1058700006212000FCF706FC2000134C134A0721E8
:10588000FCF700FC124A04212000FCF7FBFB114A44
:1058900006212000FCF7F6FB0F4A07212000FCF749
:1058A000F1FB10BD00003240C4D50D108005324020
:1058B000F8D50D1090D50D1028D50D10F4D40D107D
:1058C000C0D40D108CD40D10000332405CD50D10E7
:1058D0002CD60D1060D60D1094D60D1010B50A4BB5
:1058E0001B683E331B7883420BD9E0220F24074B01
:1058F0008000C01892008358A343194381500020B0
:1059000010BD0348FCE7C046E0AD02080000264099
:1059100001004A0010B50A4B1B683E331B788342D6
:105920000CD9E0223024074B8000C0189200835825
:105930000901A34319438150002010BD0248FCE730
:10594000E0AD02080000264001004A00054B064970
:105950001B681A000832D26F1B689B181A680A402D
:105960001A607047E0AD0208FF00FFFF074B1B689D
:10597000190008311A68CB6F8021D21813684904C6
:105980001B021B0A0B4313607047C046E0AD0208C0
:10599000054B06491B681A00883212681B689B1861
:1059A0001A680A401A607047E0AD0208FF00FFFF66
:1059B000FEE70000F8B596210020FEF7D9FEFEF7BD
:1059C000AFFE002801D1FEF799FE0120FFF708F98C
:1059D000644B65495A6C0A40E82189010A435A64BC
:1059E0005A6C120AD2B23A2A04D15A6C5F48024069
:1059F0001143596400210800FFF78CFFFFF7C8FF2F
:105A0000FFF7B4FFFFF7A2FF594D5A4C2B685A4FCE
:105A10003D331B78002B0ED0C0268023F600A25900
:105A20009B053A401343A3510120FEF74FFEA359B3
:105A30005B005B08A35100210120FEF70BFC2B68E3
:105A40003E331B78002B03D14C494D48FEF748FEEE
:105A5000E0239B00E6580F231E400AD13000FEF7DA
:105A600021FC1223FF33984203D101213000FFF7BC
:105A700035FFB122D200A35800213B408027BF054B
:105A80001F43A750083AA35808005B005B08A350C7
:105A90003C4AA3585B005B08A350FEF7DBFB0021E8
:105AA0000800FFF71BFFFFF773FFFFF75FFFFFF72C
:105AB0004DFF00210120FEF7CDFB01210020FFF763
:105AC0000DFF00210800FEF7C5FB00210220FEF7B4
:105AD000C1FB00210320FEF7BDFB00210420FEF7DF
:105AE000B9FB2948FEF704FC002802D00420FFF788
:105AF0005FFF2648FEF7B0FC002802D00420FFF725
:105B000057FF00210800FFF7E9FE00210800FFF71A
:105B100001FF00210120FEF79DFB00210220FFF77D
:105B2000DDFE01210220FFF7F5FE2B683E331B78D6
:105B3000022B06D9E22280239200A1581B060B43B8
:105B4000A3508022124B1206E15800200A43012183
:105B5000E250E2580A43E2506331FEF709FEFFF7D4
:105B600005FAF8BD00002740FF00FFFFFFC5FFDF7B
:105B7000E0AD020800002640FFFFFFCF6E060000E8
:105B8000C8D60D108C05000024D70D10400D030061
:105B90000C050000437802781B021A438378C07812
:105BA0001B0413430006184370470000F7B5A54BCC
:105BB000A54A9A58D10700D47BE00F22A34FBB68B7
:105BC0003D680093A24BDC6F0193009B1440073AA1
:105BD000141B9C4200D91C009E4E002C18D1009B27
:105BE0003D60BB60002B0CD1F92201209549D20009
:105BF0008B5883438B50B861FB69002B01D0FB6944
:105C00009847F8230122DB008E49CA50CB58F7BDD4
:105C1000082C16D12800FFF7BDFF3060281DFFF7C4
:105C2000B9FF3060009B2D191B1B0093019BDC6F9B
:105C30000F231C40073B1C1B009B9C42CDD91C0022
:105C4000CBE7012C03D12A78834B1A60EAE7022CB8
:105C500006D12A786B781B021343804A1360E1E770
:105C6000032C07D16B782A781B0213437B4A1360FD
:105C7000AA78E9E72800FFF78DFF042CD1D0306027
:105C8000052C01D12A79DFE7062C02D12A796B791C
:105C9000E1E7072C07D16B792A791B0213436F4A7E
:105CA0001360AA79D0E7281DFFF774FF082430603D
:105CB000B8E7910700D4A4E00F22644D68496C69ED
:105CC000EB6808688C460240A24200D92200654970
:105CD000654E002A16D1EB606C61002C0DD1F922C3
:105CE00002215848D20083588B4383500320A86177
:105CF0002B6A002B01D02B6A9847F8236C61DB00DC
:105D0000022281E7082A19D10868070A18705F7013
:105D1000070C000E9F70D8700868070A18715F7131
:105D2000070C000E9F71D8719B18A41A62460F20B1
:105D300012680240A242CCD92200CAE7012A03D14C
:105D40004A4800681870EFE7022A04D130681870DA
:105D5000000A5870E8E7032A07D130681870000A73
:105D60005870424800689870DEE7042A08D1086835
:105D7000070A18705F70070C000E9F70D870D3E789
:105D8000052A0BD10868070A18705F70070C000E0F
:105D9000D87036489F7000681871C5E7062A0CD184
:105DA0000868070A18705F70070C000E9F70D870A3
:105DB00030681871000A5871B6E7072A0FD10868D1
:105DC000070A18705F70070C000E9F70D87030685B
:105DD0001871000A5871254800689871A4E70A688C
:105DE000100A1A705870100C120E9870DA700A6847
:105DF000100A1A715871100C120EDA71987108227B
:105E000092E704210A4207D00520104A9061F82247
:105E1000D20099509B58FAE608210A4202D00B4A58
:105E20000620F3E71020024206D00721074A9161BD
:105E3000F822D2009850EDE72020024200D1E6E699
:105E4000024AF4E700004240CC07000004B0020818
:105E50000800424098004240900042409400424076
:105E6000C4004240D8004240D4004240D0004240EA
:105E700073B5684602001E4B12CB12C262B61D49B2
:105E8000FEF7B6FB021E05D01B4B1C491B68D868E9
:105E900002F0A2F8FA221A4D92002B0019491A4872
:105EA000FDF71AFB041E1ED1020001211648FDF762
:105EB00077FB29001448FDF79DFD0F4E134833680A
:105EC000D96802F0E3F82A0011490F48FEF792F86A
:105ED000041E08D133680F48D96802F0D7F82100B2
:105EE0000948FDF747FB80220B4B20001A6076BD66
:105EF000C8D90D10AD5B0D1084A1020847DA0D1052
:105F000004B002083CD40D100000424087DA0D10A6
:105F1000B8D90D10A4DA0D1000E100E00C4B1B689D
:105F20009B691B68032B08D10023CB7083B21B0A2B
:105F300088704B70000C08707047042BFCD183B242
:105F4000C8701B0A000C48708B70000AF3E7C0464B
:105F50005CA80208F0B50F2787B002ABFF1800233A
:105F600016003B708B690500DA6BDB6A03921B68D5
:105F70003A00DBB200960C00FDF766FD021E06D06B
:105F8000104B11491B68D86802F026F813E06B46E5
:105F90003A781B7B1A409A420DD03200210028002B
:105FA000FDF7ACFD021E08D1320021002800FDF7EC
:105FB00069FD0028F8D107B0F0BD024B03491B680A
:105FC000E1E7C04684A10208D0D90D100CDA0D100B
:105FD000F0B589B004000E00049217221A4D059303
:105FE000296802A88B6912189F6ADB6A20001B6867
:105FF0000096DBB2FDF728FD002823D13200296886
:106000002000FDF705FD00281CD1059B01900093A1
:106010000296049B0E9A29682000FDF7E3FD0028F4
:1060200010D1320029682000FDF72CFD0028F8D19E
:1060300017223B6802A900965218DBB2296820009B
:10604000FDF702FD09B0F0BD5CA8020870B54B6811
:10605000056801229D4216D38A689B1800229D4242
:1060600011D20C694B699C420FD20C236343CE685A
:106070000134F3180E685A701E705A8042685D60D1
:106080009A6001220C61100070BD0C235B428B6191
:10609000F9E7000010B502006F2809D0074B084946
:1060A00018686F23C06801F097FF1620404210BDAA
:1060B00080235B050B600020F9E7C04684A102083D
:1060C000A5DB0D1010B50F4B02001879904215D0CA
:1060D000187E904214D018002C30047801204042E1
:1060E00094420AD1033014224243101D181808604C
:1060F00000209B181A6901321A6110BD0020F2E7D6
:106100000120F0E740A1020810B5021E0BD0011FCC
:106110000C4B0868984207D00B49137808680B4964
:10612000C06801F059FF10BD0B69002B07D1064B69
:1061300012781B680649D86801F04EFFF3E7013B6F
:106140000B61F0E7EFBE0DD084A10208BDDA0D109F
:10615000DDDA0D1070B544680F480C1901211500E7
:106160001E00FDF707FA80235B05E2180B4B9A42ED
:1061700003D90B4B9B78002B05D03200290020005F
:1061800000F04EF970BD074B07491B68D86801F055
:1061900023FF01204042F5E700004240FFFFFF17C8
:1061A00020AE020884A1020838DB0D10F0B51500FE
:1061B000F0221D4F87B003933B684468DB681206EA
:1061C0000C199B18A34216D800211848FDF7D2F9E4
:1061D0003B6805AED8688023201A5B05C0183100E3
:1061E000FFF79CFE0096039B2A0011490F48FFF71A
:1061F000EFFE07B0F0BD80235B05E2180D4B9A421D
:1062000003D90D4B9B78002B05D0039A2900200061
:1062100000F09CF9EDE7094B09491B68D86801F0CB
:10622000DBFE01204042E4E75CA802080000424097
:1062300004B00208FFFFFF1720AE020884A1020885
:106240006EDB0D10F0B51500F0222E4F44683B6850
:106250001206DB680C199B18C5B0A3423AD800217E
:106260002948FDF787F980220021520004A801F097
:1062700059FF3B680020D9688023641A5B052E0A09
:10628000E418002E14D0002801D045B0F0BD03AFB3
:1062900020003900FFF742FE802300975B0004AA2C
:1062A0001A4919480134FFF793FEFF34013EE8E72D
:1062B000EDB2002DE9D00028E7D103AE3100200077
:1062C000FFF72CFE00962B0004AA10490E48FFF79A
:1062D0007FFEDAE780235B05E2180D4B9A4203D973
:1062E0000C4B9B78002B04D02900200000F038F9DB
:1062F000CBE7094B09491B68D86801F06DFE012006
:106300004042C2E75CA802080000424004B0020814
:10631000FFFFFF1720AE020884A1020801DB0D1069
:1063200010B5007800F08CF910BD01307047000006
:10633000431E022B15D8022808D003280BD00A4B85
:1063400098680860DB68002013607047064BD869C6
:1063500008601B6AF7E7F0231B030B6080235B01D7
:10636000F1E701204042F0E740A1020830B589B0D2
:106370000C00150002A903AA0190FFF7D9FF00281D
:1063800011D1236805900693084B079001AA18685D
:106390000749049500F00EF80798002801D1059BE5
:1063A000236009B030BD01204042FAE71CAE02086C
:1063B0004D600D10F0B50024260043688BB00291AB
:1063C0001B6906A905A8039298470194069BB3424E
:1063D00001D80BB0F0BD059BF700DF197B68019D6C
:1063E0000893019B3A68EB1A9A4202D8013601954C
:1063F000ECE707940995039907A8029B98470028A2
:10640000E7D0089B0135E418EBE70000024B03607E
:1064100001230B607047C046D0DB0D100020704791
:106420000B00802110B549054118180001F071FEDC
:10643000002010BDF0B5264CF023A54400240390A5
:1064400020001B06CB1801935B0A5B0204AF02928B
:10645000FD1A029AA24201D900280CD01D4B984285
:1064600034D01D4B984231D0431E984140008523C3
:106470009B009D44F0BD8022010092009E18019A6D
:106480009A421DD8029AA2421AD9039A125DEA547E
:10649000002906D18021490559180978511A4A1E48
:1064A000914101340133B342E9D1002904D00B4BAF
:1064B0003900F018FBF76CFD094BED183300C8E705
:1064C000802252059A181278EA54EBE70120CEE7B1
:1064D000ECFDFFFF020052000600520000FEFF0F1D
:1064E00000FEFFFF00207047F8B5124C0023A142C8
:1064F0001CD91E00104C8D18AC425E410F4CA142BD
:1065000015D91F000E4CAC425F413C000D4FB94203
:1065100002D90D4FAF425B41344323430124002B8A
:1065200002D0FFF787FF04002000F8BD1E00002402
:106530002300F1E7FFFFFF0F00001010FFFFFF1324
:1065400000800014FF070016000A00160B008021CF
:1065500010B5490541181800FFF7C6FF10BD00002F
:106560008023F0B55B05C0184518334CEB05A544F6
:10657000C605DB0DF60D01936B0A039333005A1E1B
:106580009341400AC0186B0A1B1A009343021F0074
:1065900000240293009B002B3ED1002E1AD0274AE4
:1065A000029B944663441C001900320004A801F0C9
:1065B000B0FD2000FBF7AEFC43425841FEF778FFE8
:1065C0002100320004A8FFF78FFF04006042604101
:1065D000FEF76EFF019B002B19D08024A400E41A63
:1065E0002200290004A801F094FD039B5802FBF748
:1065F00091FC43425841FEF75BFF2200290004A8AA
:10660000FFF772FF040060426041FEF751FF200077
:1066100085239B009D44F0BD3800FBF77BFC040004
:1066200060426041FEF744FF80239B00FF18009BFF
:10663000013B0093AEE7C046ECFDFFFF00FEFFFF0D
:106640000420704710B510220949040001F052FDE2
:106650000123002808D0230010332268013205D11D
:1066600004349C42F9D10323180010BD0223FBE738
:10667000F0DB0D1030B5040091B001200D00FEF7E5
:1066800017FFA168102310396A462000FFF762FD4A
:10669000002802D0012011B030BD6846FFF7D2FFBC
:1066A00028702378032B0CD10120FEF701FFA1688D
:1066B0000123AA1C18392000FFF74CFD431E984106
:1066C000E9E70120FEF7F4FE0120FEF7F1FEA168E4
:1066D0006A1C203901232000FFF73CFD0028E3D08D
:1066E000D8E737B50D00C0B201A9FFF7EBFC0124D4
:1066F000002807D129000198FFF7BCFF040001988A
:10670000FFF702FD20003EBDF7B501206946FFF707
:10671000E8FF002801D0FF20FEBD01AC21000220CF
:10672000FFF7DFFF0028F6D12078A678234C6B46D0
:10673000220019789D785F7812322378002B01D0DF
:106740008B422FD16378002B01D083422AD1A378CA
:10675000002B01D0AB4225D1E378002B01D0B3420E
:1067600020D12379002B1BD1154B164A1B68D86802
:106770006379022B06D0144A032B03D0134A042B4F
:1067800000D0134A134901F027FC0222002063794C
:10679000023BDBB29A424041FEF78AFE6079BBE7DA
:1067A000BB42E1D006349442C7D1054B0A481B686E
:1067B000D96801F06BFC0120AEE7C04600DC0D108B
:1067C00084A1020817DC0D1012DC0D102EDC0D1058
:1067D0001CDC0D1035DC0D104BDC0D10F0B597B046
:1067E0001CAB1B780390049313781400302B16D144
:1067F0009378022B13D106AD40220021280001F02E
:1068000091FCE278A1184B79901D0979C01802908B
:10681000022904D1D1186078043188422AD010208E
:1068200017B0F0BD059A0F1A5618B446A444664630
:1068300036790822B44604AEB61862462037F255BF
:1068400001318842EED100220299C91A64189A4295
:106850000AD16B46188A402300950193039A203B86
:106860000A49F9F775FEDBE7D11AA05C403168549C
:106870000132ECE7202B00DD20231000202A00DD70
:106880002020121A00210592DBE7C04609000610FD
:10689000002803D1044B1B7F1800704700230128F8
:1068A000FAD1014BDB7FF7E720AE0208F0B5F7B075
:1068B0000500029111A8594917000493F9F7D0FE79
:1068C00000284CD17C9B002B3FD100242B89EA6807
:1068D0009B180393039BA34214D9039B049E1B1B89
:1068E0009E4200D91E0033003A0021000298FFF7B3
:1068F00031FC002833D13200390011A8F9F7BEFE6F
:1069000000282ED008AB202209A911A8F9F7C6FE4D
:10691000002824D17E9B002B04D0202209A9180036
:1069200001F0F7FBEB682C8907ADE4182A0004237B
:1069300021000298FFF70EFC002810D1384B2A885E
:106940009A4210D00120404209E07D9B002BBCDD23
:106950001A007C9911A8F9F791FE0028B5D077B0FC
:10696000F0BDA419B6E76B8801251B190593043403
:10697000039004906D42059B9C4205D3049B002B21
:10698000E0D003980138EAE708AF04233A00210079
:106990000298FFF7DFFB0028E1D13B787E88102BBF
:1069A00017D1202ECED1211D330011AA0298FFF756
:1069B000D1FB0028D3D1320011A909A801F09AFB1C
:1069C0000028BFD10123049308AB5B880433E4188B
:1069D000D1E7012B04D17F98FFF75AFF0500F3E7B9
:1069E000222BF1D13300483BB82BABD8211D33000B
:1069F00011AA0298FFF7AEFB0028A3D1EDB27B8865
:106A000011AA0095202109A80125FFF7E7FE6D4294
:106A10000028D9D101230393D6E7C046090000011D
:106A200007690000F7B50700002401262000FFF7E2
:106A30007CFC01A9C0B2FFF745FB3500011E0AD15D
:106A40002C2363430B4A0198D2182023FFF782FBC3
:106A50000500681E85410198FFF756FB002D04D004
:106A6000012C00D13D002800FEBD012CFBD03400DC
:106A7000DCE7C04660A8020873B50C00C0B201A9EB
:106A80001500FFF71FFB0126002807D12A0021006F
:106A90000198FFF7D7FB0600701E86410198FFF7AB
:106AA00033FB300076BD0000F0B52C244443344B5A
:106AB00087B01C19236805001A00324B9A4201D096
:106AC00001204AE02369DB06FAD4FFF72EFC04A973
:106AD000C0B2FFF7F7FA03000120002B3ED1E368B4
:106AE000268905AFF6183A00042331000498FFF711
:106AF00031FB0028E4D1244B3A889A4201D17888AE
:106B000080192C236B431E4AD3181B6A9B6883424F
:106B1000D6D31E4BA27A1B789A42D1D12000F9F726
:106B200031FB0028CCD123681A00164B9A4217D1AA
:106B3000802302900190009003955B00144A049911
:106B40002000FFF7B3FE00280AD10498FFF7DCFA13
:106B50002000F9F73BFB431E9841404207B0F0BDCF
:106B6000002D04D0049800218268FFF76BFB094BCD
:106B70002A001B680849D86801F02EFAA0E7C04631
:106B800060A802083DB8F3960769000020AE02082D
:106B9000D0AC020884A10208F2DD0D100023F0B58C
:106BA000B04CB14AB14DA544012013602B60FFF7F2
:106BB0007BFFAF4B040001201F79FFF769FE002C1B
:106BC00047D1AC4BC2B2DB6C39005E6880235B05F9
:106BD000F3180293A84BF618300013ABFAF7F6FF40
:106BE000041E36D105A8F9F77DFD8021A34A89004E
:106BF00005A8F9F785FD05A90B20F9F791FD041EFD
:106C000027D1102313AA9E490B20F9F759FD012320
:106C1000041E2B601DD1994A0B211BA8F9F7ACFC6F
:106C2000041E16D1102217A91BA8F9F7C7FC041ED1
:106C30000FD1202204AB2DAD019300922B00310027
:106C40001BA8F9F7CBFC049B0400202B10D00124D7
:106C50006442864B1B68002B05D00B20F9F7D4FC4F
:106C6000002800D004002000D3239B009D44F0BDE9
:106C70000028EED1020004AB29001BA8F9F78CFC18
:106C8000041EE6D107AE33002A0013CA13C37D4F9A
:106C9000126831A91A603800102201F03AFA05A9E9
:106CA0000C20F9F73DFD041ED3D1102332007449A6
:106CB0000C20F9F705FD01226B4B041E1A60C8D1A8
:106CC00071496DA8F9F7CCFC041EC2D1029B029A4F
:106CD0001B890C21D3181BA8684A0393F9F74CFCB5
:106CE000041EB6D1102239001BA8F9F767FC041E58
:106CF000AFD1802604AB7600019300962B003200C2
:106D000003991BA8F9F76AFC049B0400B3429ED1C7
:106D100000289ED12D9B2E89AA7A309F3199581C2C
:106D200000D194E7C90600D591E75249C96C89683A
:106D3000B94200D28BE755498B4200D087E74C4BD4
:106D40001B78934200D082E78022290052006DA870
:106D5000F9F794FC041E00D07BE7F619330AF6B26B
:106D6000771EBE4101279B190293039B3E029E1989
:106D7000029BBB4222D9002C00D06AE704AB0193EE
:106D800080232DAA5B000093130080223100520063
:106D90001BA8F9F723FC8023049A04005B009A42A5
:106DA00009D1002805D11A002DA96DA8F9F766FCB4
:106DB00004000137D9E701246442FAE7002C00D02F
:106DC00047E704AF3B0020220BA96DA8F9F766FC4A
:106DD000041E00D03DE780225200019700922B0054
:106DE00031001BA8F9F7FAFB041E00D031E70200BE
:106DF0003B0029001BA8F9F7CFFB2D9B244A9BB22F
:106E00000400934200D022E7002800D021E72E9A08
:106E1000D3B2102B00D01AE7120C202A00D016E7AC
:106E20002FA90BA801F066F9041E00D011E7379BCB
:106E3000DBB2012B00D00AE70120FFF729FD409BC0
:106E4000DAB2222A00D002E71B0C482B00D0FEE663
:106E5000C0B2009041AA20210BA8FFF7BFFC04009C
:106E6000F7E6C046B4FCFFFF34B0020830B00208B9
:106E700020AE020860A80208200000100001600493
:106E800001000040C0AC0208090000013DB8F396C3
:106E9000076900000023F0B51D4C0700A5446946B2
:106EA000022000930193FFF70DF900280ED0012670
:106EB0000098002801D0FFF727F90198002801D099
:106EC000FFF722F93000134B9D44F0BD01A90120CA
:106ED000FFF7F8F80600041EE9D10098A742E7D9A9
:106EE00080233D1BDB009D4200D91D002B0002AA20
:106EF0002100FFF72FF90028D9D12B0002AA210089
:106F00000198FFF753F90028D1D16419E5E7C0468D
:106F1000F4FBFFFF0C040000F0B500242500614ED7
:106F20009BB033686048D96801F0B0F833685F48B7
:106F3000D96801F0ABF85E4FBB6A0393039BAB4289
:106F400069D133682200D8685A4901F045F85A4B94
:106F5000DB78002B00D1A1E0002305A902200593D6
:106F60000693FFF7AFF8002821D106A90130FFF7FB
:106F7000A9F800281BD1514A0C2108A8F9F7FCFAFE
:106F8000002814D110224E4908A8F9F717FB041E57
:106F90000DD10600BB6B0133FF330293059B5B6889
:106FA0000393029BB34200D86EE0002C46D00598B4
:106FB000002801D0FFF7A8F80698002801D0FFF7B5
:106FC000A3F8404B1B68002B02D00C20F9F71CFBE8
:106FD000102200213A4801F0A5F83B6D00219A6883
:106FE0000220FFF749FD43425841FEF761FA0C23A6
:106FF0007A6D396D013A5343CB185A6849680220BB
:10700000511A9A68FFF738FD43425841FEF750FA8B
:1070100000201BB0F0BD0C236B437A6A2100D3180B
:107020009B6801201A000293FFF726FD4342584156
:10703000FEF73EFA029B0135E4187FE7029B9D1B99
:107040008023DB009D4200D91D00039B0095991908
:107050001D4B2A00C91807AB019308A81B4BF9F771
:10706000BDFA079B0400AB420BD1002899D12B003D
:10707000164A31000698FFF799F8002897D176193B
:107080008FE7012464428CE7002C00D08FE707AB28
:1070900022000E4908A8F9F77FFA88E72000FFF7D9
:1070A000F9FE9AE784A1020863DC0D1088DC0D105C
:1070B00060A802089EDC0D1020AE020800016004EA
:1070C000C0AC020834B0020800040010C0A80208D6
:1070D00073B5164E164CF368626A5B0A01A901206B
:1070E0000193FFF743F9012500281AD1019B226D76
:1070F000A362F36801A95B0A02300193FFF736F936
:10710000051E10D1019B206A6365FFF709F906008F
:10711000A06DFFF705F9331C864200D2031C5C34D6
:107120002370280076BD0125FBE7C04640A1020878
:1071300060A80208F0B50C266E4F89B0FB6800907D
:107140005C0A7443200000F0AFFF0190200000F0C3
:10715000ABFF019B684C0290636220650020FFF743
:10716000E4F82100C0B22031FEF7ACFF43425841A1
:10717000FEF79EF90120FFF7D8F82100C0B24C318C
:10718000FEF7A0FF43425841FEF792F92100032089
:107190005831FEF797FF43425841FEF789F9FFF750
:1071A00097FF051E19D0554BFA681B68520A5449BF
:1071B000D86800F011FF019800F080FF029800F0FD
:1071C0007DFFA06DFEF7A0FFE06CFEF79DFF206A3B
:1071D000FEF79AFF280009B0F0BDFFF723FC051E5B
:1071E000E9D1FB68A06A5B0A984202D8626D9A42B4
:1071F00019D9424B43481B68D96800F047FF00206B
:10720000FFF752FC050068426841FEF751F9002D76
:107210005ED1236A00995A780A715B680C60039307
:10722000039A8A60C7E7904239D108234643626ACD
:10723000216D08369E4237D1334E7378002BDED055
:107240000C22002105A800F06DFF0120FEF730F9A7
:10725000FFF75AFA831E0500022B0DD8274B1B6837
:10726000D968F378002B2CD0284800F00FFFFFF7E7
:1072700095FC00282ED005250120FEF719F9012DD7
:10728000BDD0002D01DD052D2EDD1C4B20481B68D7
:10729000D96800F0FBFE0020FEF70AF9FEE7174B65
:1072A0001C481B68D968A8E71800D558CB580C3083
:1072B0009D4204D0114B18481B68D9689DE7030014
:1072C000B8E7164800F0E2FE0120FFF7EDFBD0E73B
:1072D000032570E70120FEF7EBF8FFF71DFE4342A0
:1072E0005841FEF7E5F8C7E70020FFF79BFB051EB6
:1072F00085D060E740A1020860A8020884A10208C6
:10730000CCDC0D1011DD0D1020AE0208BBDD0D1020
:10731000E3DD0D1043DD0D1082DD0D10CDDD0D1010
:1073200010B5017804000A00303AD3B2092B1FD8F7
:1073300011000A0161780B00303BD8B2092824D82B
:107340009918A27809011300303BD8B209282AD82D
:107350005A18E378120118003038C1B28018092990
:1073600005D91900413905292BD8373B981810BD8C
:107370000B00413B052B01D83739DAE70B00613BA5
:107380000020052BF3D85739D3E70B00413B052BE1
:1073900002D837398918D4E70B00613B0020052B50
:1073A000E5D85739F6E71300413B052B02D8373AA9
:1073B0005218CEE71300613B0020052BD7D8573A6F
:1073C000F6E71900613900200529D0D8573BCDE7F1
:1073D000F7B50B7807004E1C222B0FD00026554B1B
:1073E00019603000FEBD02331A780130222A08D01D
:1073F000002A06D05C2AF6D00133F5E733000020DE
:10740000F2E74D4B1B6898470190041E07D1019E7F
:10741000E7E7721C5C2B13D023700134160033781D
:10742000222B01D0002BF4D1002323703378223B90
:107430005A425341F618019B3B610423FB60D0E79D
:1074400073786E2B17D007D8611C622B0CD0662B7B
:107450000FD0237001340AE0742B0ED0752B0ED0A0
:10746000722BF6D10D23F4E7082323700C000132B0
:10747000D4E70C23F9E70A23EBE70923E9E7B01C7B
:10748000FFF74EFF2D4B2E49C3180500721D8B428E
:10749000EDD90028EBD02B4BC3188B4227D8B379FA
:1074A0005C2BE4D1F379752BE1D130000830FFF784
:1074B00037FF3200214B2249C3180B328B42D6D8FA
:1074C000214BAD021D4080238005800D05435B02EA
:1074D000ED181E4BE11C9D4223D803234C1E3F2078
:1074E00080212840494201432170AD0910E07F28E6
:1074F00009D8012301341648611EC05C013B0543D5
:107500000D70E418B3E7134B9842E2D8022302341B
:107510003F20802128404942013C01432170AD09B0
:10752000E9E73F20802328405B420343E370AD0935
:107530000423D3E7D0AD020880A102080024FFFF96
:10754000FF0300000028FFFF00FC0F00FFFF00000A
:1075500019DE0D10FF070000002803D00378013B5F
:107560001F2B00D970470130F6E70000064B10B51D
:107570001B6828209847041E03D02822002100F011
:10758000D1FD200010BDC04680A10208F0B5050065
:1075900087B00E1E01D1002413E00422754930008B
:1075A00001F045FC002803D10223EB60341D08E004
:1075B00005227149300001F03AFC002804D1E8604E
:1075C000741D200007B0F0BD04226C49300001F0AA
:1075D0002EFC002806D101230122EB600023AA61C2
:1075E000EB61E3E73378222B05D131002800FFF768
:1075F000EFFE0400E5E71A00303AD2B22D2B01D09D
:10760000092A1AD8340000E0013423781A00303AED
:10761000092AF9D92D2BF7D0A71B3A00310068466B
:1076200000F077FD00236A466846D35500F0CEFC93
:107630000323A861E961EB60C3E75B2B37D1563BBD
:10764000EB60701CFFF788FF037804005D2B01D10D
:107650000134B6E7FFF78AFF061EA8609BD0200022
:10766000FFF77AFF01003000FFF790FFFFF774FF8C
:107670000400002C00D18EE723782C2B04D05D2B46
:10768000E6D03F4B1C6086E7FFF770FF051E00D178
:1076900081E730604660601CFFF75EFF0100280054
:1076A000FFF774FFFFF758FF2E000400E1E77B2B84
:1076B0005DD1753BEB60701CFFF74EFF0378040053
:1076C0007D2BC5D0FFF752FF061EA86000D162E7F0
:1076D0002000FFF741FF01003000FFF779FEFFF7C0
:1076E0003BFF002800D156E7002433693461336240
:1076F00003783A2B02D0224B186062E70130FFF783
:107700002BFF01003000FFF741FFFFF725FF0400CA
:10771000002C00D13FE723782C2B02D07D2B97D073
:10772000AFE7FFF723FF051E00D134E73060466066
:10773000601CFFF711FF01002800FFF749FEFFF76B
:107740000BFF002800D126E700242B692C612B6257
:1077500003783A2BCFD10130FFF7FEFE010028005D
:10776000FFF714FFFFF7F8FE2E000400D0E7044BEC
:107770001E6010E720DE0D1025DE0D102BDE0D1033
:10778000D0AD02080849094A002803D1084B0B6014
:10779000084B07E00368002B00D1054B0B604368E2
:1077A000002BF5D01360704780A102087CA102086D
:1077B000A9800D10BD800D10F8B58026040076005C
:1077C000002C00D1F8BDE3682768334204D1A068DB
:1077D000002801D0FFF7F0FFE3680B4D334204D1DE
:1077E0002069002801D02B6898478022E368920026
:1077F000134204D1206A002801D02B68984720004A
:107800002B6898473C00DBE77CA10208F7B5050030
:107810000E000192FFF7AAFE0023134F04003B6005
:1078200098420CD02800FFF797FE01002000FFF7D8
:10783000ADFE051E05D12000FFF7BEFF002420008D
:10784000FEBD019B002B0AD0FFF786FE03780500E2
:10785000002B04D02000FFF7AFFF3D60EEE7002EC5
:10786000EDD03560EBE7C046D0AD0208002210B580
:107870001100FFF7CBFF10BD0300093B0122042BD1
:1078800002D920384242424110007047F0B500252D
:10789000170006002C0089B003930E9B02901B0C6E
:1078A000DBB204930E9B00911B0ADBB205930E9B87
:1078B000DBB20793731C069333780193002B08D037
:1078C000009B002B22DB029A731C9B1A009A9A429F
:1078D0001CDA0E9BDBB2002B00D1B4E0019A9A4275
:1078E00000D0AEE0009B002B06DB029A731C9B1AB3
:1078F000009A934200DDA4E0B31C7678032D00D9F2
:10790000A1E0280000F0ACF88989637B0198FFF7BB
:10791000B3FF002839D1079B019A9342D9D04F4E2B
:107920001100300001F05CFA031E08D1049B019A9B
:1079300093420BD0059B93426FD133003F33032D0D
:1079400023D8280000F08CF80510233533003E338F
:10795000F5E7002F06D0039A94425ED23F4A9B1A65
:107960009B003B55012510E0621C002F0BD00399B2
:107970008A4252D239493C195B1A217818110143C5
:107980001B012170BB5414000225069E92E7621C65
:10799000002F0BD003998A423FD230493C195B1A21
:1079A0002178981001439B012170BB5414000325DA
:1079B000EBE7002F08D0039A94422ED227493A19B8
:1079C0005B1A11780B43137001340025DDE71D00AD
:1079D000002E22D0009B002B22DB029B009AEB1A88
:1079E0009A421DDA019BB34217D1009B002B04DDA4
:1079F000029B009AEB1A93420FDC2E786B1C029AC2
:107A00009D1A002E04D0009B002B11DBAB420FDA35
:107A1000002F18D03B5D002B15D00124644219E0E3
:107A20003000FFF729FF0028DCD02E780135CFE7A2
:107A30003000FFF721FF0028EFD0029B5E5D01358B
:107A4000DFE7002DE9D1039B9C42E6D2002F01D055
:107A500000233B55200009B0F0BDC04630DE0D10BC
:107A600002B4714649084900095C49008E4402BCD1
:107A70007047C046002243088B4274D303098B42EF
:107A80005FD3030A8B4244D3030B8B4228D3030CEE
:107A90008B420DD3FF22090212BA030C8B4202D390
:107AA0001212090265D0030B8B4219D300E0090AB8
:107AB000C30B8B4201D3CB03C01A5241830B8B42C1
:107AC00001D38B03C01A5241430B8B4201D34B03AA
:107AD000C01A5241030B8B4201D30B03C01A52410F
:107AE000C30A8B4201D3CB02C01A5241830A8B4294
:107AF00001D38B02C01A5241430A8B4201D34B027D
:107B0000C01A5241030A8B4201D30B02C01A5241E0
:107B1000CDD2C3098B4201D3CB01C01A5241830994
:107B20008B4201D38B01C01A524143098B4201D3CE
:107B30004B01C01A524103098B4201D30B01C01AF9
:107B40005241C3088B4201D3CB00C01A5241830873
:107B50008B4201D38B00C01A524143088B4201D3A0
:107B60004B00C01A5241411A00D201465241104600
:107B70007047FFE701B5002000F0F0F802BDC046F5
:107B80000029F7D076E7704703460B437FD40022E5
:107B900043088B4274D303098B425FD3030A8B42A1
:107BA00044D3030B8B4228D3030C8B420DD3FF220B
:107BB000090212BA030C8B4202D31212090265D0D9
:107BC000030B8B4219D300E0090AC30B8B4201D38C
:107BD000CB03C01A5241830B8B4201D38B03C01AD3
:107BE0005241430B8B4201D34B03C01A5241030B4A
:107BF0008B4201D30B03C01A5241C30A8B4201D3FB
:107C0000CB02C01A5241830A8B4201D38B02C01AA5
:107C10005241430A8B4201D34B02C01A5241030A1C
:107C20008B4201D30B02C01A5241CDD2C3098B4201
:107C300001D3CB01C01A524183098B4201D38B017E
:107C4000C01A524143098B4201D34B01C01A524121
:107C500003098B4201D30B01C01A5241C3088B4266
:107C600001D3CB00C01A524183088B4201D38B0051
:107C7000C01A524143088B4201D34B00C01A5241F3
:107C8000411A00D201465241104670475DE0CA0FCA
:107C900000D04942031000D34042534000229C468A
:107CA00003098B422DD3030A8B4212D3FC22890194
:107CB00012BA030A8B420CD3890192118B4208D36A
:107CC000890192118B4204D389013AD0921100E0CC
:107CD0008909C3098B4201D3CB01C01A52418309E0
:107CE0008B4201D38B01C01A524143098B4201D30D
:107CF0004B01C01A524103098B4201D30B01C01A38
:107D00005241C3088B4201D3CB00C01A52418308B1
:107D10008B4201D38B00C01A5241D9D243088B4207
:107D200001D34B00C01A5241411A00D201466346AA
:107D300052415B10104601D34042002B00D549420E
:107D4000704763465B1000D3404201B5002000F04D
:107D500005F802BD0029F8D016E770477047C04605
:107D6000002B11D1002A0FD1002900D1002802D008
:107D70000021C943081C07B4024802A14018029020
:107D800003BDC046D9FFFFFF03B4684601B50298A2
:107D900000F030F8019B9E4602B00CBC7047C04614
:107DA000F0B5CE46474615042D0C2E0080B50704CD
:107DB000140C3F0C9946030C7E435D4367436343B9
:107DC0007F19340CE4199C46A54203D980235B0239
:107DD0009846C4444B4643435143250C36046544FE
:107DE000360C2404A4195B19591820000CBC9046C9
:107DF0009946F0BDF0B54F464646D646C0B504009C
:107E000082B00D00914698468B422FD82CD0414627
:107E1000484600F0CFF829000600200000F0CAF81C
:107E2000331A9C46203B9A4600D576E04B46524694
:107E300093401F004B46624693401E00AF4228D835
:107E400025D05346A41BBD41002B00DA7BE0002265
:107E50000023009201930123524693400193012392
:107E600062469340009318E08242D0D9002200235A
:107E7000009201930A9B002B01D01C605D6000986A
:107E8000019902B01CBC90469946A246F0BDA3429F
:107E9000D7D900220023009201936346002BE9D03A
:107EA000FB079846414672080A437B0866460EE087
:107EB000AB4201D1A2420CD8A41A9D410120241941
:107EC0006D410021013E24184D41002E06D0AB42E9
:107ED000EED9013E24196D41002EF8D10098019988
:107EE000534600196941002B23DB2B005246D34037
:107EF0002A006446E2401C0053461500002B2DDB8F
:107F000026005746BE40330026006746BE4032007A
:107F1000801A994100900191ACE7624620239B1A98
:107F20004A46DA406146130042468A4017001F4322
:107F300080E7624620239B1A2A0066469A40230067
:107F4000F3401343D4E76246202300219B1A00220A
:107F5000009101920122DA40019280E720236246DB
:107F600026009B1ADE402F00B0466646B7404646C4
:107F70003B003343C8E7C0461C2101231B04984241
:107F800001D3000C10391B0A984201D3000A0839AA
:107F90001B09984201D30009043902A2105C401861
:107FA0007047C04604030202010101010000000005
:107FB0000000000010B5002903D1FFF7DDFF2030DD
:107FC00002E0081CFFF7D8FF10BDC04610B50A221A
:107FD000002100F0FDFF10BD0EB403B5010003AB9E
:107FE000044804CB0068019300F074F902B008BCA7
:107FF00003B0184784A1020870B505000E001400F4
:10800000002804D08369002B01D102F02BF81C4B0F
:108010009C420FD16C68A3891B0702D52369002BF2
:1080200021D12100280001F049F800281BD00120AF
:10803000404270BD134B9C4201D1AC68EBE7124B40
:108040009C42E8D1EC68E6E7A3680136013BA360F7
:10805000002B04DAA26993420ADB0A2908D02368BC
:108060005A1C2260197031780029EDD10800E0E730
:108070002200280000F0C0FF431CF4D1D7E7C0461F
:10808000F4DF0D1014E00D10D4DF0D1010B5034B0C
:108090000A0001001868FFF7AFFF10BD84A10208B5
:1080A000EC3000687047000010B5034B0100186801
:1080B00000F08AF810BDC04684A1020810B5034B39
:1080C0000100186800F036F810BDC04684A102080F
:1080D00082B0002900D101A9101E06D0002B06D0C5
:1080E00013780B601078431E984102B0704702204D
:1080F0004042FAE730B50024A24201D1002005E059
:10810000035D651C0C5DA34201D0181B30BD2C0023
:10811000F2E7002310B59A4200D110BDCC5CC454E4
:108120000133F8E703001218934200D17047197029
:108130000133F9E770B50500002910D00C1F236842
:10814000002B00DAE418280002F0A3F81D4A136897
:10815000002B05D163601460280002F09BF870BD0D
:10816000A34209D9216860188342F3D118685B687B
:1081700041182160EEE713005A68002A01D0A2429C
:10818000F9D919685818A0420BD120680918581855
:1081900019608242E0D110685268411819605A6033
:1081A000DAE7A04202D90C232B60D5E721686018DA
:1081B000824203D1106852684118216062605C609D
:1081C000CAE7C046D4AD0208032370B5CD1C9D4359
:1081D000083506000C2D1ED20C25A9421DD83000F2
:1081E00002F057F8254A14682100002919D1244CBF
:1081F0002368002B03D1300000F0E0FD206029004F
:10820000300000F0DBFD431C2BD10C233000336029
:1082100002F040F803E0002DDFDA0C233360002089
:1082200070BD0B685B1B19D40B2B03D90B60CC18EA
:10823000256003E04B688C420DD11360300002F0E2
:1082400029F8200007220B30231D9043C31AE7D0E2
:108250005A42E250E4E763600C00EFE70C00496823
:10826000C3E70323C41C9C43A042E1D0211A300081
:1082700000F0A4FD431CDBD1C7E7C046D4AD020823
:10828000D8AD0208936810B5013B9360002B04DA67
:108290009469A34207DB0A2905D01368581C1060B3
:1082A0001970080010BD00F0A7FE0100F9E7F8B54D
:1082B00006000F001400D518AC4201D1002007E0E1
:1082C00021783A003000FFF7DDFF0134431CF3D181
:1082D000F8BD0000F0B59FB002900F0016000593A6
:1082E000002805D083690493002B01D101F0BAFE68
:1082F0007B4B9F425BD1029B5F68BB891B0762D5AA
:108300003B69002B5FD0002306AC636120336376AA
:108310001033A37635002B78002B01D0252B5CD1B0
:10832000AB1B04930CD0320039000298FFF7BFFF5B
:10833000431C00D1C4E06269049B944663446361BA
:108340002B78002B00D1BBE0012200235242626057
:1083500002A9543252186E1C2360E360A3601370AC
:10836000A365317805225F4801F088FF751C00285D
:1083700035D12268D30604D5532302A95B182021E6
:108380001970130704D5532302A95B182B21197008
:1083900033782A2B2CD0350000210A20E3682A7874
:1083A0006E1C303A092A64D900292ED026E04E4BA3
:1083B0009F4202D1029B9F689FE74C4B9F429CD1FA
:1083C000029BDF6899E73900029800F077FE0028E9
:1083D00099D0012040421FB0F0BD01359BE7414BD1
:1083E0002268C01A01238340134323602E00B8E79C
:1083F000059B191D1B680591002B01DB099304E007
:108400005B42E3600223134323602B782E2B0AD1B7
:108410006B782A2B35D1059B02351A1D1B680592F6
:10842000002B2BDB0793324E29780322300001F01A
:1084300025FF002806D04023801B83402268013599
:1084400013432360297806222A486E1C217601F006
:1084500015FF00283AD0284B002B25D10722059B79
:1084600007339343083305936369039A9B18636149
:1084700050E7434301219B18350090E701235B42FD
:10848000D0E700230A201A000135636029786E1CAA
:108490003039092903D9002BC5D00792C3E74243DD
:1084A000012352183500F1E705AB00933A00134B56
:1084B0002100029800F0C0F80390039B0133D3D150
:1084C000BB895B0600D584E70B9884E705AB009376
:1084D0003A000A4B2100029800F068FBECE7C04626
:1084E000F4DF0D107EDE0D1014E00D10D4DF0D1042
:1084F00084DE0D1088DE0D1039860D10AF820D1050
:10850000F0B58BB014001D1E129953DA8024240696
:108510001B191D0014002D230B702023149E032211
:108520009E43462E07D03300453B59424B4110999C
:10853000013ACB18109309AB049308AB0393139B38
:1085400000920293109B220001932B0000F0B2FED8
:108550000700472E02D1119BDB0724D5109BFB1887
:108560000793462E14D13B78302B0CD100220023E8
:108570002000290002F052FA002804D10123109AA9
:108580009B1A139A1360139B079A1B68D3180793BF
:10859000002200232000290002F040FA30220028A7
:1085A0000DD0079B09933800099B159ADB1B1360BC
:1085B0000BB0F0BD0023AFE7591C09911A70099B5D
:1085C00007998B42F8D3EEE7F0B5831C85B0019391
:1085D00006000C0002702B23002901DA2D234C42E7
:1085E0007370092C22DD02ABDD1D20000A21FFF78C
:1085F000B1FB6F1E3031397020000A21FFF7C4FA39
:10860000040009280BDC023D3034019B2C7002AAC7
:1086100007321800AA4204D8801B05B0F0BD3D0007
:10862000E3E72A7801351A700133F0E73023E418C4
:10863000B370301DF470EFE7F0B595B00C000A92FE
:108640000B931A9D099001F0A1FD036818000C938B
:1086500000F0E6FB0023129323680E900D930D9912
:10866000277E2B680722C90545D59B1893431A001E
:1086700008322A601A685B68A264E3640122E56C30
:10868000A66C6B005B080F935242AC4B30000F9905
:1086900003F0D2FE002830D10122A84B5242300014
:1086A0000F9902F0CBF9002827D1002200233000D7
:1086B000290002F0B9F9002803D023002D2243330A
:1086C0001A709F4D472F00D89E4D032300260D9A08
:1086D000236101339A4322600B9B13AA009321006C
:1086E0000A9B099800F0F4F9431C00D093E00120A4
:1086F000404215B0F0BD0733B8E732002B00300020
:10870000290003F099FE002804D08F4D472FDCD8B4
:108710008E4DDAE780230D996268DB000B43511C14
:1087200043D10732626012AA0021059211AA039276
:10873000232223600691019308A9636852180292CC
:10874000009332002B0004970998FFF7D9FE2023ED
:108750003A0005009A43472A07D1119BDA1C02DB35
:108760006268934245DD023FFFB21199652F25D81B
:10877000200001393A0050301191FFF725FF129A7D
:10878000060013182361012A02DC2268D20701D5F2
:1087900001332361232308AA9B181B78002B9BD04D
:1087A00023002D2243331A7096E7672F00D176E11C
:1087B000472FB8D1002AB6D10122B3E7662F19D1CD
:1087C000636800290CDD2161002B02D12268D207E9
:1087D00002D501335B182361119B0026A365D9E7FD
:1087E000002B03D101222168114200D09A1C226182
:1087F000F2E76727119B129A934205DB22682361F7
:10880000D207E9D50133E6E70121002B01DC491845
:10881000C91A5218EBE72268530508D423692A00C5
:108820000A9909980B9DA847431C29D15FE7652F3A
:1088300000D8E0E0A06CE16C0022002302F0EEF82A
:10884000002834D00123424A0A9909980B9DA84771
:10885000431C00D14BE7119B129A934202DB236821
:10886000DB070DD50B9D0E9B0C9A0A990998A8471A
:108870000025431C00D13AE7129B013BAB420ADCC6
:1088800023689B0700D508E1139BE068984200DB52
:108890002FE718002DE7220001231A320A990998C0
:1088A0000B9EB047431C00D121E70135E4E7119B43
:1088B000002B2DDC0123264A0A9909980B9EB0470C
:1088C000431C00D113E7119B002B05D1129B002BF9
:1088D00002D12368DB07D3D50B9E0E9B0C9A0A9915
:1088E0000998B0470026431C00D100E7119B5B426A
:1088F000B34201DC129B92E7220001231A320A994B
:1089000009980B9FB847431C00D1F0E60136EDE70C
:10891000A36D129F9F4200DD1F00002F08DD3B006A
:108920002A000A9909980B9EB047431C00D1DEE645
:1089300000230D93FB43DB170F9318E0FFFFEF7F3E
:1089400093DE0D108FDE0D109BDE0D1097DE0D10E7
:108950009FDE0D10220001231A320A9909980B9EFE
:10896000B047431C00D1C2E60D9B01330D930F9B12
:10897000A66D0D9A3B40F31A9342EBDC119B129AC1
:10898000AD19934210DB2368DB070DD4129F119BB6
:10899000BE1BFF1AB74200DD3700002F0DDCFE437F
:1089A000F31700250C931CE00E9B0C9A0A9909986A
:1089B0000B9FB847431CE9D199E63B002A000A996E
:1089C00009980B9DA847431CE9D190E6220001239A
:1089D0001A320A9909980B9EB047431C00D186E6CB
:1089E0000135119A129B0C999B1A3A000A409B1A66
:1089F000AB42EBDC44E7129B012B02DC01231A4261
:108A000032D001232A000A9909980B9FB847431CCA
:108A100000D16CE60E9B0C9A0A9909980B9F0135C0
:108A2000B847431C00D162E6A06CE16C129B0022A7
:108A30005F1E002301F0F2FF3B00002814D0002548
:108A40000AE0220001231A320A9909980B9FB847BD
:108A5000431C00D14BE60135129B013BAB42F0DCDD
:108A6000220033005032DBE62A000A9909980B9D58
:108A7000A847431CF4D13AE62200012319320A998F
:108A800009980B9EB047431C00D130E60135E368DE
:108A9000139A9B1AAB42EFDCF6E60025F7E7002AB3
:108AA00000D189E60021069112A9059111A903912F
:108AB000232108A809182360019300922B00049732
:108AC000029132000998FFF71BFD050045E6C046FC
:108AD000F7B5150001938A680B6900900C0093426A
:108AE00000DA130022002B6043321278002A01D0F2
:108AF00001332B6023689B0602D52B6802332B6061
:108B0000062723681F4027D0230043331B785A1EB3
:108B100093412268920630D4220001994332009892
:108B2000089EB047431C25D0062320682A68E168C8
:108B300003400025042B03D18D1AEB43DB171D40A6
:108B4000A3682269934201DD9B1AED180027BD42FC
:108B500020D1002010E00137E3682A689B1ABB424D
:108B6000D2DD22000123193201990098089EB047F6
:108B7000431CF0D101204042FEBD3020E1184331BA
:108B8000087021005A1C45310978A218433202337B
:108B90001170C1E7220001231A3201990098089E42
:108BA000B047431CE6D00137D1E70000F0B589B0EB
:108BB00004920A0043320593039002920A7E0C004D
:108BC0000E9B6E2A00D186E01FD8632A33D008D8C6
:108BD000002A00D18CE0582A4DD0250042352A7059
:108BE00030E0642A01D0692AF7D1196825680A1D86
:108BF000280629D508681A60002803DA2D23029A6E
:108C0000404213706B4E0A274FE0732A74D008D885
:108C10006F2A1FD0702AE0D1202209680A432260FF
:108C200003E0752A16D0782AD7D122007821453260
:108C30001170614E22E025001A684235111D19603D
:108C400013682B70012365E008681A606906D3D5A4
:108C500000B2D1E719682568081D186008682E065B
:108C600005D5544E08276F2A1BD00A2719E06D0638
:108C7000F7D580B2F5E745314E4E0A701868226884
:108C8000011D00681960150621D5D30702D52023E0
:108C90001A4322601027002803D1202322689A4318
:108CA00022602300002243331A706368A360002B04
:108CB00058DB0422216891432160002854D1029D91
:108CC000002B5AD02500337842352B7055E05506DD
:108CD000DBD580B2D9E71A680D68101D49691860A4
:108CE00013682E0601D5196002E06D06FBD51980C8
:108CF0000023029D23614FE01A68111D1960156859
:108D000000216268280001F0B9FA002801D0401B58
:108D10006060636823610023029A13703CE023695A
:108D20002A0004990398059DA847431C3ED0236858
:108D30009B0715D4079BE068984239DA180037E0A2
:108D400022000123193204990398059EB047431C61
:108D50002CD00135E368079A9B1AAB42F0DCE9E7B7
:108D60000025F7E70028ADD0029D3900FEF708FF87
:108D7000735C013D2B700028F7D1082F09D12368BF
:108D8000DB0706D563682269934202DC3023013D8C
:108D90002B70029B5B1B2361059B07AA009321009C
:108DA000049B0398FFF794FE431CB8D10120404276
:108DB00009B0F0BDA1DE0D10B2DE0D10002370B5BC
:108DC000064C05000800236003F014FC431C03D18B
:108DD0002368002B00D02B6070BDC0463CB0020859
:108DE000C9B20378002B04D08B4200D17047013008
:108DF000F7E74B42594149420840F7E702780B78C0
:108E0000002A03D0013001319A42F7D0D01A7047BE
:108E100003000A7801311A700133002AF9D1704732
:108E20000023C25C0133002AFBD1581E7047002387
:108E300030B59A420AD0013AC45CCD5CAC4204D150
:108E4000934202D00133002CF6D1631B180030BDD1
:108E500030B50500002A00D130BD0C78013A6B1CFA
:108E60002C700131002C05D19A189A42F4D01C7054
:108E70000133FAE71D00EDE7F0B51F000E008DB0DD
:108E80000B900291039212983478FFF709F90822A7
:108E900000194378751C134053D12D2C53D174788D
:108EA000B51C01330193002F00D18AE0102F0AD1A5
:108EB000302C08D120222B789343582B00D07AE015
:108EC00010276C780235019B002B41D1013B0493A4
:108ED0003E4B05933A00FB17049805990893FEF75B
:108EE0003FFF002309900E00002000210A9222007B
:108EF000303A092A31D81400A7423DDD5A1C1DD052
:108F0000B14236D802D1099B984232D8099B83429C
:108F100006D18E4204D101230A9A5B42A2420DDBA4
:108F20000B00020008993800FEF73AFFE317069499
:108F30000793069B079CC018614101232C780135DB
:108F4000D5E72E009FE72B2CACD1B51C7478A9E790
:108F50000023049380231B06BBE72200413A192A11
:108F600001D8373CC8E72200613A192A04D8573C97
:108F7000C2E701235B42E1E75A1C09D10B9A233374
:108F80001360039B04980599002B0ED10DB0F0BD22
:108F9000019A002A04D006000F0000217042B94156
:108FA000039A002AF2D0002B01D06B1E0293039B80
:108FB000029A1A60EAE73024002F00D083E70827DE
:108FC00081E7302C00D175E70A277CE7FFFFFF7FA0
:108FD00037B51300064A05001068046A002C00D15A
:108FE000044C0A0000942900FFF746FF03B030BD8F
:108FF00084A10208E8A10208F8B505000E001400DB
:10900000002804D08369002B01D101F02BF8224BFA
:109010009C422DD16C68A369A360A3891B0731D53D
:109020002369002B2ED023682269F7B2981A63694E
:10903000F6B2834205DC2100280000F0A5FF0028DD
:1090400026D1A3680130013BA36023685A1C22602B
:109050001F706369834204D0A389DB071AD50A2EE7
:1090600018D12100280000F08FFF002812D00FE057
:109070000A4B9C4201D1AC68CDE7094B9C42CAD156
:10908000EC68C8E72100280000F018F80028CAD0D2
:10909000012676423000F8BDF4DF0D1014E00D100B
:1090A000D4DF0D100B1E04D0FF2A04D98A230360DD
:1090B0008B3B180070470A700123FAE7364B70B5F6
:1090C0001D6806000C00002D05D0AB69002B02D1F5
:1090D000280000F0C7FF314B9C420FD16C680C2375
:1090E000E25E93B219072DD4D90611D409230120C9
:1090F000336037331343A381404270BD284B9C42F9
:1091000001D1AC68EBE7274B9C42E8D1EC68E6E77D
:109110005B0713D5616B002908D0230044339942C3
:1091200002D03000FFF706F8002363632422A389EE
:109130009343A38100236360236923600823A289EA
:109140001343A3812369002B0BD1A0218022A38983
:10915000890092000B40934203D02100300001F0BF
:1091600049F80123A289134011D00023A360636949
:109170005B42A361002023698342BED10C23E25EDF
:109180001306BAD540231343A3810138B5E79207EC
:1091900000D46369A360EDE784A10208F4DF0D1039
:1091A00014E00D10D4DF0D10F0B503690C6989B01F
:1091B000070005910026A34265DB0B00013C143338
:1091C000A50003935B1904930300143302935D1904
:1091D000049B28681B68591C0193FEF74BFC019007
:1091E000B04229D0039B02989C460696624608CA64
:1091F0009446019A99B251431B0C534389190A0CA6
:109200009B1807931E0C036889B29AB2069BD2186A
:109210000368521A190C6B469B8BCB1A11145B18FE
:10922000191492B21B041A43049B069104C06345AF
:10923000DCD22B68002B2DD00599380001F040FAC4
:1092400000281FDB0025019B02980133039901933D
:10925000026808C992B255199AB2AA1A05681B0C7D
:109260002D0CEB1A15145B191D1492B21B04134339
:1092700008C0049B8B42EBD2029AA300D3181A6851
:10928000002A11D0019E300009B0F0BD2B68002BE0
:1092900004D1013C029B043DAB42F7D33C61CBE7D8
:1092A0001A68002A04D1013C029A043B9A42F7D37F
:1092B0003C61E7E7F0B516001F00446A9BB00290DE
:1092C000239D06960797002C08D11020FEF7ECFE90
:1092D000029B5862446084600460C460029B5B6AC5
:1092E000196800290BD05A68012393404A608B60AB
:1092F000029801F008F80022029B5B6A1A60002FB6
:1093000020DA01232B607B005B080793079CB24B9C
:10931000220017931A409A4217D1B04B229A136039
:10932000069B002B03D1240301D100F087FDAC4B39
:10933000249A0893002A02D0AA4B249A1360089812
:109340001BB0F0BD00232B60E0E7069E079F0022C4
:1093500000233000390001F061FB051E0BD0012312
:10936000229A1360A04B249A0893002AE7D09F4AC0
:1093700024990A60E3E718AB019319AB009332001C
:109380003B00029801F01AFA630003905B0D74D061
:109390003A03974C120B14432100964A300016955D
:1093A0009E180022944B02F0FFFC944A944B02F06A
:1093B00089FA944A944B01F05FFB040030000D00E1
:1093C00003F08CF8914A924B02F07CFA02000B00F9
:1093D0002000290001F050FB04000D0003F048F8C4
:1093E0000022070000232000290001F01DFB0028B7
:1093F00009D0380003F072F82B00220001F00EFBB8
:10940000434258413F1A01231493162F0DD8814926
:10941000FB00C91808684968069A079B01F018FB09
:10942000002846D00023013F1493189B9E1B002365
:109430000A933300013B0B9304D501239B1B0A9332
:1094400000230B93002F36DB0B9B1197DB190B933B
:1094500000230493209B0124092B00D984E0052BD1
:1094600002DD0024043B2093209B981E032800D992
:1094700084E0FEF7F5FA7577286A189B199A9E180A
:10948000654BF218202A0FDD40239B1A9C40634B4A
:109490000698F318D840204303F05AF80123604C93
:1094A000013E091916937CE7202306989B1A9840E1
:1094B000F2E71490B9E70A9BDB1B0A937B42049303
:1094C00000231193C6E701230D93219B002B59DD47
:1094D0000C930993029A556A00226A6004321000C4
:1094E00014306968984252D9029800F0D4FE029B69
:1094F00028605B6A1B680893099B0E2B00D90AE160
:10950000002C00D107E1069B079C12931394002FB7
:1095100000DC89E00F213A003E4B0A40D2009B1844
:109520001D685E6802233C110E93E3060BD53D4B8C
:109530000C401A6A5B6A1298139901F0B9FD032373
:10954000069007910E9300233AE001230D93219B8F
:10955000FB180C9301330993002BBBDC0123B9E703
:109560000023B1E70023F1E700230D942093013B92
:1095700000220C93099313332192ABE701230D933F
:10958000023BF5E701230C9309931A00F4E701313C
:1095900069605200A3E701231C420ED00E9B214AB2
:1095A00001330E93109B2800DB009B1831001A68D2
:1095B0005B6802F087F905000E00109B6410013310
:1095C0001093002CE7D1069807992A00330001F088
:1095D0006FFD0690079142E00000F07F0F2700002A
:1095E000CDDF0D10D0DF0D109FDE0D10A0DE0D10B1
:1095F0000000F03F01FCFFFF0000F83F61436F6394
:10960000A787D23FB3C8608B288AC63FFB799F509B
:109610001344D33F60E00D10320400001204000038
:10962000000010FE38E00D1002230E93002F16D01C
:10963000129813997C420D332340CE4ADB00D31895
:109640001A685B6802F03EF9002301261D000690AF
:1096500007912411002C00D08CE0002BB9D1149B71
:10966000002B00D196E0069C079D0022C24B2000F3
:10967000290001F0D9F9002800D18BE0099B002BCB
:1096800000D187E00C9B002B41DDBC4B0022200069
:10969000290002F017F90E9B0690079101330E93F3
:1096A0000C9B7E1E0E98109302F018FF069A079BE3
:1096B00002F008F90022B24B01F0DEF9B14A0E9037
:1096C0000F910E9C0F9D94460F9B634415931D00B4
:1096D000109B002B61D1069807990022AA4B02F03B
:1096E00063FB2200159B0690079101F0B1F9002859
:1096F00000D0A8E2A5480F99844661440B00069863
:109700000799220001F090F9002800D095E2129B01
:10971000139C06930794199B002B00DA5CE10E2F33
:1097200000DD59E1934BFA009B185C681B680493B9
:109730000594219B002B00DBD8E0099B002B00DD6A
:10974000D4E000D07DE20498059900228E4B02F00F
:10975000B9F8069A079B01F085F9099B04931E004E
:10976000002800D04FE2089B089A5D1C3123013786
:1097700013704BE234420AD00E9B854A01330E939C
:10978000EB009B181A685B6802F09CF833006410C9
:1097900001355FE73E00099B84E7109B0D995A1E37
:1097A000744BD2009B181A685B68002949D00020CE
:1097B000784901F07DFC2B00220002F0F5FA089BAD
:1097C0000E900F9115930698079902F051FE040030
:1097D00002F084FE02000B000698079902F0E4FAFA
:1097E000159B30345D1C1C700E9A0F9B06900791E0
:1097F00001F01AF900286CD1069A079B00205E49F7
:1098000002F0D2FA0E9A0F9B01F00EF9002800D058
:10981000C3E0089B109AEB1A9A4200DC77E70E9897
:109820000F990022554B02F04DF800220E900F9137
:1098300006980799514B02F045F815950690079147
:10984000C1E72000290002F03DF8089C109A23008F
:1098500094460E900F91634415930698079902F071
:1098600007FE050002F03AFE0B0002000698079979
:1098700002F09AFA3035159B257001340690079155
:10988000A3422AD10E980F99089A109B94466344DC
:1098900000221D003F4B01F0EFF802000B0006987C
:1098A000079901F0D5F8002800D076E00E9A0F9BBA
:1098B0000020384902F078FA02000B000698079958
:1098C00001F0B2F8002800D121E76B1E1A78302A87
:1098D00001D037003FE01D00F7E706980799002206
:1098E000264B01F0EFFF06900791B6E7089E049A19
:1098F000059B0698079901F0DBFB02F0B9FD040017
:1099000002F0ECFD049A059B01F0DCFF02000B0065
:109910000698079902F048FA230030333370099A09
:10992000089B751CEB1A9A4248D102000B0001F00B
:10993000A3F8049A059B0690079101F089F8002886
:109940002AD1049A059B0698079901F067F8002828
:1099500001D0E30720D40399029800F0D4FC00233F
:109960002B70229B01371F60249B002B00D1E6E463
:109970001D60E4E460E00D100000F03F00002440B2
:1099800000001C400000C0FC000014400000C07C2F
:1099900038E00D100000E03F3E006B1E1A78392AB7
:1099A00006D1089A9A4207D130231370130001366A
:1099B0001A7801321A708CE71D00EEE70022A44BE2
:1099C00001F080FF00220023069007912E0001F095
:1099D00025F800288BD0BEE70D9A002A00D1DAE0E6
:1099E000209A012A00DDBDE0169A002A00D1B5E0D8
:1099F000984A9B18049D0A9C0A9A0121D2180A923F
:109A00000B9A0298D3180B9300F01DFD0600002C52
:109A10000EDD0B9B002B0BDD0B9A2300944200DD27
:109A200013000A9AE41AD21A0A920B9AD31A0B93C9
:109A3000049B002B1FD00D9B002B00D1AFE0002D0D
:109A400011D031002A00029800F096FD039A01001F
:109A50000600029800F000FD03991090029800F0B3
:109A600052FC109B0393049B5A1B04D00399029849
:109A700000F082FD03900121029800F0E4FC119BAC
:109A80000490002B00D1E3E11A000100029800F0DD
:109A900073FD209B0490012B00DD82E00025069BD6
:109AA000AB420ED1079B1B03AB420AD1179B079A0F
:109AB000134206D00A9B013501330A930B9B0133F5
:109AC0000B93119B0120002B6CD10B9B18181F23AB
:109AD00018407ED001331B1A042B70DD1C23181A8A
:109AE0000A9B24181B180A930B9B1B180B930A9BA9
:109AF000002B05DD1A000399029800F08FFD0390FA
:109B00000B9B002B05DD1A000499029800F086FDDE
:109B10000490149B002B5ED00499039800F0D0FDB4
:109B2000002858DA00230A220399029800F004FC66
:109B30000D9B013F0390002B00D190E100233100E9
:109B40000A22029800F0F8FB0C9B0600002B00DDB7
:109B500088E0209B022B00DC84E044E03623189A46
:109B60009B1A47E7099B5D1E049BAB4208DB5D1B0C
:109B7000099B002B0CDA0A9B099A9C1A00233BE7ED
:109B8000049B0495EA1A119B00259B181193EFE79B
:109B90000A9C099B30E7049D0A9C0D9E37E7049AB6
:109BA00064E70025049B049A1B69109303339B0010
:109BB000D318586800F0FEFB2023181A85E7042B01
:109BC00095D00A9A1C33D2180A920B9AE418D3182B
:109BD0008CE70300F5E7099B002B3DDC209B022B63
:109BE0003ADD099B0C930C9B002B0CD104990522A8
:109BF000029800F0A1FB04900100039800F060FDC2
:109C0000002800DDAFE5219B089DDF430023099379
:109C10000499029800F077FB002E00D19BE6099B87
:109C2000002B05D0B34203D01900029800F06BFB63
:109C30003100029800F067FB8DE6109B04931E0034
:109C4000E1E70023FAE7109B370004931E008AE542
:109C500000002440330400000D9B002B00D1B2E033
:109C6000099B0C93002C05DD31002200029800F0C6
:109C7000D5FC06003000002D11D07168029800F06C
:109C80000AFB3100040033690C319A1C92000C303D
:109C9000FEF73FFA01222100029800F0BFFC09966E
:109CA0000600089B0A9304990398FFF77DFA099927
:109CB0000D900400039800F003FD32001090049909
:109CC000029800F017FD01230B93C36830340500A0
:109CD000002B04D10100039800F0F2FC0B90290046
:109CE000029800F010FB0B9B209A13430ED1069AAA
:109CF000013313420AD1392C26D0109B002B01DDF1
:109D00000D9C31340A9B5D1C1C7081E7109B002B5D
:109D100007DB1D00209B1D4322D10123069A13421D
:109D20001ED10B9B002BEDDD03990122029800F060
:109D300075FC0499039000F0C3FC002802DCE1D11B
:109D4000E307DFD5392CDBD10A9B0A9A5D1C392346
:109D500013706B1E1A78392A67D001321A7057E7D0
:109D60000A9B5D1C0B9B002B04DD392CECD00134CD
:109D70000A9BC9E70A9B0C9A1C70089BEB1A93423A
:109D80003ED000230A220399029800F0D5FA099BDD
:109D90000390B34209D100230A220999029800F0E6
:109DA000CBFA099006000A957DE7099900230A225B
:109DB000029800F0C1FA002309900A2231000298AB
:109DC00000F0BAFAEEE7099B0C93089B06930499FE
:109DD0000398FFF7E9F9069B30305D1C18700C9A68
:109DE000089B0400EB1A9A4208DD00230A2203991B
:109DF000029800F0A1FA06950390E8E70023099382
:109E000003990122029800F009FC0499039000F0E4
:109E100057FC00289DDC01D1E3079AD46B1E1A7809
:109E2000302A00D0F4E61D00F8E7089A9A4203D1E0
:109E3000312301371370EBE61D008AE70B4B249AA0
:109E400008930B4B002A01D0FFF777FAFFF777FA58
:109E5000209B012B00DC21E6119D012035E60C9BA7
:109E6000002BB2DC209B022BAFDDBCE6C4DF0D1063
:109E7000CCDF0D10F7B58A8905000C00130760D4FC
:109E80004B68002B04DC0B6C002B01DC0020FEBDBA
:109E9000E76A002FFAD000232E682B6080235B0135
:109EA000216A1A4034D0606DA3895B0706D56368C8
:109EB000C01A636B002B01D0236CC01A0200216A08
:109EC00000232800E76AB847A189431C06D12B6804
:109ED0001D2B30D82B4ADA40D3072CD500236360E2
:109EE00023692360CB0405D5431C02D12B68002BCA
:109EF00000D16065616B2E600029C7D02300443318
:109F0000994202D02800FEF715F900206063BEE7F1
:109F100001232800B847431CC6D12B68002BC3D0AF
:109F20001D2B01D0162B01D12E60AFE74023A28953
:109F30001343A381ABE740230B430120A38140429D
:109F4000A5E70F69002FA1D00B680F60DB1B019301
:109F50000023920700D14B69A360019B002B00DC1A
:109F600094E7019B3A00216A2800A66AB0470028BE
:109F700003DC4023A2891343DFE7019B3F181B1A30
:109F80000193EAE7010040200B6970B505000C0061
:109F9000002B01D1002070BD002804D08369002B64
:109FA00001D100F05FF80B4B9C4209D16C680C2288
:109FB000A35E002BEED021002800FFF75BFFEAE74D
:109FC000054B9C4201D1AC68F1E7044B9C42EED1B9
:109FD000EC68ECE7F4DF0D1014E00D10D4DF0D1089
:109FE000002310B5040003604360836081814366F1
:109FF000C281036143618361190008225C30FEF76E
:10A0000091F8054B24626362044BA362044BE36244
:10A01000044B236310BDC04681A80D10A9A80D10E4
:10A02000E1A80D100DA90D1010B5024900F08CF833
:10A0300010BDC046899F0D1070B568254A1E554356
:10A040000E0029007431FEF7BFF8041E08D000216D
:10A050002A00016046600C30A0606832FEF762F8AA
:10A06000200070BD836913B50400002B28D18364E0
:10A07000C3640365134B144A1B68826201939842C0
:10A0800001D101238361200000F020F860602000EE
:10A0900000F01CF8A060200000F018F80022E0603A
:10A0A00004216068FFF79CFF01220921A068FFF7E7
:10A0B00097FF02221221E068FFF792FF0123A361BC
:10A0C00013BDC04670DE0D1029A00D10F8B51C4B55
:10A0D00007001E68B369002B02D13000FFF7C2FFF2
:10A0E0004836B4687368013B04D53368002B07D049
:10A0F0003668F6E70C22A55E002D0DD06834F2E735
:10A1000004213800FFF798FF30600028F0D10C23BD
:10A1100004003B602000F8BD20000A4B6566256006
:10A120006560A560E36025616561A561082229007D
:10A130005C30FDF7F7FF6563A563A564E564E9E7B7
:10A1400070DE0D100100FFFFF7B5040007000026C8
:10A1500001914834002C01D13000FEBD6368A56830
:10A160000093009B013B009301D52468F2E7AB8983
:10A17000012B08D90E22AB5E013304D02900380030
:10A18000019B984706436835EBE70000034B1B68CB
:10A19000186A002800D10248F030704784A10208F4
:10A1A000E8A1020870B50E001D000E23C95E96B02E
:10A1B0001400002907DA00232B60B3891B0611D491
:10A1C0008023DB000FE06A4600F0CCFB0028F2DBC6
:10A1D000F022019B12021340054A9B185A42534138
:10A1E0002B60EDE740230020236016B070BDC04611
:10A1F00000E0FFFFF7B502268B8905000C00334213
:10A2000006D0230047332360236101236361F7BD38
:10A2100001AB6A46FFF7C6FF009907002800FDF76B
:10A22000D3FF002808D10C22A35E9A05EFD40322A5
:10A2300093431E43A681E4E70F4BAB628023A289C0
:10A2400020601343A381009B20616361019B002B6D
:10A250000DD00E23E15E280000F096FB002806D00A
:10A260000322A38993431A0001231343A381A089E6
:10A270003843A081CBE7C04629A00D10C9B282188F
:10A28000904201D10020704703788B42FBD001300F
:10A29000F6E77047704770B5466A04000D00002E5F
:10A2A00007D11020FDF700FF6062466086600660FF
:10A2B000C660666AF368002B13D0636AAA00DB6885
:10A2C0009B181868002818D101210E00AE40721D9D
:10A2D0009200200000F0C6FA00280CD0456086608D
:10A2E0000DE021220421200000F0BCFA636AF06036
:10A2F000DB68002BE1D1002070BD02681A600023EA
:10A300000361C360F8E770B5446A06000D00002CD5
:10A3100007D11020FDF7C8FE7062446084600460BD
:10A32000C460002D07D0736A6A68DB6892009B18CE
:10A330001A682A601D6070BDF7B51E0014239C4684
:10A3400007000C0000200D698C4463461B68013037
:10A3500099B263461B6851431B0C534389190E0C79
:10A360009B1989B21E0C1B045B18614608C18C4600
:10A370008542EADC002E1BD0A368AB4212DC636886
:10A380003800591CFFF787FF2100236901909A1CB0
:10A3900092000C310C30FDF7BCFE21003800FFF7B5
:10A3A000B2FF019C2B1D9B00E31801355E60256107
:10A3B0002000FEBD0300020C0020824201D11B04DC
:10A3C00010301A0E01D108301B021A0F01D10430CF
:10A3D0001B019A0F01D102309B00002B03DB0130DF
:10A3E0005B0000D4202070470722036810B50100ED
:10A3F0001A400DD001240020234205D1023003422F
:10A4000003D0E34020000B6010BD9B080B60FBE70E
:10A410009CB21000002C01D110201B0CDAB2002AD3
:10A4200001D108301B0A1A0701D104301B099A0711
:10A4300001D102309B08DA07E8D45B0801D0013073
:10A44000E4E72020E0E710B50C000121FFF723FF2F
:10A4500001234461036110BDF0B50B69140012695A
:10A4600089B00D00934201DA25000C002F6926699E
:10A470006968BB190293AB68BA19934200DA0131DB
:10A48000FFF709FF0200BB1914329B00D3189C464A
:10A4900000211300049063451DD31435BF00EB1950
:10A4A0001434B6000593A319039501940793079BF1
:10A4B0000199994211D3029B002B06DD04235B42D4
:10A4C0009C4463461B68002B51D0049B029A1800E1
:10A4D0001A6109B0F0BD02C3DDE7019B1B6898B2A9
:10A4E00000281CD015000026039F02CF2C688BB2D9
:10A4F0004343090C4143A4B21B199B190E00296860
:10A500000695090C71181E0C89190E0C9BB20904D2
:10A510000B4308C5059BBB42E7D8069B5E60019BC9
:10A520001B681D0C1ED0100000271368039E3168A5
:10A53000046889B26943240C0919C9190F049BB234
:10A540003B43036080CE43683F0C6F439BB2FB18D4
:10A55000090C5B18059906901F0C0430B142E6D82F
:10A5600006994B60019B0432043301939FE7029BE1
:10A57000013B02939FE700000323F7B5134005005A
:10A580000E001400002B08D02249013B9A005258BB
:10A5900000233100FFF7D0FE0600A310019336D050
:10A5A0006C6A002C07D11020FDF77EFD68624460C4
:10A5B00084600460C4606F6ABC68002C07D11649CF
:10A5C0002800FFF740FF00230400B8600360012269
:10A5D000019B13420AD0310022002800FFF73CFF04
:10A5E000070031002800FFF78EFE3E00019B5B1044
:10A5F00001930CD02068002807D1220021002800F8
:10A60000FFF72AFF0023206003600400DFE730002B
:10A61000FEBDC04628E10D1071020000F0B50D002E
:10A6200017002B69541185B0E3180193013300938F
:10A630004968AB680290009A934235DB0298FFF7B5
:10A640002AFE00230200060019001432A3422EDB6A
:10A65000E343DB171C402B00A40014192A691433B0
:10A6600092009A1894461F22174024D00132D21B20
:10A670000392002219682000B9400A4304C404CBA5
:10A680000399CA409C45F5D84260002A02D0019B3C
:10A6900002330093009B0298013B33612900FFF7CE
:10A6A00032FE300005B0F0BD01315B00C3E7980019
:10A6B00011500133CAE704CB04C49C45FBD8E9E739
:10A6C0000A69036930B59B1A0DD192001430143118
:10A6D00084188918043C043925680A68954204D016
:10A6E0000123954204D3180030BDA042F2D3FAE70B
:10A6F0005B42F8E7F0B50D0085B0070011002800B7
:10A700001400FFF7DDFF061E08D101003800FFF737
:10A71000C2FD01234661036105B0F0BD0123019331
:10A72000002804DB23002C001D0000230193616836
:10A730003800FFF7B0FD2F000022019B2669C3609F
:10A740001434B300E31802932B6914379B00FB18F1
:10A75000039303009446143320CC04CF0192AAB291
:10A7600094446A46614692882D0C8A1A0199090C14
:10A77000691A151449190D1492B209040A431A6092
:10A78000039AAC460433BA42E6D802991A008C42C6
:10A7900005D3043A1368002B0ED00661BCE704CC45
:10A7A00091B261440D14120C5219151489B212049D
:10A7B0000A43AC4604C3E8E7013EEAE7F7B51D00EB
:10A7C00001211400089FFFF766FD2B036D000600B2
:10A7D0001B0B6D0D24D10193002C27D068460094EB
:10A7E000FFF702FE009C00281ED0019B20211A00CA
:10A7F000091A8A40C340224372610193019CB461EB
:10A80000631E9C4101343461002D18D0124BED18A9
:10A8100035232D183D60181A099B18603000FEBDC5
:10A82000802252031343D6E77461E7E701A8FFF7DC
:10A83000DBFD0124019B346173612030E4E7074BA9
:10A84000C018074B3860E3189B00F3185869FFF7EE
:10A85000B1FD6401201ADFE7CDFBFFFFCEFBFFFF58
:10A86000FFFFFF3F4A4370B511001400FDF7ACFC39
:10A87000051E03D022000021FDF754FC280070BD06
:10A8800070B50C000E25495F00F0A4F8002803DB2A
:10A89000636D1B18636570BDA389024A1340A381D1
:10A8A000F9E7C046FFEFFFFFF8B51F008B890500F1
:10A8B0000C001600DB0505D50E23C95E002202231D
:10A8C00000F074F8A389054A28001340A3813200E0
:10A8D0000E23E15E3B0000F01FF8F8BDFFEFFFFF25
:10A8E00070B50C000E25495F00F060F8A389421C8A
:10A8F00003D1054A1340A38170BD80225201134346
:10A90000A3816065F8E7C046FFEFFFFF10B50E2397
:10A91000C95E00F015F810BD70B505000800110003
:10A920000022064C22601A00F7F7EAF9431C03D113
:10A930002368002B00D02B6070BDC0463CB00208DD
:10A94000002370B5064C05000800236001F032FEBC
:10A95000431C03D12368002B00D02B6070BDC04680
:10A960003CB00208002370B5064C05000800110039
:10A97000236001F027FE431C03D12368002B00D085
:10A980002B6070BD3CB00208002370B5064C05007A
:10A990000800236001F01EFE431C03D12368002B36
:10A9A00000D02B6070BDC0463CB0020870B50500F9
:10A9B000080011000022064C22601A0001F012FE6D
:10A9C000431C03D12368002B00D02B6070BDC04610
:10A9D0003CB0020870B50500080011000022064CCA
:10A9E00022601A00F7F79EF9431C03D12368002B5D
:10A9F00000D02B6070BDC0463CB002088446101CDD
:10AA000062468C46191C634600E0C0461FB500F044
:10AA1000F1FE002801D40021C8421FBD10B500F08E
:10AA200049FE4042013010BD10B500F0E3FE0028A1
:10AA300001DB002010BD012010BDC04610B500F0A4
:10AA4000D9FE002801DD002010BD012010BDC04648
:10AA500010B500F06BFE002801DC002010BD0120C5
:10AA600010BDC04610B500F061FE002801DA0020DC
:10AA700010BD012010BDC046F0B54F464646D64633
:10AA80000C000903C0B5490A470F5E0039431F0394
:10AA9000DB0F9C4665007B0A570F1F436D0DE40FCB
:10AAA000760DA146C000B846D200AB1B64457BD0F2
:10AAB000002B5FDD002E00D0A4E03E00164300D145
:10AAC00012E15E1E002E00D09EE1871A4346B84276
:10AAD00080410125C91A4042091A0B0200D431E114
:10AAE00049024E0A002E00D16EE13000FDF744FA13
:10AAF0000300083B1F2B00DD61E120223900D21A40
:10AB00009E40D1409F400E439D4200DD51E15D1BC0
:10AB10006B1C1F2B00DD7CE12021C91A3D00300099
:10AB20008F408840DD40791E8F4131000722284345
:10AB3000D940002507433A40002A09D00F233B4063
:10AB4000042B05D03B1DBB42BF417F42C9191F00EA
:10AB50000B0200D426E26A1CC64B55056D0D9A42C5
:10AB600000D106E1C44AFF080A40530752023B43A2
:10AB7000120B8EE0002B00D0B8E06B1C5B055B0D68
:10AB8000012B00DC30E1871A4346B842B641CB1AAC
:10AB900076429E1B330200D54CE13B003343A1D1EA
:10ABA00000220024002570E0002B00DCE5E0002EF0
:10ABB00000D183E0AF4EB54260D0802636043743E3
:10ABC000B846382B00DC3EE1434613431F007A1E93
:10ABD00097413F1887428041404209180B0200D438
:10ABE000B0E0A44B01359D4200D1C3E0A24A7B08EE
:10ABF0000A4001210F401F435108D30707221F437A
:10AC00003A4099E79B4EB54238D080263604374308
:10AC1000B846382B00DDDCE01F2B00DC30E11E00E5
:10AC20004746203EF740BC46202B04D04026F31A6E
:10AC300046469E403243170063467A1E97411F43A3
:10AC4000CCE0002B00D104E24346134300D159E18C
:10AC50004B07C00818438023C9081B03194208D0BA
:10AC60004546ED081D4204D14346D0085907084324
:10AC70002900420FC9007F4D1143C0004B07CA088D
:10AC80007C49C00803438D4268D012036D05120B46
:10AC90006D0D002112031800130B0A0D12051A4343
:10ACA000764B2D0513402B435B00E4075B082343E1
:10ACB00019001CBC90469946A246F0BD3E001643C2
:10ACC00012D05E1E002E00D000E18718874280411E
:10ACD00041444042091801250B0233D5022585E77E
:10ACE00064463300414610001D00C7E7002D00D028
:10ACF000DAE00C000443F3D05C1C00D19FE15D4C12
:10AD0000A64200D12FE1DB43382B00DD66E11F2B8B
:10AD100000DD83E120240500E41A0F00DD40D94066
:10AD2000A0404346A7405B1A441EA04198462F43CB
:10AD30003843171ABA42924143465242991A64461E
:10AD40003500CAE607223A40002A00D0F6E64B0753
:10AD5000CA084849FF083B438D4296D11900114368
:10AD600000D19EE1802109030A431203120B414DD9
:10AD70008FE71500002200238BE7002B00D0C7E0EF
:10AD80006B1C5F057F0D012F00DCF1E0394DAB42FC
:10AD900000D1B9E085180A00854289414244494200
:10ADA00051180722CF076D082F4349083A401D006C
:10ADB000C2E607223049ED1A31403A40BCE63E0077
:10ADC0002838864000279FE63800FDF7D5F8203068
:10ADD0008EE6434613431F007A1E9741C71BB842B5
:10ADE00080414042091A78E60E003B0006431343B7
:10ADF000002D61D1002E00D0F4E0002B00D11BE12A
:10AE000064463900100039E71A4FBB427AD033004C
:10AE1000FFE630001F3DE840202B03D04021CB1A35
:10AE20009E4037437B1E9F41072207433A40002143
:10AE3000002589E7171A4346BA42B641591A7642A5
:10AE40008E1B64464EE61F2B00DDADE020264746F4
:10AE5000F61AB740B9461700B246DF404E463E43A9
:10AE600037005646B240561EB24117434246DA40BA
:10AE70008918AEE6FF070000FFFF7FFFFFFF0F808E
:10AE800020264746F61AB740B9461700B246DF40BB
:10AE90004E463E4337005646B240561EB241174317
:10AEA0004246DA40891A99E77F4CA6425BD080245B
:10AEB00024045B42214327E7002E0CD1002B00D154
:10AEC000CBE0644639001000774DD7E6764FBB42A1
:10AED00018D0330075E6002B14D04B07C008184378
:10AEE0008023C9081B03194207D0FC081C4204D167
:10AEF0007907D0080843E14621004C46420FC900BB
:10AF00001143C000684DB9E61D0000220023C0E6D1
:10AF1000002D5BD10D00054300D1E2E65D1C00D1A0
:10AF2000B0E0614DAE421FD0DB43382B71DC1F2BEC
:10AF300000DD96E020250F00ED1AAF40B94607006E
:10AF4000AA46DF404D463D432F005546A840D94014
:10AF5000451EA84188440743BF1897429241514279
:10AF6000414435003AE6644635004146100085E626
:10AF70000B000343002D00D063E6002BF5D04346C1
:10AF8000134300D17AE68718874280410722414463
:10AF9000404209183A400B0200D4D5E6434B013534
:10AFA0001940C9E5380069E61E004746203EF740D3
:10AFB000BC46202B04D04026F31A46469E4032431E
:10AFC000170063467A1E97411F4302E6364DAE4294
:10AFD000CAD080252D045B422943A6E70843411EC1
:10AFE0008841A6E6002B00D148E6871A4346B842BE
:10AFF000B641CB1A76429E1B33024BD5171A4346F5
:10B00000BA429241591A5242891A072264463A407A
:10B0100092E501430F00791E8F419DE71C000F0050
:10B02000203CE740202B03D04024E31A99400843FA
:10B03000411E884138437CE60022002425E6171A89
:10B040004346BA429241591A5242891A644635001F
:10B0500043E541461000144D10E6802200241203FF
:10B0600080E61D000F00203DEF40BC46202B03D0A2
:10B070004025EB1A9940084307006346781E874134
:10B080001F4369E7871897429B4141445B42C918B7
:10B090003500A3E53B003343CED0072231003A40D0
:10B0A00052E600231A00F4E5FF070000FFFF7FFFD0
:10B0B000F0B55746DE464E464546E0B583460700A6
:10B0C0000E03480085B092461C00360B400DCD0F94
:10B0D000002800D19DE0954B984239D08023F6009E
:10B0E0001B041E43924A7B0F334399469446030048
:10B0F0006344009300230026FF00029323031B0BED
:10B1000098466300E40F52465B0D019400D1B3E012
:10B1100086498B4200D19EE04246D1008022120433
:10B120000A435146490F11438B46814952468C468A
:10B1300000996344CB1A0021D20000932B00634096
:10B140009A460F2E00D905E17A4BB6009B599F46CF
:10B150005B463343994600D0B8E002230826002717
:10B1600000900293CAE7CB463A0002990195019BF1
:10B170009A46022927D0032900D180E2012944D030
:10B180006D49009B8C4663441C00002C38DD53073E
:10B1900000D013E2D2085B46DB0109D55946674B64
:10B1A00019408B468021C9008C46009B63441C00DB
:10B1B000634B9C4207DC5B4664055F075B021743F9
:10B1C0001B0B620D02E000230027584A00211B03DD
:10B1D0001C0B0B0D1B05234314055A4A3800134062
:10B1E0001C4353466400DB0764081C43210005B080
:10B1F0003CBC90469946A246AB46F0BD0122524265
:10B2000001231B1B382B00DCADE1002200230027AB
:10B21000DCE75B46334399465ED0002E00D18AE1DD
:10B220003000FCF7A9FE03000B3B1C2B00DD7BE18B
:10B230001D22D31A5A460100DA4008398E40130005
:10B240005F46334399468F403F4B00261B1A0093BD
:10B250000023029352E7414653460B433B499B462A
:10B260008C46009B634400935B46002B3BD102233A
:10B2700000221E43022161E7434613439B4637D019
:10B280004346002B00D162E14046FCF775FE030007
:10B290000B3B1C2B00DD53E102004146083A914074
:10B2A00088461D21CB1A5146D9400B0041460B431D
:10B2B0009B46534693401A00009B25499C46604498
:10B2C00003008C4663440093002137E70323B14613
:10B2D00000900C26029311E700230093013304260B
:10B2E000002702930AE70323C3461E43032125E7F1
:10B2F00001331E430022012120E700239A468023C8
:10B3000000271B03094A61E7802349461B031942B2
:10B3100000D1E2E05946194200D0DEE00B431B03A6
:10B3200017001B0BA246014A50E7C046FF0700006A
:10B3300001FCFFFF34E10D10FF030000FFFFFFFEE3
:10B34000FE070000FFFF0F800DFCFFFF01F8FFFF6D
:10B35000F3030000D94500D9CBE000D1C6E03C00A2
:10B3600048460027009B013B00935B46160E1B02DC
:10B370001E431302984633041B0C9946310C01916D
:10B38000FCF7FEFB4A4642430B04210C050019431F
:10B390008A4207D98919013D8E4203D88A4201D9D0
:10B3A000851E8919881A0199FCF7EAFB09048C4665
:10B3B0004A46210464464243090C030021438A4261
:10B3C00004D98919013B8E4200D8F1E02D041D43B8
:10B3D000AB464346891A4246280C12041D0C5B46B4
:10B3E000140C22001B041B0C5A4303946B4344436C
:10B3F000029568431B19150CEB189C4203D9802455
:10B400006402A44660441C0C15041B042D0C201877
:10B410005D19814277D373D00C1AA24A7D1BAF42CB
:10B42000BF419446009B7F426344E01B1C00864260
:10B4300000D1DBE00199FCF7A3FB4A4642430B0431
:10B44000290C070019438A4207D98919013F8E4206
:10B4500003D88A4201D9871E8919881A0199FCF7F5
:10B460008FFB09044A46894629044D464243090C8C
:10B47000030029438A4207D98919013B8E4203D828
:10B480008A4201D9831E89193F04891A3A00039F11
:10B490001A43380013041B0C584381460298150CBC
:10B4A0006F43434345434846000C8446DB196344DD
:10B4B0009F4203D9802040028446654448461F0CC1
:10B4C00000041B04000C7D191818A94200D284E066
:10B4D00000D17FE001231A4357E680234A461B032D
:10B4E00013431B031B0BAA466F4A6FE6BA4200D9EF
:10B4F00035E74B46DC0758087B081C43FF0734E759
:10B500000024AF4289D247444745A4415B46644288
:10B51000A4196418013BA6421ED2A0426DD800D1E6
:10B52000B6E0241A9B4678E703005A46283B9A4027
:10B530000027914688E65846FCF71EFD203072E64B
:10B5400003005246283B9A4093460022B4E65046F8
:10B55000FCF712FD20309AE6A642E2D1B845DCD9CC
:10B56000341A9B4659E71F2B65DC504C0099A446C2
:10B570005C46614408008C4011008240D940501E56
:10B5800082410C4314435A46DA401300620709D043
:10B590000F222240042A05D02200141D9442894122
:10B5A00049425B181A0262D50122002300270DE6EA
:10B5B0008A4200D80AE7831E891907E70F23134040
:10B5C000042B00D1E6E5171D9742924153429B445C
:10B5D000FA08E0E5002800D1D7E57118531EB14202
:10B5E00027D3A94215D358D01A0073E7002B00DCEB
:10B5F00004E6012300229B44CDE50223474447454E
:10B6000089415B429C46494289190C19E344241A3A
:10B6100003E743465F0047459B41B8465B429E199E
:10B62000023A8919A94200D054E7404500D051E7B9
:10B63000ABE51A00F6E71F215F4649420C1BE740C5
:10B64000202B07D01A49009B8C46634418005B46A8
:10B6500083401A43501E82413A4307270023174074
:10B6600009D00F21002311401400042995D1220094
:10B670005F075B021B0BD20817430022A6E580235D
:10B6800059461B030B431B0317001B0B064A9DE582
:10B69000BD42B2D89B460024BFE68045B9D31A000C
:10B6A000C3E7C046FF030000FF0700001E040000C0
:10B6B0003E040000F0B54F464646D6468446C0B527
:10B6C0008046194E18030F034D00000B5C008246A4
:10B6D0003F0B6D0DC90F9146640DDB0F0120B54284
:10B6E0000AD0B44203D0A54201D157450CD01CBCAE
:10B6F00090469946A246F0BD66463E43F7D1AC421D
:10B70000F5D154461443F2D10120C845EFD19942F6
:10B7100007D0002DEBD163461F433800471EB841C8
:10B72000E5E70020E3E7C046FF070000F0B54F461D
:10B730004646D6464D00C0B50E03C90F8A462C4971
:10B740001F035C008046360B6D0D91463F0B640D68
:10B75000DB0F8D421ED08C4216D0002D1ED13043FF
:10B760008446002C01D13A4323D06246002A1AD0E5
:10B770009A4529D0514602200139084001381CBCA5
:10B7800090469946A246F0BD39001143E5D002200B
:10B790004042F4E73043FAD1AC420FD0002C0FD135
:10B7A0003A43E7D00CE00122013B934318000130FB
:10B7B000E5E763460020002BE1D0DBE73A43E6D122
:10B7C0009A45D7D1A542D5DCA54205DBBE42D1D8EA
:10B7D00008D00020BE42D2D25046012301389843FF
:10B7E0000130CCE7C845C5D80020C845F4D3C6E72A
:10B7F000FF070000F0B54F464646D6464D00C0B59F
:10B800000E03C90F8A462E491F035C008046360B83
:10B810006D0D91463F0B640DDB0F8D4218D08C42AD
:10B8200011D0002D18D130438446002C1ED13A434C
:10B830001CD163460020002B30D051460220013934
:10B84000084001382AE039001143EAD0022025E0FF
:10B850003043FBD1AC4226D0002C26D13A4324D130
:10B860005146022001390840013817E06246002A9B
:10B870000FD09A45E1D1A54205DBBE42DDD819D0F3
:10B880000020BE420AD250460123013898430130BD
:10B8900004E00122013B9343180001301CBC904698
:10B8A0009946A246F0BD3A43D0D19A45C5D1A542AA
:10B8B000C3DCE0E7C845C0D80020C845E3D3EDE7C6
:10B8C000FF070000F0B55746DE464E464546E0B558
:10B8D000834606000F03480087B092461D003F0BC9
:10B8E000400DCC0F002800D16FE0DE4B984238D0DD
:10B8F0008023FF001B041F43730F3B430193DA4B6C
:10B900000027994600239B46F60081442B036900DB
:10B910001B0B52469846490DED0F002900D185E0DA
:10B92000D04B994200D173E04346DA0080231B04D8
:10B9300013435246CC48520F8446134352460020CC
:10B940006144D20089442100694000918C46012164
:10B9500049448A460F2F00D990E0C449BF00CF590F
:10B96000BF465B463B43019300D06AE102230827B0
:10B97000002681469B46C9E732005846019B614636
:10B980000091022800D175E0032800D1FEE10128D2
:10B9900000D02CE100230027002600253F032A0DBC
:10B9A0003F0BB34812053A4302401B051343009A6C
:10B9B0005B00D1075B080B433000190007B03CBCAB
:10B9C00090469946A246AB46F0BD5B463B43019389
:10B9D00000D12FE1002F00D1A5E13800FCF7CCFA0F
:10B9E00003000B3B1C2B00DD96E11D22D31A5A46A7
:10B9F0000100DA405E4608398F4013008E403B4319
:10BA000001939C4B00271B1A994600239B467DE718
:10BA1000414653460B4393498C46E144002B00D0EA
:10BA20001AE102220220174300228CE7134300D1BF
:10BA30000DE14346002B00D181E14046FCF79CFA22
:10BA400002000B3A1C2A00DD72E10100434608396E
:10BA50008B4098461D239A1A5346D3401A004346FA
:10BA6000134352468A404946081A8249894681440E
:10BA7000002068E77B4B002700268EE7140C120499
:10BA8000120C1100370C3604350C794328008C4613
:10BA90002E0060436044834656432100300C8046AC
:10BAA0005846794340440291844506D9884680210E
:10BAB00049028C46E044414602913604010C360CA2
:10BAC00000048B4681191E0C1B041B0C03911900EA
:10BAD00079438C46280075436544A8465843050CB5
:10BAE00045447743A94203D9802149028C466744E3
:10BAF000290C8C4639000004000C2D042D186144DB
:10BB0000AB4405915946049101990F043F0C080C70
:10BB1000390051434243904602008C46090C8B4643
:10BB200062437C4344445C44A04503D980214902DC
:10BB300088464244210C884661460904090C8C461B
:10BB400039005943434370437E430F0CF6182404D5
:10BB5000BE19644442448C46B34203D980235B023D
:10BB600098464044029B61469846049B37044344F0
:10BB70009B46AB45AD416B420D0405992D0C8C469F
:10BB80007F196744FD18A8465D462D19A542A441BA
:10BB900093466442A446C344DC448F42BF41984567
:10BBA0009B4193459241A445A4415B427F421F4380
:10BBB000360C52426442BF192243BF1862463818FD
:10BBC0004302D20D039913436A020A43501E824175
:10BBD0006146ED0D2A434E023243D90100D4B3E051
:10BBE0000126500832400243DE0732435B08224CF4
:10BBF0005444002C62DD510709D00F201040042866
:10BC000005D0101D9042924152429B180200D9016A
:10BC100004D580241948E400034054441848844261
:10BC200000DD27E75E075B02D2081F0B63051643A2
:10BC30005B0DB2E6002399460133042700269B469C
:10BC400064E60323019781460C279B465EE60122AA
:10BC500001201743002276E6032303201F434346B7
:10BC600071E6C046FF07000001FCFFFF74E10D1004
:10BC7000FFFF0F800DFCFFFFFF030000FFFFFFFE33
:10BC8000FE0700000023802700933F030026434B5C
:10BC900083E6019B3200A446584670E6AC466EE649
:10BCA000802701993F0339422DD03B422BD11F43BE
:10BCB0003F033F0B00951600384B6EE601252D1B08
:10BCC000382D00DD66E61F2D40DC35481C00504451
:10BCD000160082408440EE40501E8241344314439B
:10BCE000EB40620709D00F222240042A05D022002F
:10BCF000141D9442804140421B181A023ED5012374
:10BD00000027002649E68027019B3F031F433F038E
:10BD10003F0B0094214B40E603005A46283B9A40D3
:10BD2000002601926DE65846FCF726F9203057E6CA
:10BD300003005246283B9A401300002293E65046E7
:10BD4000FCF71AF920307BE6CA4650E71F201E0098
:10BD50004042041BE640202D03D0124C5444A34023
:10BD60001A43501E8241324307260027164009D04D
:10BD70000F200023104014000428B9D122005E07D0
:10BD80005B021F0BD2081643002306E680273F0301
:10BD90001F433F033F0B1600004BFEE5FF0700006B
:10BDA0001E0400003E040000F8B557464E464546C6
:10BDB000DE460C000903E0B5490A460F5F00314337
:10BDC0001E03DB0F760A9B46530F3343C84E6500B4
:10BDD000C000E40FD2006D0DA24681467F0D9C4647
:10BDE0009046B74200D1B9E05B46012673409B46BE
:10BDF000EE1BA34500D183E0002E63DD002F00D0B1
:10BE0000B1E06346134300D123E1731E002B00D041
:10BE1000BAE1861A6346B04280410125C91A404200
:10BE2000091A0B0200D447E149024B0A98464346DF
:10BE3000002B00D189E14046FCF79EF80300083B47
:10BE40001F2B00DD7CE120223000D21A4146D04079
:10BE5000994002009E400A439D4200DD6AE15D1B5D
:10BE60006B1C1F2B00DD94E1202110003500C91A46
:10BE70008E40DA408840DD40711E8E41110007225D
:10BE80002843002506433240002A09D00F233340BF
:10BE9000042B05D0331DB342B641764289191E00EA
:10BEA0000B0200D43DE26A1C914B55056D0D9A4280
:10BEB00000D119E18F4AF6080A405707520237436A
:10BEC000120B9BE0002E00D0C5E06E1C7605760DAF
:10BED000012E00DC48E16746861ACB1BB042BF4109
:10BEE0007F42B8461F004346FF1A3B00B8461B027C
:10BEF00000D55FE137439AD100220024002579E084
:10BF0000002E00DCFAE0002F00D18DE0784B9D423E
:10BF100067D0802367461B041F43BC46382E00DCD5
:10BF200052E1634613435A1E93411E1886428041D4
:10BF3000404209180B0200D4BEE06D4B01359D4212
:10BF400000D1D2E06B4A73080A4001210E401E4323
:10BF50005108D30707221E43324095E71E001643BF
:10BF600000D045E740E7624B9D423AD080236746C8
:10BF70001B041F43BC46382E00DDEBE01F2E00DC07
:10BF80003AE133006746203BDF403B00202E05D0DE
:10BF90004027BF1B6646BE40324390464646721E4F
:10BFA00096413343DAE0002B00D114E26346134399
:10BFB00000D168E180234E07C008C9081B0306436F
:10BFC000194208D06046C008184204D163460100F7
:10BFD000D2085E071643F3009946C900720F444D1C
:10BFE00011434B46DE08424B4F073743CA089D4278
:10BFF00000D16EE012036D05120B6D0D00211203CE
:10C00000130B0A0D12051A433B4B2D0513402B430E
:10C010005B00E4075B082343380019003CBC9046F2
:10C020009946A246AB46F8BD6346134311D0731E32
:10C03000002B00D007E186188642804161444042CF
:10C04000091801250B0237D502257BE73E00614622
:10C0500091463500C5E75C46002D00D0E1E00B00BD
:10C060000343F3D0731C00D1ACE1214B9F4200D1BC
:10C070003AE1F343382B00DD6FE11F2B00DD8CE14B
:10C0800020250E00ED1AAE40B0460600AA46DE405E
:10C09000454635432E005546D940A8406346451EC7
:10C0A000A8415B1A9C463043161AB242924163463D
:10C0B0005242991A3D00B4E607223240002A00D0CD
:10C0C000E4E60B4BF6084F073743CA089D4200D001
:10C0D00090E73B00134300D1A6E180231B031A43E2
:10C0E0001203120B024D89E715000022002785E795
:10C0F000FF070000FFFF7FFFFFFF0F80002E00D033
:10C10000C7E06B1C5E05760D012E00DCF0E0C84D2B
:10C11000AB4200D1B9E085180A00854289416244EA
:10C12000494251180722CE076D082E434908324074
:10C130001D00A9E6BF49ED1A114007223240A3E6CF
:10C14000320028388240002686E63000FBF714FFD4
:10C15000203073E6634613435A1E9341C61AB04219
:10C1600080414042091A5CE60E00674606431743C9
:10C17000002D5ED1002E00D0F3E0002F00D11EE193
:10C180005C46614691462CE7A94FBE427BD01E001B
:10C19000F1E610001F3DE840202B03D04021CB1AD0
:10C1A0009A401643731E9E410722064332400021E7
:10C1B000002583E7161A6346B2428041591A40426D
:10C1C0000B1A98465C4632E61F2E00DDABE02027B6
:10C1D000BB1B9A4663465746BB40994613004F46E1
:10C1E000F3401F433B005746BA40571EBA41134322
:10C1F0006246F240891898E62027BB1B9A466346A0
:10C200005746BB40994613004F46F3401F433B003F
:10C210005746BA40571EBA4113436246F240891A44
:10C220009CE7834B9F425FD080252D0473422943B6
:10C2300020E7002E0CD1002F00D1D0E05C466146F3
:10C2400091467B4DCDE67A4FBE421CD01E0065E67E
:10C25000002F18D0C0084E0706438020C9080003ED
:10C26000014208D06346DC08044204D12100DA46CA
:10C27000D2085E071643F300994601245346C900CD
:10C28000720F11431C406A4DABE61D0000220027CF
:10C29000B4E6002D59D10B00034300D1D6E6731C40
:10C2A00000D1B2E0624B9F421ED0F343382B6FDCCB
:10C2B0001F2B00DD97E020250E00ED1AAE40B046A2
:10C2C0000600AA46DE40454635432E005546A840A6
:10C2D000D940451EA8418C440643B6189642924167
:10C2E000514261443D0025E63D006146914678E6B5
:10C2F0000B000343002D00D055E6002BF5D063461C
:10C30000134300D16DE68618864280416144404265
:10C31000091800220B0200D4D0E6464B0135194023
:10C32000B2E5B1465DE633006746203BDF403B00A7
:10C33000202E05D04027BF1B6646BE4032439046A4
:10C340004646721E96413343EFE5394B9F42CBD0B0
:10C3500080252D0473422943A8E70843411E8841E4
:10C36000A2E6002F00D13CE66346861ACF1AB042FF
:10C370009B415B42FB1A98461B024ED5161A634638
:10C38000B2429241591A5242891A5C4600227BE518
:10C3900001430E00711E8E419FE71D000E00203DDF
:10C3A000EE40B046202B04D04025EB1A99400843BC
:10C3B000814648464346411E8841184374E60022A0
:10C3C000002417E6161A6346B2429241591A5242A5
:10C3D000891A3D0025E561469146154D01E680220A
:10C3E0000024120379E61D000E00203DEE40B04609
:10C3F000202B04D04025EB1A9940084381464E4635
:10C400004346711E8E411E4367E7861896429B4144
:10C4100061445B42C9183D008CE547463743CED0A6
:10C4200007224146324049E600273A00E6E5C04689
:10C43000FF070000FFFF7FFF70B50C4E0D031C03CC
:10C4400049005B002D0B490D240B5B0DB14208D058
:10C45000064900208B4203D114432000441EA04112
:10C4600070BD05430120002DFAD1F1E7FF07000060
:10C4700030B5144D0A034B00120B5B0DC90F00249D
:10C48000AB4211DD104CA34210DC80246403224334
:10C490000E4CE41A1F2C0CDD0D48C31ADA401300B1
:10C4A0005C42002900D11C00200030BD094BCC1893
:10C4B000FAE7094DE040AC4663449A401300034359
:10C4C000EEE7C046FE0300001D0400003304000038
:10C4D00013040000FFFFFF7FEDFBFFFF70B5002896
:10C4E0002DD0C317C5185D40C40F2800FBF744FDCD
:10C4F000154B1B1A5B055B0D0A2815DD0B388540B3
:10C5000000222D032D0B002110002D030A0D2D0BF1
:10C5100012052A430D4D1B052A4013435B00E40717
:10C520005B082343190070BD0200290015329140B9
:10C530000A000B21081AC5402D032D0BE3E7002448
:10C54000002300250022DEE71E040000FFFF0F800D
:10C5500010B5041E25D0FBF70FFD144B1B1A5B050D
:10C560005B0D0A2812DD0B38844000222403240BC3
:10C570000021100024030A0D240B120522430C4C49
:10C580001B05224013435B00590810BD0200210027
:10C59000153291400A000B21081AC4402403240BD1
:10C5A000E6E7002300240022E2E7C0461E04000064
:10C5B000FFFF0F8058220120014B40421A60704754
:10C5C0003CB0020858220120014B40421A607047DB
:10C5D0003CB002085822024B00201A607047C04647
:10C5E0003CB0020858220120014B40421A607047BB
:10C5F0003CB00208044A1368002B00D1034B181802
:10C60000106018007047C046DCAD02080000020848
:10C61000F8B5C046F8BC08BC9E467047F8B5C046A1
:10C62000F8BC08BC9E46704701B40248844601BC71
:10C63000604700BFEFA3020801B40248844601BC72
:10C64000604700BF01A7020801B40248844601BC4C
:10C65000604700BF1DA5020801B40248844601BC22
:10C66000604700BF03A702080000000007000103A5
:10C6700000000100030300003F00010300000F0061
:10C68000C0102040030300004000010300000F0021
:10C6900000112040030300003F00010300000F00D1
:10C6A00040112040030300007F00010300000F0041
:10C6B00080112040000300000F00010300000F0064
:10C6C00040122040030300003F00010300000F0060
:10C6D00080122040000300000F00010300000F0043
:10C6E00000162040000300000F00010300000F00AF
:10C6F00040162040000300000F00010300000F005F
:10C7000080162040000300000F00010300000F000E
:10C7100000172040000300007F00010300000F000D
:10C7200040002040030300007F00010300000F00D1
:10C73000C0002040030300007F00010300000F0041
:10C7400000012040030300007F00010300000F00F0
:10C7500080012040000001400900000300000F009C
:10C76000010300000F000000004101401300070713
:10C7700000007F0080222440010301000000070721
:10C78000000003000021244001030100010007070D
:10C7900000000300C020244001030100020007073D
:10C7A00000000F0080202440010301000500050562
:10C7B00000017E0040202440010301000600030325
:10C7C00000017E0000202440010301000CC000078E
:10C7D00000000F0000222440010301000D000101B0
:10C7E0000001700040222440010301000E000303F9
:10C7F00000000100C0212440010301000FC0070711
:10C8000000000F00802124400103010010000303F9
:10C810000000040040212440010301000CDF000758
:10C8200000000F00402224400103010070726F7667
:10C830005F726571007265736F7572636573004234
:10C840004F4F5400555047524144450073697A6533
:10C85000006C61756E6368006D6F6E6F746F6E69EA
:10C860006300656E637279707400656E63727970CF
:10C87000745F6B65795F6964006261636B757000FA
:10C88000626F6F745F617574680075706772616460
:10C89000655F6175746800736D69665F69640072D5
:10C8A0006570726F6772616D00737461727400728B
:10C8B0006570726F766973696F6E00626F6F745F17
:10C8C0006C6F61646572006B6579735F616E645F44
:10C8D000706F6C6963696573006D307000706572AC
:10C8E0006D697373696F6E00636F6E74726F6C0045
:10C8F0006B6579006D340073797374656D007379BD
:10C900007363616C6C006D6D696F00726D610064C2
:10C91000657374726F795F667573657300646573B0
:10C9200074726F795F666C617368007072657365AD
:10C930006E74006669726D7761726500636572740A
:10C9400069666963617465006F70656E0064697320
:10C9500061626C656400656E61626C656400616C47
:10C960006C6F77656400646562756700776F756EDC
:10C9700064696E6700626F6F745F7570677261647F
:10C98000650074797065006172726179006974651F
:10C990006D73006E756D62657200696E74656765B2
:10C9A0007200626F6F6C65616E00737472696E679E
:10C9B000006D6178696D756D006D696E696D756D7D
:10C9C000007065726970686572616C730062617392
:10C9D000655F61646472657373006D656D6F726924
:10C9E000657300776F726B666C6173680073666C59
:10C9F000617368007372616D00736F667477617242
:10CA000065006361706162696C69747900464C41CC
:10CA100053485F5043315F53504D00464C4153489B
:10CA20005F50433200464C4153485F504333004609
:10CA30004C4153485F50433400464C4153485F4D8E
:10CA400041494E5F434F444500464C4153485F4D7A
:10CA500041494E5F584F00464C4153485F4D414954
:10CA60004E5F4441544100464C4153485F5355503A
:10CA700045525649534F525900464C4153485F570F
:10CA80004F524B5F53454355524500464C41534826
:10CA90005F574F524B005352414D5F5043305F50F0
:10CAA000524956005352414D5F5043305F505542FA
:10CAB000005352414D5F53504D5F50524956005301
:10CAC00052414D5F53504D5F505542005352414DBE
:10CAD0005F5043315F50524956005352414D5F50B1
:10CAE00043325F50524956005352414D5F504333D9
:10CAF0005F50524956005352414D5F5043345F508E
:10CB0000524956005352414D5F4D41494E005352D8
:10CB1000414D5F44415000534D49465F434F4445AA
:10CB200000534D49465F584F00534D49465F4441BD
:10CB30005441000000002140000025400000014059
:10CB4000000034400000244000003140000032402A
:10CB500000001F41000023400000114001010101BD
:10CB60000101010101101010800019005500F000B2
:10CB70000501053B04101C01010000000FC000006E
:10CB80000004000001010101011D3A5778960008D8
:10CB90002000101208000000001F00000010000F0D
:10CBA000002000023F06080E00080009000A000BE2
:10CBB00024282C30340000001000000090000000F9
:10CBC00088000000080000008000000004F0000061
:10CBD00000F00000400200002005A000D00100018C
:10CBE0008001A0012000000010000000433A5C47D3
:10CBF00069744C61622D52756E6E65725C62756906
:10CC00006C64735C32643334316331325C305C7237
:10CC100065706F5C6379626F6F746C6F616465726D
:10CC20005C70736F633670646C5C64726976657295
:10CC3000735C696E636C7564652F63795F6970639B
:10CC40005F6472762E6800433A2F4769744C6162C4
:10CC50002D52756E6E65722F6275696C64732F321A
:10CC6000643334316331322F302F7265706F2F632C
:10CC700079626F6F746C6F616465722F70736F632C
:10CC80003670646C2F647269766572732F736F757A
:10CC90007263652F63795F6770696F2E6300433A33
:10CCA0005C4769744C61622D52756E6E65725C6290
:10CCB00075696C64735C32643334316331325C3077
:10CCC0005C7265706F5C6379626F6F746C6F6164C6
:10CCD00065725C70736F633670646C5C64726976E5
:10CCE0006572735C696E636C7564652F63795F67E9
:10CCF00070696F2E6800433A2F4769744C61622D4A
:10CD000052756E6E65722F6275696C64732F326432
:10CD10003334316331322F302F7265706F2F637966
:10CD2000626F6F746C6F616465722F70736F6336BE
:10CD300070646C2F647269766572732F736F75728D
:10CD400063652F63795F6970635F6472762E630039
:10CD5000433A2F4769744C61622D52756E6E65724D
:10CD60002F6275696C64732F3264333431633132EE
:10CD70002F302F7265706F2F6379626F6F746C6FD5
:10CD8000616465722F70736F633670646C2F6472A8
:10CD900069766572732F736F757263652F63795F40
:10CDA0006970635F706970652E6300433A2F47694D
:10CDB000744C61622D52756E6E65722F6275696C6E
:10CDC00064732F32643334316331322F302F726504
:10CDD000706F2F6379626F6F746C6F616465722F0F
:10CDE00070736F633670646C2F64726976657273EA
:10CDF0002F736F757263652F63795F70726F742E16
:10CE00006300433A2F4769744C61622D52756E6E10
:10CE100065722F6275696C64732F326433343163C9
:10CE200031322F302F7265706F2F6379626F6F749C
:10CE30006C6F616465722F70736F633670646C2FF2
:10CE4000647269766572732F736F757263652F6391
:10CE5000795F7363625F756172742E6300433A2F6A
:10CE60004769744C61622D52756E6E65722F6275E2
:10CE7000696C64732F32643334316331322F302F55
:10CE80007265706F2F6379626F6F746C6F61646528
:10CE9000722F70736F633670646C2F64726976657D
:10CEA00072732F736F757263652F63795F736D692A
:10CEB000662E6300010010008000E80310000001EE
:10CEC000A00F00FA433A2F4769744C61622D5275E6
:10CED0006E6E65722F6275696C64732F32643334C1
:10CEE000316331322F302F7265706F2F6379626F2B
:10CEF0006F746C6F616465722F70736F63367064EA
:10CF00006C2F647269766572732F736F75726365C7
:10CF10002F63795F736D69665F6D656D736C6F7498
:10CF20002E6300433A2F4769744C61622D52756E2F
:10CF30006E65722F6275696C64732F32643334319D
:10CF40006331322F302F7265706F2F6379626F6F8C
:10CF5000746C6F616465722F70736F633670646C8C
:10CF60002F647269766572732F736F757263652FA4
:10CF700063795F737973636C6B2E6300433A2F4759
:10CF800069744C61622D52756E6E65722F6275699F
:10CF90006C64732F32643334316331322F302F722B
:10CFA00065706F2F6379626F6F746C6F6164657207
:10CFB0002F70736F633670646C2F6472697665725C
:10CFC000732F736F757263652F63795F73797369FC
:10CFD0006E742E6300433A2F4769744C61622D5280
:10CFE000756E6E65722F6275696C64732F3264336F
:10CFF00034316331322F302F7265706F2F63796255
:10D000006F6F746C6F616465722F70736F633670CD
:10D01000646C2F647269766572732F736F757263B7
:10D02000652F63795F737973706D2E6300433A2FB8
:10D030004769744C61622D52756E6E65722F627510
:10D04000696C64732F32643334316331322F302F83
:10D050007265706F2F6379626F6F746C6F61646556
:10D06000722F70736F633670646C2F6465766963BA
:10D0700065732F70736F63362F737461727475707C
:10D080002F73797374656D5F70736F63365F636D53
:10D0900030706C75732E6300010000000600000004
:10D0A000120000000000000000000000000000006E
:10D0B0000000000000000000000000000000000070
:10D0C0000000000000000000000000005B4552521C
:10D0D0005D20546865726520697320616E206572F9
:10D0E000726F72206F63637572726564206475720B
:10D0F000696E6720626F6F746C6F61646572206621
:10D100006C6F772E204D43552073746F707065647B
:10D110002E0A0D005B4552525D204572726F7220DF
:10D120002578207768696C6520656E61626C696E30
:10D130006720434D342061636365737320706F72A1
:10D14000740A0D005B494E465D2054455354204DF2
:10D150004F44450A0D0000000300000001000000DC
:10D160000100000000000000050360000400000052
:10D170000100000000000000010000000604600043
:10D18000080000001CC0020879520D1050534F4394
:10D19000365F464C415348005B494E465D20200AAD
:10D1A0000D005B494E465D202F2A2A2A2A2A2A2A68
:10D1B0002A2A2A2A2A2A2A2A2A2A2A2A2A2A2A2ACF
:10D1C0002A2A2A2A2A2A2A2A2A2A2A2A2A2A2A2ABF
:10D1D0002A2A2A2A2A2A2A2A2A2A2A2A2A2A2A2FAA
:10D1E0000A0D005B494E465D202050536F433620A8
:10D1F0004379426F6F746C6F616465722041707027
:10D200006C69636174696F6E2025752E25752E25F6
:10D21000752E2575200A0D005B494E465D2053741E
:10D22000617274696E6720626F6F746C6F616465A0
:10D23000720A0D005B4552525D20506F6C69637934
:10D2400020636F6E7461696E7320616E20696E6316
:10D250006F727265637420736D69665F6964203DE7
:10D260002025692C2069676E6F7265640A0D005B6A
:10D270004552525D204170706C79696E6720707202
:10D280006F74656374696F6E2073657474696E671B
:10D2900073206661696C6564207769746820636FC8
:10D2A00064652025690A0D005B4552525D20534D8F
:10D2B000494620626C6F636B206661696C6564200F
:10D2C000746F20737461727420776974682065725A
:10D2D000726F7220636F64652025690A0D005B49D7
:10D2E0004E465D20534D4946204D656D6F72792F36
:10D2F000584950204D6F64650A0D005B494E465DEC
:10D3000020736D69665F696420697320736574209A
:10D31000746F20302C20627574205550475241475D
:10D320004520736C6F74207374617274732066721D
:10D330006F6D20534D49462061726561203078251C
:10D3400030386C782E205570677261646520667580
:10D350006E6374696F6E616C69747920646973615E
:10D36000626C65642E0A0D005B494E465D2050726A
:10D370006F63657373696E6720617661696C616262
:10D380006C6520696D616765730A0D005B455252DB
:10D390005D20556E61626C6520746F2066696E64F5
:10D3A00020626F6F7461626C6520696D6167650AE8
:10D3B0000D005B494E465D204A756D70696E6720B1
:10D3C000746F2074686520696D61676520696E20DF
:10D3D000736C6F7420300A0D005B4552525D204E15
:10D3E000657665722073686F756C6420676574205C
:10D3F000686572650A0D005B4552525D20506F6C86
:10D400006963792070617273696E67206661696C07
:10D410006564207769746820636F64652025690AF4
:10D420000D0000008CD10D10E5640D10000000000F
:10D4300024D40D10D8DB0D10000000000000000007
:10D4400007000000010000000000000000000000D4
:10D4500008000000080000000002000000000000BA
:10D4600000000000000000000000000000000000BC
:10D4700000000000000000000B0000003F00000062
:10D48000000000003F00000000000000010000005C
:10D490000E0000001100000000000000000000006D
:10D4A000000000000000000000000000000000007C
:10D4B000000000000000000000000000000000006C
:10D4C000010000000E00000011000000000000003C
:10D4D000000000000000000000000000000000004C
:10D4E000000000000000000000000000000000003C
:10D4F00000000000010000000E000000110000000C
:10D50000000000000000000000000000000000001B
:10D51000000000000000000000000000000000000B
:10D520000000000000000000010000000E000000EC
:10D5300011000000000000000000000000000000DA
:10D5400000000000000000000000000000000000DB
:10D5500000000000000000000000000001000000CA
:10D5600006000000110000000000000000000000A4
:10D5700000000000000000000000000000000000AB
:10D58000000000000000000000000000000000009B
:10D590000100000006000000110000000000000073
:10D5A000000000000000000000000000000000007B
:10D5B000000000000000000000000000000000006B
:10D5C000000000000100000000000000000000005A
:10D5D000000000000000000000000000000000004B
:10D5E000000000000000000000000000000000003B
:10D5F000000000000000000001000000000000002A
:10D60000000000000000000000000000000000001A
:10D61000000000000000000000000000000000000A
:10D6200000000000000000000000000001000000F9
:10D63000060000001D0000000000000000000000C7
:10D6400000000000000000000000000000000000DA
:10D6500000000000000000000000000000000000CA
:10D66000010000000A0000001D0000000000000092
:10D6700000000000000000000000000000000000AA
:10D68000000000000000000000000000000000009A
:10D6900000000000010000000B0000001D00000061
:10D6A000000000000000000000000000000000007A
:10D6B000000000000000000000000000000000006A
:10D6C0000000000000000000433A5C4769744C61B0
:10D6D000622D52756E6E65725C6275696C64735C06
:10D6E00032643334316331325C305C7265706F5C4C
:10D6F0006379626F6F746C6F616465725C70736F75
:10D70000633670646C5C647269766572735C696EB2
:10D71000636C7564652F63795F737973636C6B2ECB
:10D7200068000000F4010000140004010A0009056B
:10D730000800030063010000020000000300000075
:10D740000000000000000018000080000000000041
:10D7500020D90D106000000000000000FFFFFFFF57
:10D760000000000000000000000000002000000099
:10D7700000000000FFFFFFFF0000000000000000AD
:10D78000000000000200000000000000FFFFFFFF9B
:10D79000000000000000000000000000EB0000009E
:10D7A000000200000100000002000000080000006C
:10D7B000020000003500000000000000FFFFFFFF36
:10D7C0000000000000000000000000000500000054
:10D7D00000000000FFFFFFFF00000000000000004D
:10D7E000000000000400000000000000FFFFFFFF39
:10D7F0000000000000000000000000000600000023
:10D8000000000000FFFFFFFF00000000000000001C
:10D81000000000000100000000000000FFFFFFFF0B
:10D8200000000000000000000000000001000000F7
:10D8300003000000000000000000001800000001CC
:10D84000000000006CD90D10600000000000000016
:10D85000FFFFFFFF000000000000000000000000CC
:10D860002000000000000000FFFFFFFF000000009C
:10D87000000000000000000038000000000200006E
:10D88000FFFFFFFF02000000000000000200000098
:10D89000EB00000000020000010000000200000098
:10D8A000040000000200000035000000000000003D
:10D8B000FFFFFFFF0000000000000000000000006C
:10D8C0000500000000000000FFFFFFFF0000000057
:10D8D0000000000000000000040000000000000044
:10D8E000FFFFFFFF0000000000000000000000003C
:10D8F0000600000000000000FFFFFFFF0000000026
:10D900000000000000000000010000000000000016
:10D91000FFFFFFFF0000000000000000000000000B
:10D9200003000000000080009CD70D10FCD70D10F4
:10D93000E4D70D106CD70D100010000054D70D1057
:10D9400084D70D1000010000CCD70D10B4D70D10F6
:10D9500014D80D10000000000100000002000000BB
:10D9600041000000D8D60000C20100000300000002
:10D970000000000190D80D10F0D80D10D8D80D106F
:10D9800060D80D100010000048D80D1078D80D1088
:10D9900000010000C0D80D10A8D80D1008D90D1036
:10D9A0000000000001000000020000008C000000E8
:10D9B000409C0000FA000000010000005CA8020882
:10D9C000010000001400000007008E0001000000AC
:10D9D0005B4552525D204D656D6F7279204D6F64CD
:10D9E000756C652052656164205374617475732091
:10D9F0006661696C65642077697468206572726F0E
:10DA00007220636F64652025690A0D005B455252E0
:10DA10005D204D656D6F7279204D6F64756C65206A
:10DA200051756164456E61626C65206661696C6503
:10DA3000642077697468206572726F7220636F6406
:10DA4000652025690A0D005B4552525D20534D4902
:10DA50004620496E7465727275707420696E6974BF
:10DA600069616C697A6174696F6E206661696C6561
:10DA7000642077697468206572726F7220636F64C6
:10DA8000652025690A0D005B494E465D20534D49CE
:10DA90004620426C6F636B20456E61626C65640D5D
:10DAA0000A0A0D005B494E465D20534D4946204E03
:10DAB0006F726D616C204D6F64650A0D005B45529D
:10DAC000525D20696E76616C6964206172656120C7
:10DAD000257020286964202575290A0D005B4552B0
:10DAE000525D206172656120257520757365206324
:10DAF0006F756E7420756E646572666C6F770A0D53
:10DB0000005B4552525D20496E636F7272656374AB
:10DB100020657261736520696D6167652061646469
:10DB2000726573732030782530386C782C206967E3
:10DB30006E6F7265640A0D005B4552525D20496E3E
:10DB4000636F7272656374207265616420696D61D0
:10DB5000676520616464726573732030782530389E
:10DB60006C782C2069676E6F7265640A0D005B45E6
:10DB700052525D20496E636F7272656374207772D2
:10DB800069746520696D616765206164647265739D
:10DB9000732030782530386C782C2069676E6F726E
:10DBA00065640A0D005B4552525D20696E76616CBA
:10DBB000696420666C6173682049442025643B20B9
:10DBC00065787065637465642025640A0D00000043
:10DBD000000008000002000021640D104D650D10CA
:10DBE00061650D101D640D100D640D100400000022
:10DBF00077C295F360D2EF7F3552500F2CB6798003
:10DC0000000100FF00020001000100030103FF000A
:10DC100001047065726D0074657374004255473B72
:10DC20002063616E27742068617070656E00726594
:10DC300076657274005B494E465D205377617020B3
:10DC4000747970653A2025730A0D005B494E465D74
:10DC5000205377617020747970653A206E6F6E651D
:10DC60000A0D005B494E465D20496D616765207570
:10DC700070677261646520736C6F7431202D3E2073
:10DC8000736C6F74300A0D005B494E465D2045721F
:10DC90006173696E6720736C6F74300A0D005B49A5
:10DCA0004E465D20436F7079696E6720736C6F74A8
:10DCB000203120746F20736C6F7420303A203078DC
:10DCC000256C782062797465730A0D005B57524E9B
:10DCD0005D204661696C65642072656164696E6788
:10DCE00020736563746F72733B20424F4F545F4DD6
:10DCF00041585F494D475F534543544F52533D256B
:10DD000064202D20746F6F20736D616C6C3F0A0D61
:10DD1000005B57524E5D2043616E6E6F74207570CC
:10DD200067726164653A206D6F7265207365637414
:10DD30006F7273207468616E20616C6C6F776564BC
:10DD40000A0D005B57524E5D2043616E6E6F74206A
:10DD5000757067726164653A206E756D62657220D8
:10DD60006F6620736563746F72732064696666659D
:10DD700072206265747765656E20736C6F74730AC8
:10DD80000D005B57524E5D2043616E6E6F742075BF
:10DD90007067726164653A20616E20696E636F6DB1
:10DDA00070617469626C6520736563746F7220774B
:10DDB000617320666F756E640A0D005B494E465DA7
:10DDC00020456E637279707465640A0D005B494E7C
:10DDD000465D204E4F4E2D456E63727970746564BA
:10DDE0000A0D005B4552525D2070616E6963210A25
:10DDF0000D005B4552525D20496D61676520696E7B
:10DE000020736C6F74202564206973206E6F7420FA
:10DE100076616C6964210A0D000000C0E0F0F8FC36
:10DE20006E756C6C0066616C73650074727565006C
:10DE30004142434445464748494A4B4C4D4E4F505A
:10DE40005152535455565758595A61626364656626
:10DE50006768696A6B6C6D6E6F70717273747576DA
:10DE60007778797A303132333435363738390000C3
:10DE700088A102084300504F534958002E00232D1B
:10DE8000302B2000686C4C006566674546470049AA
:10DE90004E4600696E66004E414E006E616E003067
:10DEA0000030313233343536373839414243444516
:10DEB0004600303132333435363738396162636485
:10DEC00065660000202020202020202020282828EF
:10DED0002828202020202020202020202020202032
:10DEE000202020208810101010101010101010107A
:10DEF000101010100404040404040404040410109A
:10DF00001010101010414141414141010101010136
:10DF100001010101010101010101010101010110E2
:10DF2000101010101042424242424202020202020B
:10DF300002020202020202020202020202020210B3
:10DF40001010102000000000000000000000000081
:10DF500000000000000000000000000000000000C1
:10DF600000000000000000000000000000000000B1
:10DF700000000000000000000000000000000000A1
:10DF80000000000000000000000000000000000091
:10DF90000000000000000000000000000000000081
:10DFA0000000000000000000000000000000000071
:10DFB0000000000000000000000000000000000061
:10DFC00000000000496E66696E697479004E614E0A
:10DFD0000000000000000000000000000000000041
:10DFE0000000000000000000000000000000000031
:10DFF0000000000000000000000000000000000021
:10E000000000000000000000000000000000000010
:10E010000000000000000000000000000000000000
:10E0200000000000000000000000000000000000F0
:10E0300000000000000000000080E03779C3414389
:10E04000176E05B5B5B89346F5F93FE9034F384D5E
:10E05000321D30F94877825A3CBF737FDD4F15750A
:10E06000000000000000F03F00000000000024401D
:10E0700000000000000059400000000000408F40F8
:10E08000000000000088C34000000000006AF84063
:10E090000000000080842E4100000000D012634187
:10E0A0000000000084D797410000000065CDCD41FD
:10E0B000000000205FA00242000000E876483742DE
:10E0C000000000A2941A6D42000040E59C30A2427C
:10E0D0000000901EC4BCD64200003426F56B0C43F1
:10E0E0000080E03779C3414300A0D8855734764398
:10E0F00000C84E676DC1AB43003D9160E458E143F9
:10E10000408CB5781DAF154450EFE2D6E41A4B446D
:10E1100092D54D06CFF08044F64AE1C7022DB544B2
:10E12000B49DD9794378EA44050000001900000045
:10E130007D00000054B30D10C6B10D100AB20D10D1
:10E140006EB10D100AB20D10FAB20D100AB20D1018
:10E150006EB10D10C6B10D10C6B10D10FAB20D1092
:10E160006EB10D1066B10D1066B10D1066B10D10D7
:10E1700008B30D107CBA0D107EB90D107EB90D10CC
:10E180009CBC0D1078B90D1078B90D1084BC0D1021
:10E190009CBC0D1078B90D1084BC0D1078B90D1011
:10E1A0009CBC0D1092BC0D1092BC0D1092BC0D10B9
:08E1B000A0BC0D1000000000EE
:08E1B8003C9CFF7F0100000008
:10E1C00000000D1000A00208C0000000E8E10D10E2
:08E1D000C0A00208F0060000E7
:10E1D800ECA702085408000000C002089C010000D7
:10E1E8000DCA0D101BCA0D1025CA0D102FCA0D100F
:10E1F80039CA0D1049CA0D1057CA0D1067CA0D103B
:10E2080079CA0D108BCA0D1096CA0D10A4CA0D102C
:10E21800B1CA0D10BFCA0D10CCCA0D10DACA0D1044
:10E22800E8CA0D10F6CA0D1004CB0D100ECB0D1058
:10E2380017CB0D1021CB0D1029CB0D1000093D0077
:10E2480000127A0000093D000000D00700093D00D7
:10E25800A00F0000040000002CD80D1038D70D10B6
:10E26800EFBE0DD0016F00000000000000000200AA
:10E2780000000000EFBE0DD0026F00000000050096
:10E288000000020000000000EFBE0DD0036F000088
:10E2980000000F000010000000000000BD800D10FD
:10E2A800A9800D1088A1020800000000F4DF0D10FD
:10E2B80014E00D10D4DF0D10000000000000000075
:10E2C8000000000000000000000000000000000046
:10E2D8000000000000000000000000000000000036
:10E2E8000000000000000000000000000000000026
:10E2F8000000000000000000000000000000000016
:10E3080000000000000000004300000000000000C2
:10E3180000000000000000000000000000000000F5
:10E3280000000000000000004300000000000000A2
:10E3380000000000000000000000000000000000D5
:10E348000000000000000000430000000000000082
:10E3580000000000000000000000000000000000B5
:10E368000000000000000000430000000000000062
:10E378000000000000000000000000000000000095
:10E388000000000000000000430000000000000042
:10E398000000000000000000000000000000000075
:10E3A8000000000000000000430000000000000022
:10E3B8000000000000000000000000000000000055
:10E3C8000000000000000000430000000000000002
:10E3D8000000000000000000000000000000000035
:10E3E8000000000000000000A5900D10D1800D1065
:10E3F80000000000C3DE0D107CDE0D10A3DA0D1046
:10E40800A3DA0D10A3DA0D10A3DA0D10A3DA0D109C
:10E41800A3DA0D10A3DA0D10A3DA0D10A3DA0D108C
:10E42800FFFFFFFFFFFFFFFFFFFFFFFFFFFF0000F2
:10E43800010041534349490000000000000000006A
:10E4480000000000000000000000000000000000C4
:10E45800000041534349490000000000000000004B
:10E4680000000000000000000000000000000000A4
:10E4780000000000E9000D10C1000D1080B230B599
:10E48800C00020D0104B07221C682300B0331B8823
:10E498005A43236AD31819680029FCDA3E210B4B2A
:10E4A800062519600A4B0B491960A3210A4BC900BC
:10E4B8005D500A4958505858206A12180020506078
:10E4C8005A58002AFCDA30BDE0AD020804012640A3
:10E4D800080126401E1F0000000026401C05000001
:10E4E80010B54378FF2B11D100F0A2F904000320E6
:10E4F80000F0C6F9C3685A6801231168194311600E
:10E5080011681942FCD1200000F0D2F910BDF7B50E
:10E5180000900020019100F0B3F93F4D06002B68F0
:10E528001A005033B43214681B780419002B5AD0DF
:10E5380000F0AEF9070003281BD000F079F9374A3C
:10E54800374B0500D358002B3EDA364A01213000FC
:10E5580000F0A6F9002837D10198FFF78FFF009B3C
:10E56800002B3ED02368002BFCDB00F069F9040087
:10E578002BE0062000F084F92B68B4331B68C01820
:10E588000368002B02DA284C2000FEBD002000F0B2
:10E598005FF9264B9842F6D00023254A19001268E5
:10E5A800012000F05DF90025A842ECD1002000F020
:10E5B8004FF91E4A1F4B904203D09D42E3D00135CC
:10E5C800F4E79D42B9D1DEE7174C032F05D10121AD
:10E5D800002000F04DF90028F9D1280000F068F972
:10E5E800D2E7154CF1E700F023F90E4A05000121A6
:10E5F800300000F055F9002809D1009B002B08D005
:10E608002368002BFCDB00F01BF90400E5E7064C4F
:10E61800E3E7094CE1E7C046E0AD02080000264008
:10E628001C05000008A80208050052000101880026
:10E6380018A80208F049020001005000F7B56E4D15
:10E6480004002A68536800931300B033198807231D
:10E658004B43126A9B181A68002AFCDA00F030F95A
:10E668002A681300B033198807234B43212800D0A8
:10E6780096E0116A5B180221D8680143D960D9680D
:10E68800C9072FD508208446944460461600D968E7
:10E69800C06F0191116888360818356807684919EC
:10E6A8000D683902FF273F040F40694689882D0A03
:10E6B8002D0639432943D960902103684F4D09013C
:10E6C8002B400B430360136830681B18186805401B
:10E6D8002943196013686246D26F9A181268326823
:10E6E8009B181B68444D2A681300B0331988072308
:10E6F8004B43126A9B1800225A600423404A11694E
:10E708000B431361012C50D030BF2A681300B0337B
:10E71800198807234B43126A9B181A68002AFCDAE7
:10E7280000F0CEF8212842D1296807220B000124E5
:10E73800B0331B8800205A430B6AD318DD68254282
:10E748001CD0080008300D68C06F2C4E28180568CA
:10E75800DB6835401B0C1B061B0C2B4303600B00AE
:10E76800883318680B6818180B6A0568D318DB68B3
:10E778002E401B0E1B023343036020000B6A02214C
:10E78800D218D3688B43D3601B4B1A681300B0337D
:10E79800198807234B43126A9B1800225A60FEBD52
:10E7A800126A9B18174ADA609CE720BFADE7002081
:10E7B800009BFC331B698342E6D1A320124B13490B
:10E7C800134A144FC0000E681D5814680F600627BE
:10E7D8001F503E20106010483E371F501F58002F12
:10E7E800FCDA00980D4FFC3007610E60A321C900C8
:10E7F8005D5001201460C7E7E0AD0208FF00FFFF8D
:10E8080000ED00E024A80208000026400801264088
:10E81800040126401E1F00001C050000AAAAAAAA7F
:10E82800FEE7024A1368002BFCDB70470001264014
:10E8380001B40248844601BC604700BF631D0D1047
:10E8480001B40248844601BC604700BF911E0D1008
:10E8580001B40248844601BC604700BF71280D100E
:10E8680001B40248844601BC604700BF79250D10F9
:10E8780001B40248844601BC604700BFFD270D1063
:10E8880001B40248844601BC604700BF5D1E0D10FC
:10E8980001B40248844601BC604700BF79510D109D
:10E8A80001B40248844601BC604700BF81230D10B3
:10E8B80001B40248844601BC604700BF6B1D0D10BF
:10E8C80001B40248844601BC604700BF2D480D10C2
:10FE0000FC010000211221010000000000000000A0
:10FE100000000D1000FE0000000001007D00000049
:10FE20000100000000DA0F100000000000000000D8
:10FE300000000000000000000000000000000000C2
:10FE400000000000000000000000000000000000B2
:10FE500000000000000000000000000000000000A2
:10FE60000000000000000000000000000000000092
:10FE70000000000000000000000000000000000082
:10FE80000000000000000000000000000000000072
:10FE90000000000000000000000000000000000062
:10FEA0000000000000000000000000000000000052
:10FEB0000000000000000000000000000000000042
:10FEC0000000000000000000000000000000000032
:10FED0000000000000000000000000000000000022
:10FEE0000000000000000000000000000000000012
:10FEF0000000000000000000000000000000000002
:10FF000000000000000000000000000000000000F1
:10FF100000000000000000000000000000000000E1
:10FF200000000000000000000000000000000000D1
:10FF300000000000000000000000000000000000C1
:10FF400000000000000000000000000000000000B1
:10FF500000000000000000000000000000000000A1
:10FF60000000000000000000000000000000000091
:10FF70000000000000000000000000000000000081
:10FF80000000000000000000000000000000000071
:10FF90000000000000000000000000000000000061
:10FFA0000000000000000000000000000000000051
:10FFB0000000000000000000000000000000000041
:10FFC0000000000000000000000000000000000031
:10FFD0000000000000000000000000000000000021
:10FFE0000000000000000000000000000000000011
:10FFF000000000000000000000000000000028D306
:04000005100D4EDFAD
:00000001FF
